:020000040800F2
:1000000000040020A51F0008F71F0008F71F0008C4
:10001000F71F0008F71F0008F71F00080000000086
:10002000000000000000000000000000F71F0008B2
:10003000F71F000800000000F71F0008612C0208ED
:10004000F92D0208FB2D0208FD2D0208012E0208E1
:10005000312E0208332E0208352E0208592E0208CE
:100060007D2E0208A12E0208C52E0208E92E0208E4
:10007000EB2E0208ED2E0208EF2E0208F12E0208E8
:10008000F32E0208F52E0208F72E0208F71F0008CB
:10009000F71F0008F71F0008F71F0008F92E0208D5
:1000A000452F0208472F0208492F02084B2F02084C
:1000B0004D2F0208512F02087D2F0208ED2F020854
:1000C000EF2F0208F12F0208F32F0208F52F020884
:1000D000F92F020869310208913002082D32020816
:1000E000E9320208AD330208AF330208B133020827
:1000F000B53302081D3402081F34020821340208F7
:10010000233402082534020827340208293402085F
:100110002D340208013502080335020805350208AE
:10012000113602081336020815360208173602087F
:1001300000000000000000000000000000000000BF
:1001400000000000000000000000000000000000AF
:10015000000000000000000000000000000000009F
:10016000000000000000000000000000000000008F
:10017000000000000000000000000000000000007F
:10018000000000000000000000000000000000006F
:10019000000000000000000000000000000000005F
:1001A000000000000000000000000000000000004F
:1001B000000000000000000000000000000000003F
:1001C000000000000000000000000000000000002F
:1001D000000000000000000000000000000000001F
:0401E0005FF8E0F1F3
:1001E800032A70B404460D4626D941EA000313F0E9
:1001F800030F13D020782B78984208BF294606D0E1
:100208001EE014F8010F11F8013F984218D1012A95
:1002180002F1FF32F5D1002070BC70470B4604464E
:1002280051F8045B50F8046BAE4204D1043A04461A
:10023800032A0B46F2D81D461046002ADAD1EBE70E
:10024800C01AE9E7032A2DE9F00109D82AB10023E9
:10025800CC5CC45401339342FAD1BDE8F001704735
:100268000B468218014603E02478013301F8014B5C
:1002780011F0030F1C46F7D113F003055DD06E4251
:10028800C5F1040CED009B594FEACC0C08E004348E
:10029800A7593B4607FA0CF748EA070741F8047BD9
:1002A800571A23FA05F8032FF1DC03E014F8013B91
:1002B80001F8013B8A42F9D8CFE753F8404C41F89E
:1002C800404C53F83C4C41F83C4C53F8384C41F8FE
:1002D800384C53F8344C41F8344C53F8304C41F80E
:1002E800304C53F82C4C41F82C4C53F8284C41F81E
:1002F800284C53F8244C41F8244C53F8204C41F82E
:10030800204C53F81C4C41F81C4C53F8184C41F83D
:10031800184C53F8144C41F8144C53F8104C41F84D
:10032800104C53F80C4C41F80C4C53F8084C41F85D
:10033800084C53F8044C41F8044C561A1D460C4618
:10034800403340313F2EB8DC2B460FE053F8101CE9
:1003580044F8101C53F80C1C44F80C1C53F8081CE7
:1003680044F8081C53F8041C44F8041C161B2146C6
:100378001D46103410330F2EE8DC2B4602E02468AB
:1003880041F8044B551A1C46032D03F10403F6DC0F
:1003980090E700BF032AC9B270B408D82AB103464F
:1003A800121803F8011B9342FBD170BC70478218E6
:1003B800044601E004F8011B14F0030FFAD14FF0D2
:1003C800013303FB01F31FE044F8403C44F83C3C94
:1003D80044F8383C44F8343C44F8303C44F82C3C6D
:1003E80044F8283C44F8243C44F8203C44F81C3C9D
:1003F80044F8183C44F8143C44F8103C44F80C3CCD
:1004080044F8083C44F8043C161B254640343F2E6B
:10041800DADC2C4607E044F8103C44F80C3C44F87D
:10042800083C44F8043C161B254610340F2EF2DC19
:1004380001E045F8043B541B032CFADC01E005F805
:10044800011B9542FBD3B0E710F0030F38B5044603
:1004580012D10368A3F1013222EA030313F0803FAB
:100468000AD1031D184653F8042BA2F1013525EAD9
:10047800020212F0803FF5D003782BB1431C1846D6
:1004880013F8012B002AFAD100F076F9204638BD7E
:10049800C9B2F0B4002950D010F0030F10D003787F
:1004A800002B79D0994246D0431C05E013F8012B64
:1004B800002A3FD091423ED013F0030F1846F5D1E1
:1004C800036841EA01270646A3F1013247EA0747D4
:1004D80022EA030212F0803F1DD187EA0303A3F149
:1004E800013222EA030313F0803F14D1043002E002
:1004F80012F0803F0FD1064650F8043BA3F10135B6
:1005080087EA030225EA0303A2F1013413F0803FCE
:1005180024EA0202ECD033783046002B3CD09942D2
:1005280009D0731C01E0914205D0184613F8012B3D
:10053800002AF8D11046F0BC704710F0030F0CD019
:100548000378002BF7D0431C03E013F8012B002A93
:10055800F1D013F0030F1846F7D102680346A2F151
:10056800013121EA020212F0803F0AD10430034629
:1005780050F8042BA2F1013121EA020212F0803F67
:10058800F5D01A781846002AD5D00133184613F842
:10059800012B002AFAD1CEE71846CCE780EA0102FF
:1005A80012F0030F3AD110F0030220F0030021F0FB
:1005B800030150F804CB08BF51F8043B0DD082F07A
:1005C80003024FEAC2026FF07F4323FA02F251F8A6
:1005D800043B4CEA020C43EA020300BFACF10132CF
:1005E8009C4501BF22EA0C0212F0803F50F804CB70
:1005F80051F8043BF2D04FEA0C604FEA1C2C01285A
:1006080028BFB0EB036F08BF1B0AF4D003F0FF0349
:100618004FEA1060A0EB0300704700BF10F0030F13
:100628000AD010F8012B11F8013B012A28BF9A4281
:10063800F4D0A2EB030070474DF8045D4DF8044D6B
:100648004FF0010242EA022242EA024201F0030CA0
:1006580021F0030150F8044B51F8045BBCF1020F80
:1006680026D04BD824F07F4CBCEB152FA4EB02030B
:1006780023EA04030DD113EAC21308BF51F8045B3F
:100688000AD18CEA040CBCEB056F0CD150F8044B72
:10069800E8E74FEA15255CE033F07F4352D10D7847
:1006A8004FEA146C55E04FEA146C05F0FF0550E072
:1006B8004FEA044CA4EB02034FEA1C4C23EA040360
:1006C800BCEB154F17D113EAC21308BF51F8045BEE
:1006D80007D18CEA040CBCEB054F08D150F8044B49
:1006E800E6E71B042ED10D884FEA144C31E04FEA9F
:1006F80005454FEA144C4FEA15452AE004F0FF0C73
:10070800BCEB156FA4EB020323EA04030DD113EA33
:10071800C21308BF51F8045B0AD18CEA040CBCEB85
:10072800052F0AD150F8044BE8E74FEA156510E0A9
:1007380014F0FF0F06D051F8045B4FEA142C25F093
:100748007F4506E04FF000005DF8044B5DF8045B60
:1007580070470CF0FF0205F0FF00012828BF904207
:1007680004BF4FEA1C2C2D0AF3D0A2EB00005DF861
:10077800044B5DF8045B704780EA0102844612F07E
:10078800030F4FD111F0030F32D14DF8044D11F082
:10079800040F51F8043B0BD0A3F101329A4312F035
:1007A800803F04BF4CF8043B51F8043B16D100BF0E
:1007B80051F8044BA3F101329A4312F0803FA4F19F
:1007C80001320BD14CF8043BA24312F0803F04BF26
:1007D80051F8043B4CF8044BEAD023460CF8013B93
:1007E80013F0FF0F4FEA3323F8D15DF8044B70473D
:1007F80011F0010F06D011F8012B0CF8012B002A7B
:1008080008BF704711F0020FBFD031F8022B12F069
:10081800FF0F16BF2CF8022B8CF8002012F47F4F24
:10082800B3D1704711F8012B0CF8012B002AF9D12C
:10083800704700BF20F0030110F00300C0F1000072
:1008480051F8043B00F1040C4FEACC0C6FF00002A5
:100858001CBF22FA0CF213434FF0010C4CEA0C2C8B
:100868004CEA0C4CA3EB0C0222EA030212EACC126B
:1008780004BF51F8043B0430F4D013F0FF0F1FBF3E
:10088800013013F47F4F013013F47F0F18BF01308C
:10089800704700BFF0B4002A46D041EA000313F0C5
:1008A80003032CD1032A07460E4643D904680D6872
:1008B800AC423FD1043A37D0A4F1013525EA04040B
:1008C80014F0803F18BF18462CD1041D0D1D0EE0F2
:1008D80054F8043B55F8041BA3F101308B4220EA7D
:1008E800030027D1043A1FD010F0803F1ED1032AFD
:1008F80027462E46ECD820462946002A1DD00478E3
:10090800013A0D78AC420CD172B18CB1002302E0EF
:1009180093420BD064B1013310F8014FCD5CAC4267
:10092800F6D0601BF0BC70471046FBE70020F9E7E3
:100938002046F7E738463146E1E724782D78F0E796
:1009480041EA000313F0030F0B4670B414BF0024F0
:100958000124032A94BF002404F001040546D4B9F5
:10096800BAB10E782B46013A03F8016B56B1AC1CAC
:100978007AB111F8015F2346013A04F8015C0134A9
:10098800002DF5D12AB19A18002103F8011B9342D2
:10099800FBD170BC7047194653F8044BA4F10136DB
:1009A80026EA040616F0803FDAD1043A45F8044BEB
:1009B800032A1946EFD8D3E701232DE9F0071D468E
:1009C80000264FF0FF37AC1900EB070C8C420DD214
:1009D8001CF805C010F80480E0452ED201252646F3
:1009E800E31BAC198C4200EB070CF1D34FF0010963
:1009F80000264D464FF0FF3C1360AC1900EB0C0885
:100A0800A1420ED918F8058010F804A0C2451AD9D9
:100A180001252646CCEB0409AC19A14200EB0C08D1
:100A2800F0D80CF101000137B8423CBF994638466E
:100A3800C2F80090BDE8F00770470BD00123374695
:100A48001D46F618BFE709D04FF00109B4464D46D8
:100A58004E44D2E79D4205D00135B4E74D4505D057
:100A68000135CAE72B4626460125ACE7A9462646A6
:100A78000125C2E72DE9F04FADF5826D81B014462E
:100A8800074610460DF580628B460C3219461D4606
:100A9800FFF792FF03AE04A901F57E72331F0090A1
:100AA80043F8045F9342FBD14DB1681E0023E25C1A
:100AB800C11A013303AEAB4246F82210F7D1DDF874
:100AC8000C142046009A6118FFF78AFB002877D19A
:100AD8000099814605F1FF380646C1F101020192ED
:100AE8005A46AB4609EB0B0501F1FF3AB81800214D
:100AF800AA1A00F0E5F900284FD1002D00F0C080B7
:100B08007B1903A913F8013C51F82330002B4CD171
:100B1800009B9E4228BF334698450FD903EB090135
:100B2800E05C7A18795C884205D038E012F8011F39
:100B3800E05C884233D101339845F7D8009A964251
:100B480080F0A48007EB090214F80A10534612F843
:100B58000A20914204BF0AEB0901791807D095E0F1
:100B680014F802C011F8010D844503D113465A1E2A
:100B7800B342F5D101369E4200F28D80DDF80C6457
:100B88002A46B144C6EB0B0609EB0B05B818002141
:100B9800AA1A00F095F90028AFD0002071E0019A58
:100BA8000026914499442A46EEE7002EFAD0DDF853
:100BB8000C2493423CBFC2EB0B0306469944F2E770
:100BC800009E4FF000080099AB1BB34238BF334674
:100BD800C1F101026E1E019201F1FF3A5A4689469F
:100BE800AB460133CDF80C3408EB0B05B8180021DF
:100BF800AA1A00F065F90028CFD1002D40D07B1942
:100C080003A913F8013C51F82330002B30D1B1452A
:100C180013D208EB090314F80910FA18FB5C99427F
:100C280018BF4B4627D14B4604E012F8011FE05C81
:100C3800884220D10133B342F7D3BAF1FF3F53467C
:100C48002CD007EB080C14F80A101CF80A20914263
:100C58000CD10AEB0802BA1804E0E05C12F8011D96
:100C6800884203D1013BF8D260460AE0DDF80C3433
:100C780098442A46B8E701992A4688449844B3E735
:100C8800284605B00DF5806DBDE8F08F009B013654
:100C98009E427FF673AF07EB0900F2E707EB080CFB
:100CA8006046EEE72DE9F04F8346037885B00C46A1
:100CB800002B00F0F9800A78A2B106460131012024
:100CC80002E011F8012B8AB1934214BF002000F012
:100CD800010016F8013F0D46002BF2D12B782BB1FD
:100CE8004FF0000B584605B0BDE8F08F0028F9D149
:100CF8000BF101002178FFF7CBFB2D1BA5F10102B9
:100D0800534243EB0203002808BF43F001030746A0
:100D180083B90BEB0508404594BFC0EB08084FF0BA
:100D280001081F2D08D9414622462B46FFF7A2FE8F
:100D38008346D7E78346D5E7294603AA2046FFF727
:100D48003BFE03996118814620464A46FFF748FA58
:100D580000284FD109F1FF33C9F10102064601927B
:100D680082464246C84699460AEB050BB818002148
:100D7800C2EB0B0200F0A4F80028B1D1BBF1000FC0
:100D8800B0D046452CBF334643469D420FD903EBAE
:100D98000A01E05C7A18795C884205D075E012F89F
:100DA800011FE05C884270D101339D42F7D1B04504
:100DB8007DD907EB0A0214F809104B4612F80920EE
:100DC800914202BF09EB0A01AC46791806D06EE0E1
:100DD800A55C11F8010D854203D113465A1EB34292
:100DE800F6D1654601369E4267D8039E5A46B244FC
:100DF800AE1BB9E7C9F10101C9EB0503424600265C
:100E080009F1FF3A88464B4538BF4B4601330393F7
:100E180006EB050BB8180021C2EB0B0200F050F8E6
:100E280000287FF45DAFBBF1000F3FF45BAF4D4589
:100E380012D906EB090314F80910FA18FB5C994259
:100E480008BF4B4605D026E012F8011FE05C884237
:100E580022D101339D42F7D1BAF1FF3F534628D042
:100E680007EB060C14F80A101CF80A20914217D157
:100E78000AEB0602BA1804E0E05C12F8011D884289
:100E88000ED1013BF8D2E3462CE7019A00269244A2
:100E98005A469A4468E74B4646445A46F618B7E716
:100EA800039B5A46F618B3E70D46012016E743465A
:100EB80098E707EB060CE34614E707EB0A0B11E784
:100EC80010F0030F034670B4C9B211D0002A22D023
:100ED80003788B421DD0013A013005E0DAB110F8F1
:100EE800014B013A8C4218D010F0030F0346F5D19C
:100EF800032A14D87AB1187888420ED0541E5D1C83
:100F080003E015F8016B8E4203D0013C2846F8D265
:100F1800002070BC70471046FBE71846F9E741EA25
:100F2800012646EA0646184653F8044B86EA0404A6
:100F3800A4F1013525EA040414F0803F03D1043AF2
:100F48001846032AEFD80346D4E700BF0000000084
:100F5800C1F30A5C0246ACF57E7C2DE9F84FACF192
:100F68000704132C0B4606460F468946804627DCA5
:100F7800002C52DB4FF6FF7CC0F20F0C4CFA04FA3F
:100F88000AEA0105054317D037A3D3E9002300F087
:100F980075F80022002300F0B3FC002856D0002F7B
:100FA80005DD4FF4801353FA04F407EB040929EA2A
:100FB8000A0900264B46324610461946BDE8F88F06
:100FC800332C07DDB4F5806FF6D100F057F80246F0
:100FD8000B46F1E74FF0FF3BACF11B0C2BFA0CFB77
:100FE8001BEA000FE8D020A3D3E9002300F046F85D
:100FF8000022002300F084FC40B3002F0ADD142CEB
:1010080006D00126C4F13404A64016EB080601D325
:1010180007F1010926EA0B0619E013A3D3E9002317
:1010280000F02CF80022002300F06AFC78B1002FB1
:1010380013DB46EA07054FF000094D45C3F6F07982
:101048000CBF2E46002608BFA94600E0B9464B460D
:10105800324610461946BDE8F88F00264FF0004981
:10106800F5E700BFAFF300809C7500883CE4377E4D
:1010780081F0004102E000BF83F0004330B54FEA41
:1010880041044FEA430594EA050F08BF90EA020FAE
:101098001FBF54EA000C55EA020C7FEA645C7FEA41
:1010A800655C00F0E2804FEA5454D4EB5555B8BF64
:1010B8006D420CDD2C4480EA020281EA030382EAD5
:1010C800000083EA010180EA020281EA0303362D67
:1010D80088BF30BD11F0004F4FEA01314FF4801C3A
:1010E8004CEA113102D0404261EB410113F0004F4C
:1010F8004FEA03334CEA133302D0524263EB430303
:1011080094EA050F00F0A780A4F10104D5F1200EA0
:101118000DDB02FA0EFC22FA05F2801841F10001FB
:1011280003FA0EF2801843FA05F359410EE0A5F1CF
:1011380020050EF1200E012A03FA0EFC28BF4CF000
:10114800020C43FA05F3C01851EBE37101F00045B6
:1011580007D54FF0000EDCF1000C7EEB00006EEBC3
:101168000101B1F5801F1BD3B1F5001F0CD349084D
:101178005FEA30004FEA3C0C04F101044FEA4452A4
:1011880012F5800F80F09A80BCF1004F08BF5FEA2B
:10119800500C50F1000041EB045141EA050130BD0B
:1011A8005FEA4C0C404141EB010111F4801FA4F1AE
:1011B8000104E9D191F0000F04BF01460020B1FA03
:1011C80081F308BF2033A3F10B03B3F120020CDA3B
:1011D8000C3208DD02F1140CC2F10C0201FA0CF019
:1011E80021FA02F10CE002F11402D8BFC2F1200C7E
:1011F80001FA02F120FA0CFCDCBF41EA0C01904034
:10120800E41AA2BF01EB0451294330BD6FEA04047C
:101218001F3C1CDA0C340EDC04F11404C4F1200267
:1012280020FA04F001FA02F340EA030021FA04F379
:1012380045EA030130BDC4F10C04C4F1200220FAD0
:1012480002F001FA04F340EA0300294630BD21FA0E
:1012580004F0294630BD94F0000F83F4801306BFD4
:1012680081F480110134013D4EE77FEA645C18BFC8
:101278007FEA655C29D094EA050F08BF90EA020F5F
:1012880005D054EA000C04BF1946104630BD91EA57
:10129800030F1EBF0021002030BD5FEA545C05D15A
:1012A8004000494128BF41F0004130BD14F5800499
:1012B8003CBF01F5801130BD01F0004545F0FE410D
:1012C80041F470014FF0000030BD7FEA645C1ABF42
:1012D800194610467FEA655C1CBF0B46024650EA79
:1012E800013406BF52EA033591EA030F41F40021A5
:1012F80030BD00BF90F0000F04BF0021704730B52B
:101308004FF4806404F132044FF000054FF00001FF
:1013180050E700BF90F0000F04BF0021704730B5C0
:101328004FF4806404F1320410F0004548BF404295
:101338004FF000013EE700BF42004FEAE2014FEAEA
:1013480031014FEA02701FBF12F07F4393F07F4FC5
:1013580081F06051704792F0000F14BF93F07F4FF7
:10136800704730B54FF4607401F0004521F000413A
:1013780020E700BF50EA010208BF704730B54FF0C0
:1013880000050AE050EA010208BF704730B511F0C5
:10139800004502D5404261EB41014FF4806404F1FD
:1013A80032045FEA915C3FF4DCAE4FF003025FEA7F
:1013B800DC0C18BF03325FEADC0C18BF033202EB07
:1013C800DC02C2F1200300FA03FC20FA02F001FA61
:1013D80003FE40EA0E0021FA02F11444C1E600BF00
:1013E80070B54FF0FF0C4CF4E06C1CEA11541DBFB3
:1013F8001CEA135594EA0C0F95EA0C0F00F0DEF87E
:101408002C4481EA030621EA4C5123EA4C5350EA62
:10141800013518BF52EA033541F4801143F48013B3
:1014280038D0A0FB02CE4FF00005E1FB02E506F044
:101438000042E0FB03E54FF00006E1FB03569CF099
:10144800000F18BF4EF0010EA4F1FF04B6F5007F9F
:1014580064F5407404D25FEA4E0E6D4146EB060611
:1014680042EAC62141EA55514FEAC52040EA5E509A
:101478004FEACE2EB4F1FD0C88BFBCF5E06F1ED844
:10148800BEF1004F08BF5FEA500E50F1000041EB7B
:10149800045170BD06F0004646EA010140EA020028
:1014A80081EA0301B4EB5C04C2BFD4EB0C0541EA4A
:1014B800045170BD41F480114FF0000E013C00F35F
:1014C800AB8014F1360FDEBF002001F0004170BD83
:1014D800C4F10004203C35DA0C341BDC04F114049C
:1014E800C4F1200500FA05F320FA04F001FA05F228
:1014F80040EA020001F0004221F0004110EBD370F5
:1015080021FA04F642EB06015EEA430E08BF20EA20
:10151800D37070BDC4F10C04C4F1200500FA04F3C3
:1015280020FA05F001FA04F240EA020001F0004155
:1015380010EBD37041F100015EEA430E08BF20EAC8
:10154800D37070BDC4F1200500FA05F24EEA020E10
:1015580020FA04F301FA05F243EA020321FA04F03F
:1015680001F0004121FA04F220EA020000EBD370F6
:101578005EEA430E08BF20EAD37070BD94F0000FF6
:101588000FD101F00046400041EB010111F4801F2A
:1015980008BF013CF7D041EA060195F0000F18BFDB
:1015A800704703F00046520043EB030313F4801F17
:1015B80008BF013DF7D043EA0603704794EA0C0FD1
:1015C8000CEA135518BF95EA0C0F0CD050EA4106E7
:1015D80018BF52EA4306D1D181EA030101F0004164
:1015E8004FF0000070BD50EA410606BF104619468C
:1015F80052EA430619D094EA0C0F02D150EA013698
:1016080013D195EA0C0F05D152EA03361CBF1046D8
:1016180019460AD181EA030101F0004141F0FE4177
:1016280041F470014FF0000070BD41F0FE4141F4FB
:10163800780170BD70B54FF0FF0C4CF4E06C1CEAFB
:1016480011541DBF1CEA135594EA0C0F95EA0C0FB0
:1016580000F0A7F8A4EB050481EA030E52EA03356B
:101668004FEA013100F088804FEA03334FF080558C
:1016780045EA131343EA12634FEA022245EA1115B9
:1016880045EA10654FEA00260EF000419D4208BF6A
:10169800964244F1FD0404F5407402D25B084FEA17
:1016A8003202B61A65EB03055B084FEA32024FF4C3
:1016B80080104FF4002CB6EB020E75EB030E22BF20
:1016C800B61A754640EA0C005B084FEA3202B6EBE0
:1016D800020E75EB030E22BFB61A754640EA5C008F
:1016E8005B084FEA3202B6EB020E75EB030E22BF1F
:1016F800B61A754640EA9C005B084FEA3202B6EB20
:10170800020E75EB030E22BFB61A754640EADC00DE
:1017180055EA060E18D04FEA051545EA16754FEA40
:1017280006164FEAC30343EA52734FEAC2025FEA5E
:101738001C1CC0D111F4801F0BD141EA00014FF0ED
:1017480000004FF0004CB6E711F4801F04BF0143BE
:101758000020B4F1FD0C88BFBCF5E06F3FF6AFAEDA
:10176800B5EB030C04BFB6EB020C5FEA500C50F16A
:10177800000041EB045170BD0EF0004E4EEA1131ED
:1017880014EB5C04C2BFD4EB0C0541EA045170BDF4
:1017980041F480114FF0000E013C90E645EA060E38
:1017A8008DE60CEA135594EA0C0F08BF95EA0C0F66
:1017B8003FF43BAF94EA0C0F0AD150EA01347FF4AE
:1017C80034AF95EA0C0F7FF425AF104619462CE785
:1017D80095EA0C0F06D152EA03353FF4FDAE1046E8
:1017E800194622E750EA410618BF52EA43067FF439
:1017F800C5AE50EA41047FF40DAF52EA43057FF4C9
:10180800EBAE12E74FF0FF3C06E000BF4FF0010CD3
:1018180002E000BF4FF0010C4DF804CD4FEA410C37
:101828007FEA6C5C4FEA430C18BF7FEA6C5C1BD004
:1018380001B050EA410C0CBF52EA430C91EA030F85
:1018480002BF90EA020F0020704710F1000F91EAE2
:10185800030F58BF994208BF90422CBFD8176FEAB0
:10186800E37040F0010070474FEA410C7FEA6C5C7E
:1018780002D150EA013C07D14FEA430C7FEA6C5C85
:10188800D6D152EA033CD3D05DF8040B704700BFB1
:101898008446104662468C461946634600E000BFFF
:1018A80001B5FFF7B7FF002848BF10F1000F01BDD1
:1018B8004DF808EDFFF7F4FF0CBF012000205DF89C
:1018C80008FB00BF4DF808EDFFF7EAFF34BF012021
:1018D80000205DF808FB00BF4DF808EDFFF7E0FFBA
:1018E80094BF012000205DF808FB00BF4DF808ED0B
:1018F800FFF7CEFF94BF012000205DF808FB00BF72
:101908004DF808EDFFF7C4FF34BF012000205DF853
:1019180008FB00BF4FEA4102B2F1E04324BFB3F530
:10192800001CDCF1FE5C0DD901F0004C4FEAC0024E
:101938004CEA5070B2F1004F40EB830008BF20F032
:101948000100704711F0804F21D113F13872BCBFEC
:1019580001F00040704741F480114FEA5252C2F141
:101968001802C2F1200C10FA0CF320FA02F018BF8A
:1019780040F001004FEAC1234FEAD32303FA0CFCDD
:1019880040EA0C0023FA02F34FEA4303CCE77FEA6C
:10199800625307D150EA01331EBF4FF0FE4040F4B6
:1019A8004000704701F0004040F0FE4040F4000065
:1019B800704700BF80F0004002E000BF81F00041A6
:1019C80042001FBF5FEA410392EA030F7FEA226CDD
:1019D8007FEA236C6AD04FEA1262D2EB1363C1BF6D
:1019E800D218414048404140B8BF5B42192B88BFDC
:1019F800704710F0004F40F4000020F07F4018BFFF
:101A0800404211F0004F41F4000121F07F4118BF1E
:101A1800494292EA030F3FD0A2F1010241FA03FCC6
:101A280010EB0C00C3F1200301FA03F100F00043AE
:101A380002D5494260EB4000B0F5000F13D3B0F176
:101A4800807F06D340084FEA310102F10102FE2AE5
:101A580051D2B1F1004F40EBC25008BF20F0010055
:101A680040EA03007047490040EB000010F4000F03
:101A7800A2F10102EDD1B0FA80FCACF1080CB2EB96
:101A88000C0200FA0CF0AABF00EBC25052421843F5
:101A9800BCBFD0401843704792F0000F81F400019A
:101AA80006BF80F400000132013BB5E74FEA41036D
:101AB8007FEA226C18BF7FEA236C21D092EA030FD9
:101AC80004D092F0000F08BF0846704790EA010F53
:101AD8001CBF0020704712F07F4F04D1400028BF80
:101AE80040F00040704712F100723CBF00F5000062
:101AF800704700F0004343F0FE4040F40000704798
:101B08007FEA226216BF08467FEA23630146420243
:101B180006BF5FEA412390EA010F40F48000704756
:101B28004FF0000304E000BF10F0004348BF4042FC
:101B38005FEA000C08BF704743F0964301464FF038
:101B480000001CE050EA010208BF70474FF0000394
:101B58000AE000BF50EA010208BF704711F00043D5
:101B680002D5404261EB41015FEA010C02BF8446A5
:101B78000146002043F0B64308BFA3F18053A3F504
:101B88000003BCFA8CF2083AA3EBC25310DB01FA4B
:101B980002FC634400FA02FCC2F12002BCF1004FCF
:101BA80020FA02F243EB020008BF20F00100704760
:101BB80002F1200201FA02FCC2F1200250EA4C00B4
:101BC80021FA02F243EB020008BF20EADC707047FA
:101BD8004FF0FF0C1CEAD0521EBF1CEAD15392EA08
:101BE8000C0F93EA0C0F6FD01A4480EA010C4002E4
:101BF80018BF5FEA41211ED04FF0006343EA50103E
:101C080043EA5111A0FB01310CF00040B1F5000F7F
:101C18003EBF490041EAD3715B0040EA010062F12E
:101C28007F02FD2A1DD8B3F1004F40EBC25008BF18
:101C380020F00100704790F0000F0CF0004C08BF36
:101C480049024CEA502040EA51207F3AC2BFD2F103
:101C5800FF0340EAC250704740F400004FF0000311
:101C6800013A5DDC12F1190FDCBF00F0004070474B
:101C7800C2F10002410021FA02F1C2F1200200FA89
:101C880002FC5FEA310040F1000053EA4C0308BF50
:101C980020EADC70704792F0000F00F0004C02BFA1
:101CA800400010F4000F013AF9D040EA0C0093F01C
:101CB800000F01F0004C02BF490011F4000F013B76
:101CC800F9D041EA0C018FE70CEAD15392EA0C0FE4
:101CD80018BF93EA0C0F0AD030F0004C18BF31F04F
:101CE800004CD8D180EA010000F00040704790F025
:101CF800000F17BF90F0004F084691F0000F91F0C9
:101D0800004F14D092EA0C0F01D142020FD193EA8E
:101D18000C0F03D14B0218BF084608D180EA010016
:101D280000F0004040F0FE4040F40000704740F0F2
:101D3800FE4040F4400070474FF0FF0C1CEAD052C0
:101D48001EBF1CEAD15392EA0C0F93EA0C0F69D01C
:101D5800A2EB030280EA010C49024FEA402037D087
:101D68004FF0805343EA111143EA10130CF000407E
:101D78008B4238BF5B0042F17D024FF4000C8B426E
:101D880024BF5B1A40EA0C00B3EB510F24BFA3EB4E
:101D9800510340EA5C00B3EB910F24BFA3EB91031E
:101DA80040EA9C00B3EBD10F24BFA3EBD10340EA78
:101DB800DC001B0118BF5FEA1C1CE0D1FD2A3FF6BE
:101DC80050AF8B4240EBC25008BF20F00100704773
:101DD8000CF0004C4CEA50207F32C2BFD2F1FF0316
:101DE80040EAC250704740F400004FF00003013A47
:101DF80037E792F0000F00F0004C02BF400010F4EB
:101E0800000F013AF9D040EA0C0093F0000F01F0FE
:101E1800004C02BF490011F4000F013BF9D041EA20
:101E28000C0195E70CEAD15392EA0C0F08D1420253
:101E38007FF47DAF93EA0C0F7FF470AF084676E726
:101E480093EA0C0F04D14B023FF44CAF08466EE7FF
:101E580030F0004C18BF31F0004CCAD130F00042CD
:101E68007FF45CAF31F000437FF43CAF5FE700BF25
:101E78004FF0FF3C06E000BF4FF0010C02E000BF4E
:101E88004FF0010C4DF804CD4FEA40024FEA4103F0
:101E98007FEA226C18BF7FEA236C11D001B052EAA6
:101EA800530C18BF90EA010F58BFB2EB030088BF6C
:101EB800C81738BF6FEAE17018BF40F001007047DB
:101EC8007FEA226C02D15FEA402C05D17FEA236CBD
:101ED800E4D15FEA412CE1D05DF8040B704700BF04
:101EE800844608466146FFE70FB5FFF7C9FF00289B
:101EF80048BF10F1000F0FBD4DF808EDFFF7F4FFD4
:101F08000CBF012000205DF808FB00BF4DF808ED6C
:101F1800FFF7EAFF34BF012000205DF808FB00BF8F
:101F28004DF808EDFFF7E0FF94BF012000205DF8B1
:101F380008FB00BF4DF808EDFFF7D2FF94BF012062
:101F480000205DF808FB00BF4DF808EDFFF7C8FF5B
:101F580034BF012000205DF808FB00BF42000ED20C
:101F6800B2F1FE4F0BD34FF09E03B3EB126209D4CC
:101F78004FEA002343F0004323FA02F070474FF082
:101F88000000704712F1610F01D1420202D14FF0F7
:101F9800FF3070474FF00000704700BF00F026F890
:101FA8000C4880F30888002103E00B4B5B58435032
:101FB80004310A480A4B42189A42F6D3094A02E009
:101FC800002342F8043B084B9A42F9D318F072FCFC
:101FD8007047000000C0002028A603080000002069
:101FE8002C1300202C130020486900207047FEE7BE
:101FF80010B586B0002301244FF46022114801A9CE
:1020080001938DF80930039204938DF808408DF8F8
:10201800144027F095FD0B48214627F0B7FD0948E5
:1020280027F0BEFD074827F0C0FD0028FAD1054873
:1020380027F0BFFD034827F0C1FD0028FAD106B0FC
:1020480010BD00BF00240140014610B50D48012213
:10205800032327F0C1FD0B48012127F0B3FD7F20A2
:1020680028F0F0FB0748022127F000FE0028F6D0F0
:102078000448022127F000FE0248BDE8104027F07E
:10208800F2BD00BF002401400C4A0C2303FB0123CE
:1020980010B59C880CB9588010BD5B8803F11304F7
:1020A800844204DA142B07D9133B834204DC0C2343
:1020B80003FB012102238B8010BD00BF042F0020E9
:1020C8000A4B10B500241C7021464FF4E0720848F2
:1020D800FEF760F9074B43F604501C70064B1C7062
:1020E8000FF0CEFE054B187010BD00BFFC15002088
:1020F800C8170020131A00209019002092190020F8
:10210800074B1978013101F01F011970054B1A7836
:102118008A4203D1013202F01F021A70704700BFD1
:1021280090190020131A002010B50E4A0E2303FB45
:1021380000200D4A014614780C4A03FB042300F1E1
:102148000C0251F8044B914243F8044BF9D10A8828
:1021580000211A800E22FEF71DF9BDE81040FFF796
:10216800CFBF00BF0016002090190020C81700201C
:10217800084B1A5C002352FA03F111F0010FD8B290
:1021880002D00130C0B270470133082BF3D10120CF
:10219800704700BFE21A002000F07F0000F574507D
:1021A8002DE9F84309300C46154698460FF068FEAD
:1021B80000284FD043F63C37002638460FF060FE23
:1021C800C0B25FFA86F988B120280FD04FEA5909C2
:1021D8004BF2B77048440FF053FEC0B208B1022862
:1021E80004D10123B340227813432370113743F6F7
:1021F800C43301369F42E0D14BF25E600FF040FEDF
:10220800C0B280B120280ED02B784BF24D6043F03D
:1022180001032B700FF034FEC0B220B1202802D089
:10222800012388F800304BF28F600FF029FEC0B20E
:1022380080B120280ED02B784BF24D6043F002037A
:102248002B700FF01DFEC0B220B1202802D0012350
:1022580088F80030BDE8F883034610465A1E10B5CA
:10226800032A1DD8DFE802F00F0F0209124A52783C
:1022780002F00202D2B2A2B111E00F4A527812F073
:1022880001020ED00BE00D4A927802F04002D2B261
:102298003AB10B4A127802F003029A4200D140B1D7
:1022A80000220848105C984203D00132052AF8D170
:1022B8000021084610BD00BF30630020083B002005
:1022C800F7410020C0170020F8B5064643F63C3514
:1022D800002428460FF0D4FDC0B2E7B268B1202828
:1022E8000BD07F084BF2B77038180FF0C9FD0128E2
:1022F80003D1A04033781843307001341135082CCD
:10230800E7D1F8BD03780E2202FB0313084AD3185D
:102318009978002351FA03F010F00100DAB202D0E4
:10232800501CC0B270470133082BF3D1704700BF6F
:10233800C81700202DE9F04101248C40284A29497A
:102348000346E4B2107891F800C019E0264F0E2633
:1023580006FB0076F178A9B996F80680B8F1000F67
:1023680010D196F80580B8F1000F0BD196F80480CB
:10237800B8F1000F06D1F67926B9013000F01F0038
:10238800054626E0FBB1012B05D0022B06D10E2114
:1023980001FB007739790C4218D014E0042B04D1E2
:1023A8000E2101FB0077B9790CE0032B04D10E2133
:1023B80001FB0077797905E0052B07D10E2101FB98
:1023C8000077F97911B11570BDE8F081013000F09E
:1023D8001F006045BAD11570FF20BDE8F08100BF2D
:1023E800131A002090190020C81700202DE9F04387
:1023F800444D454B2A780E2101FB0232917A85B073
:102408000446984639B101390523594301F56E51FF
:10241800443189B201E043F6C431204604220FF06A
:1024280040FD2B780E2505FB038393F80B80364E71
:10243800344FB8F1000F25D131232371073363716D
:102448003B7801A86B430422F15E06F0CDFB3B7894
:1024580002A805FB03630222997A06F0C5FB3B78C4
:102468000DF10A0005FB03650322697A06F0BCFB3F
:10247800A01D01A90922FEF763FA4FF00F0984F89D
:10248800108012E0B8F1010F0FD132232371053308
:1024980063713B784FF0080905FB036393F901303A
:1024A800E3713B785D43735BA371002320461A46B2
:1024B80012E010F8011BA1F13005EDB2092D04D886
:1024C800EB183029DBB203D004E037395B1800E0A1
:1024D8000A33DBB20132D2B24A45EAD10F21B3FB4B
:1024E800F1F10801411A5B1AC3F10F03DBB2092BA2
:1024F800A35401D8303300E03733A35405B0BDE806
:10250800F08300BFC6170020C8170020024B1A78B6
:1025180042F001021A7070479D1D002008B50C4B4F
:102528000C4A1B780E2101FB0323D97A21B101291A
:102538000CBF0921002100E0102140221346064863
:1025480006F076F9054B1A7842F002021A7008BDB7
:10255800C6170020C8170020931900209D1D0020D1
:10256800034B1A7802F0F8026FF3C3021A7070472F
:102578009D1D0020024B1A7842F004021A70704721
:102588009D1D0020024B1A7842F008021A7070470D
:102598009D1D002038B5114B1C7814F0010502D19F
:1025A800FFF7B4FF05E004F00405EDB21DB9FFF72D
:1025B800E1FF284638BD04F00805EDB215B9FFF76C
:1025C800E1FFF6E704F00204E4B21CB9FFF7A6FF46
:1025D800204638BDFFF7C4FF012038BD9D1D0020EF
:1025E800014B1878704700BFFC15002030B51E4B12
:1025F80085B01B780446002B34D11C4D2B78034141
:1026080013F0010F2ED01A4B1A4A1B780E2101FB2A
:102618000323DA78024112F0010F1CD11B79034120
:1026280013F0010317D110F0010001F1F1014FEA95
:10263800540206D001320091019302926D20FE39B6
:1026480005E001320091019002923C200121032211
:102658000B460FF093FC012313FA04F42B7823EABA
:1026680004042C7005B030BD92190020891900208F
:10267800131A0020C8170020037830B513F0010F93
:10268800144A4FF00E0419D104FB01210133012231
:1026980012FA03F3CD7825EA0303CB7004780D7999
:1026A800A41812FA04F425EA04040C7103789B18A0
:1026B8009A408B7823EA02028A7030BD04FB01211C
:1026C800013B012212FA03F38A7822EA03038B7092
:1026D80030BD00BFC817002010B50023027859008C
:1026E80052FA01F404F00304022C05D1013414FA5F
:1026F80001F122EA010202700133042BEED110BD70
:102708002DE9F04F85B00192BDF838201C46734B77
:102718000092DA78054612F020028B4640F0D88005
:102728008DF80E208DF80F208DF80D20DCB99B78E0
:1027380003F04003DBB21BB101238DF80F3020E01A
:10274800674B1B7803F04003DBB21BB101238DF804
:102758000E3016E00DF10F010DF10E020DF10D0313
:10276800FFF71AFD0DE0012C0BD19B7803F0400315
:10277800DBB223B90DF10F00FFF7A6FD01E08DF8DC
:102788000F409DF80F3023B99DF80E00002800F087
:10279800A28044B905F07F01490001F574510DF19B
:1027A8000A00663109E0012C0AD1E90101F51E4150
:1027B800E8310DF10A0001EB4B0102220FF071FB29
:1027C800BDF90A3013B9002C00F08480009B33B99E
:1027D800444B454F93F80080FFF792FC08E0434BC9
:1027E800434F93F8008008F1010202F01F021A70AB
:1027F8000DF10F00FFF770FF002C44D1BDF80A302F
:1028080069B240F6B83212EA210238BF4FF47A7240
:10281800D2180E2303FB08F3ADF80A20FA529DF8EC
:102828000F90224649460120FE18FFF715FD49463C
:10283800F07022460220FFF70FFD86F802903071F3
:102848009DF80E90224649460420FFF705FD4946AB
:10285800B071824622460320FFF7FEFC05F07F0593
:1028680070713572BAF1000F00D128B1214B1B7875
:1028780013B99DF80D3000E00023F37186F809B014
:10288800019AB2721CE0012C1AD10E2303FB08F343
:10289800BDF80A202046FA529DF80F600022314602
:1028A800FD18FFF7D9FC3146E87000220220FFF737
:1028B800D3FC00232871AE70AB716B71EB71AB72F6
:1028C8000E2303FB0877FC72009B0120BB8102E00A
:1028D800002000E0204605B0BDE8F08F083B00204E
:1028E8003063002090190020C8170020FB15002035
:1028F80000160020821D002073B5154B04461B7876
:102908000E46D3B11348214622F009FE0546A0B968
:10291800012E04F1010606D12046FFF729FC009597
:102928000246812005E02046FFF722FC009502467A
:10293800982031462B46FFF7E3FE2146054822F052
:10294800D8FD0548214602B0BDE8704022F0DCBD44
:10295800911900204E1C0020311A00202DE9F74360
:102968007B4B04461B7843B17A4B1B7803F0240356
:10297800042B02D1002900F0E880774B774F1B78B1
:10298800002B00F0C7807648214622F0C8FD0028B9
:1029980040F0C08007F5C470214622F0C0FD804693
:1029A800002840F0B7803B1993F880302D2B01D0D8
:1029B800532B3AD16B4E357845B30FF0C9FD04F16E
:1029C8000108054650B12046FFF7D2FB337802468E
:1029D8001E33009393204146002307E02046FFF76B
:1029E800C7FB00950246414693202B46FFF788FE19
:1029F8000FF0AEFD014628B1337803201E33009353
:102A0800002101E0009003200A4680E02046FFF7FD
:102A1800AFFB611C02462B4693200095FFF770FE22
:102A28000095032029462A4671E0542B09D12046F7
:102A3800FFF79EFBCDF800800246611C94204346B8
:102A480066E0462B474D20D12E78BEB10FF080FDB1
:102A580004F10109064648B12046FFF789FB2B78A7
:102A680002461E3300939A20494622E02046FFF78B
:102A78007FFB0096024649469A2025E02046FFF74C
:102A880077FB009602469A2039E02E78002E2CD04B
:102A98000FF05EFD04F11C09064660B12046FFF701
:102AA80067FB2B7802461E3369F07F000093C0B2A3
:102AB800611C434609E02046FFF75AFB024669F0CD
:102AC8007F000096C0B2611C3346FFF719FE0FF075
:102AD8003FFD21B2024628B12B7803201E33009314
:102AE800002214E00090032011E02046FFF740FB8D
:102AF800024604F11C0060F07F000096C0B2611C21
:102B08003346FFF7FDFD0096032021463246012398
:102B1800FFF7F6FD124821463F1922F0EAFC97F824
:102B280080302D2B0AD0532B08D0542B06D0462B9F
:102B380004D00D48214622F0F2FC30B10B48214662
:102B480003B0BDE8F04322F0DFBC03B0BDE8F0837A
:102B5800FE1500203C1C002091190020302D00207B
:102B68004E1C0020A61C0020B82E0020461C002069
:102B7800002302780E2101FB0232044901338A182E
:102B88000021062B9170F4D1704700BFC8170020B0
:102B9800064B00201870064B1A78064B1B789A4291
:102BA80002D00146FFF7C6BBFF207047FC15002086
:102BB80090190020131A00200121814038B5114BCB
:102BC800C9431A78104BC9B202F0030203F5E07446
:102BD800012A04D1DD7801EA0505DD7005E0022A45
:102BE80003D11D7901EA05051D710E33A342EFD10A
:102BF800FFF7FCFC43F604500FF042F9034B187042
:102C080038BD00BFF7410020C817002092190020E6
:102C18002DE9F743A34D8DF807002B78A24C1BB183
:102C28002378C2B29A4204D043F604500FF028F930
:102C380028709DF8073023709C4C2278072A00F2F0
:102C48002D81DFE812F008002400360054005D00F2
:102C580072008D00BA00964A3C211170954A1946B7
:102C6800107800F00300FFF765FB934BFF281870FE
:102C780000F0368121F04AF9904B002093F8742037
:102C880042F0010283F874208D4B187064E0884B81
:102C98001B78002B00F0248121F000FB012840F074
:102CA8004D812378142201332370864B01381A7022
:102CB80047E17F4B1B78002B00F01281814E307862
:102CC80008B901234AE021F0E9FA022804D021F0EA
:102CD800E5FA032840F0328121F018F9237804221C
:102CE800013323701D233370774B1A7026E1704B24
:102CF8003C221A707548FFF779FB2378013323705B
:102D08006B4B1B78002B00F0EB806E4B1D78002D71
:102D180040F014811020FFF73DFC002800F01181DD
:102D280023782846013323700BE1614B1B78002B75
:102D380000F0D68005F0E6FD002800F00281614B26
:102D48007D221A705E4B002018705C4B93F874203B
:102D580042F0010283F87420237801332370F0E0F5
:102D6800534B1B78002B00F0BB8021F097FA012809
:102D7800544E03D021F092FA03280FD19DF8072072
:102D8800012111FA02F2524B197821EA02021A7053
:102D980064233370237801332370CFE03078002820
:102DA80040F0CC80484A032323701378013BDBB200
:102DB8001370002B00F09480C3E0404A414E92F813
:102DC8006A201AB13278002A40F0B88000223270A6
:102DD800013212FA03F3DFF8E0803E4F98F8001052
:102DE8004FF00E0909FB0172DB4392F803E0DBB2F6
:102DF80003EA0E0E907882F803E092F804E003EA02
:102E08000E0E0340937082F804E00DF10700FFF7FF
:102E180033FC98F8003009FB0372D278DFF89490FD
:102E28002AB999F8002002F00302012A0AD00E22DA
:102E380002FB03721279B2B999F8002002F003027A
:102E4800022A10D10E2202FB0377BA785AB9224F10
:102E58003A789A4207D11848FFF78AFE3B7801333F
:102E680003F01F033B7099F800009DF8071000F06D
:102E78000300FFF75FFA144B0422FF281A7088F842
:102E88000000164B42D0987800F04000C0B20028ED
:102E98003CD1032323701A33337052E00020207092
:102EA8004FE000BF92190020FF150020FC150020FC
:102EB8008A190020F7410020C61700207C41002015
:102EC800FD150020FA15002088190020931900200C
:102ED80089190020C8170020131A0020083B002079
:102EE800FFF73EFB0023237021F010F82B78013BFD
:102EF800DBB22B702BB1144B9B7803F04003DBB291
:102F0800F3B19DF80700FFF757FE19E09B780E4ACA
:102F180003F04003DBB22BB1136843F400031360E2
:102F2800FFF7CEF8FFF71CFB20F0F0FF002323701B
:102F380043F604500EF0A4FF287001E0002000E0E2
:102F4800FF20BDE8FE8300BF083B0020044B1A7831
:102F58000AB1013A1A701B780BB9FFF72DBE7047FA
:102F680092190020044A054B10781B7803EA501088
:102F780000F00100704700BF083B0020141C00202F
:102F8800044B054A1B781078C3F3400303EA10107A
:102F9800704700BF141C0020083B0020034B044A64
:102FA8001B78D078C3F3800318407047141C0020A6
:102FB800083B0020044B054A1B78D078C3F3C003B4
:102FC80003EA5000704700BF141C0020083B002093
:102FD800044B054A1B78D078C3F3001303EA90002A
:102FE800704700BF141C0020083B0020044B1878D1
:102FF800044BDB785B005BB2DB1103EAD01070474F
:10300800141C0020083B002008B50E2104481DF0C0
:103018007DF9044B5B7803EA000000F0010008BD6D
:103028001C1A0020141C002070B500241BE0304638
:10303800E9B21DF0A9F980B14FF436636343342235
:1030480002FB05330A4AD3181B7A13F0010F04D088
:10305800084B1878C0F3001070BD0135382DE6D143
:103068000134022C02D0E6B20025E0E7002070BD52
:10307800D0420020141C002008B51CF0A1FA034B14
:103088001B7800EA931000F0010008BD141C002012
:10309800044B054A1B78D078C3F3401303EAD000E9
:1030A800704700BF141C0020083B00202DE9F74F93
:1030B800FFF758FF8246FFF763FF8346FFF76EFF6F
:1030C8000190FFF777FF8146FFF782FF0446FFF77D
:1030D800ABFF0546FFF7DCFF8046FFF7CDFF07464D
:1030E800FFF784FF0646FFF78FFF019B45EA0404BC
:1030F8009B0043EA4B0343EA0A0343EAC90343EA52
:10310800481343EA871343EAC61343EA0023E0B2AD
:1031180043EA0010BDE8FE8F044B987800F00F00DA
:10312800A0F10203584240EB03007047821A0020C6
:10313800044B987800F00F00A0F10102504240EBD8
:1031480002007047821A0020044B987800F00F00A4
:10315800A0F10301484240EB01007047821A0020A9
:10316800054B987800F00F00A0F1060CDCF1000088
:1031780040EB0C00704700BF821A0020514AF0B59E
:1031880013781446012B29D003D3022B40F09880E2
:103198005EE04D484D4B047819786FF3C304047012
:1031A80001F0F80158786FF3C301197000F080013D
:1031B800C9B2002900F08480012111709C78062290
:1031C80004F00F04544302464148005D60F30602D0
:1031D8005A701A7861F302021A70F0BD3B494D78B3
:1031E8000B4625F07F00002838D00A7802F0080244
:1031F800D2B222B9344A117841F0080111709A7894
:1032080002F00F02012A04D12F4A117841F001017E
:10321800117015F07F0F53D119789E7801F00700CF
:10322800062206F00F0602FB0606294F5D78BE5DF2
:10323800013066F3060500F007005D7090FBF2F5BB
:1032480002FB150262F30201197002232370F0BD1C
:103258001E494D780B4625F07F0028B98B7860F31E
:1032680003038B701070F0BD174A11786FF3C30118
:103278001170997801F00F01012903D111786FF3CA
:103288000001117015F07F0F1AD119789E7801F09E
:103298000700062206F00F0602FB06060C4F5D78B3
:1032A800BE5D013066F3060500F007005D7090FB17
:1032B800F2F502FB150262F3020119700123237073
:1032C800F0BD00BFD11A0020301A0020821A002059
:1032D800ECA8020810B51F4A1F4B92F9031009B158
:1032E800002231E008B1032119701978032930D878
:1032F800DFE801F00209192C1178002929D01548B6
:1033080081700121197092F90200124920B1134B02
:103318001A786FF3861217E0487808B9032213E089
:1033280088700221197092F902100A4889B90B4A6B
:10333800147861F386141470026861F30F22D1B215
:1033480061F31742026001221A7010BD002111605A
:10335800197010BDA81C00202B1A0020783F0020EF
:1033680070B543F6EF23044643F6F020012A08BF60
:1033780018460D460EF084FD2678C0B20640164C5D
:103388000CD001201DF0E0F943F6EE200EF078FD98
:10339800236860F307036FF30F2314E02B781842B8
:1033A80012D030461DF0D0F90C4B43F6EE201A88A7
:1033B80066F34D321A800EF063FD2368C0B260F3E5
:1033C800070360F30F23236094F9003013B1024B15
:1033D8000F22DA7070BD00BFA81C00203C1C002022
:1033E80008B543F6FB200EF04BFD014B187008BDE5
:1033F8002C1A0020014B1870704700BF1E1C0020BB
:103408002DE9F0474FEAD2084BF25F79C14402F048
:1034180007030446012748460D469F4016460EF00E
:103428002FFDFFB2C1B215B921EA070100E0394307
:1034380008F5D048484608F14E080EF017FD4046FA
:103448000EF01EFDC1B214B921EA070100E03943AC
:1034580040460EF00BFD254305D106483146BDE830
:10346800F04722F051B803483146BDE8F04722F052
:1034780040B800BF851A0020024B1A5C6FF30302A4
:103488001A5470472B1B002070B50C46C10001F57B
:10349800D2411B483F3108220EF003FD0025184891
:1034A8002946EEB222F03BF808B9237823BB154B26
:1034B8002278EB5C1A421FD13046FFF7DDFFF60891
:1034C8004BF25F7030180EF0DBFC05F00703C0B25A
:1034D800184110F0010F0FD10B48294622F01FF8B0
:1034E80050B12946084822F00FF8074B06F5D0409E
:1034F8004E30995D0EF0BAFC0135402DCFD170BD2C
:10350800201C0020E21A0020851A002038B546F653
:10351800960540242046FFF7AFFFA5F5D043094A9A
:10352800563BD15C11F0100F06D06FF30411D15443
:10353800284600210EF09AFC0134E4B20135E92C4A
:10354800E8D138BD2B1B00203F287FB5054607D89A
:1035580000F5E440C1300EF093FCC3B22BB930E162
:103568009C4A1478002C00F031819B4E725D02F069
:103578000F014C1C04F00F0464F303023F2D725535
:1035880033D8002C00F0228101339C4240F01B818B
:10359800924B5A1992F88020522A725D03D161F336
:1035A800030272550FE16FF30302EC081B19725501
:1035B80093F8902105F0070352FA03F313F0010F73
:1035C80040F003812946864821F093FF844B04F597
:1035D800D040195D4E3001240EF048FC2D1902230D
:1035E80000930194029518209EE0002C00F0EE80D4
:1035F800784B1B7801339C4240F0E580735D05F5FC
:10360800D0406FF303035630012173550EF02EFCA2
:10361800735D43F010037355A5F14003DBB2072B2C
:1036280007D8042200920133023201920293192032
:10363800B3E0A5F14803DBB2072B07D804220092B8
:1036480001330332019202931A2061E0A5F150037D
:10365800DBB2062B07D80422009201330332019211
:1036680002931B2054E0A5F15703DBB2032B07D8C4
:10367800042200920133033201920293212047E091
:10368800A5F15B03DBB2012B07D8042200920133BA
:1036980002320192029322207FE05D2D06D104239D
:1036A80000930193043B0293284684E05E2D07D1E2
:1036B8000423009301330193053B02935E207AE0D3
:1036C800A5F15F03DBB26F2B09D804220092013306
:1036D80092180192029333200121053A6DE005F119
:1036E8003103DBB2072B07D80422009201330332DF
:1036F800019202935F200BE005F12903DBB2012B55
:1037080009D8042200920133033201920293602007
:103718000121043A51E0DA2D0CD10423009301244D
:10372800043B0194029361202146032223460EF0B4
:1037380025FC4BE0D92D07D104230093023B0193CC
:10374800023B0293622036E0DD2D08D1042300936A
:103758000322043B01920293632001212DE0DB2D1B
:1037680006D104230093043B01930293642022E0D2
:10377800DC2D06D104230093043B019302937020AF
:1037880019E005F12203DBB2032B09D804220092C9
:10379800013302320192029368200121033A0CE0BE
:1037A8001E35EDB2062D10D80423009301350233DF
:1037B800019302956A20012103220B460EF0DEFBDD
:1037C80003E01C4602E0002400E00124204604B087
:1037D80070BD00BF000000202B1B0020302D0020F2
:1037E800851A0020024B185CC0F30010704700BF18
:1037F8002B1B0020F8B508220E4600210746FCF7CF
:10380800C9FD46F63F1500243378234113F0010F14
:1038180008D02946064808220EF043FB38460449DA
:1038280021F035FE01340835082CEDD1F8BD00BF74
:103838002A1C0020024846F64E0108220EF031BB31
:10384800851A002070B5044600F56A5044300EF021
:1038580017FB0B4D06462B7813F0010F02D1CC2035
:1038680022F082FC2B8843F001032B80054B1E5568
:10387800054B13F8242042F0010203F8242070BD00
:103888003C1C0020621A0020411A0020024B185CE0
:10389800084100F001007047E21A002070B50546A3
:1038A8000024094BE0B2E618E35C4BB12946FFF768
:1038B800EDFF28B1002333700448214621F024FE8F
:1038C8000134402CEDD170BD5E1C0020721A00201E
:1038D80038B5054600242846E1B2FFF7D7FF10B1F6
:1038E800044BE35C23B90134082CF4D1002038BD23
:1038F800012038BD621A002038B505460EF028FEB2
:10390800A0B100242846E1B2FFF7C0FF40B1084B40
:1039180013F8243013F0010F02D0064BE35C23B1F7
:103928000134082CEED1002038BD012038BD00BF7D
:10393800411A0020621A0020F8B5114800214022DF
:10394800FCF728FD46F63F15002401270D482946B7
:103958000822A7400EF0A5FAFFB200260948314612
:1039680021F0DDFD20B1064BF25C47EA0202F25479
:103978000136402EF2D101340835082CE5D1F8BDC6
:10398800E21A00202A1C00202DE9FF4100263446B7
:10399800B0461A4B1B78234113F00102184B23D071
:1039A800184F1D5D17F82430A84538BFA84613F0F6
:1039B800010F1AD0CDB965F3000307F8243023B2FC
:1039C8000122F71902935B2029462B4600920195A4
:1039D8000EF0D4FA7B78B878F9781843621C2B4635
:1039E8000095FEF78DFE00E01A5501340436082CC8
:1039F800CFD1054B83F80080BDE8FF812C1A002049
:103A0800621A0020411A00202A1A002010B50C4B17
:103A18001B78A3B10B4B1B788BB100240A482146B5
:103A280021F07DFD40B10948214621F078FD18B903
:103A380020460121FEF792FF0134402CEED110BD43
:103A480091190020FE150020461C00202A24002081
:103A58002DE9F043324C334A238800266FF386134E
:103A68006FF3C4032380304B304F85B016701E703F
:103A78009146984617F8013B5BB32278D20052B2C0
:103A880043EAA2122388402E62F3C40343F04003A2
:103A980023801ED000253046E9B2FFF7F7FEA8B113
:103AA80017F8013C13F0010F06D00122AA4099F83B
:103AB80000100A4389F8002013F0020F06D00123F2
:103AC800AB4098F80020134388F800300135082DE2
:103AD800E1D10136F6B2412ECCD1237803F040056E
:103AE800EDB2D5B903F02403042B0BD1FFF78EFFF9
:103AF800FF2300934020294601222B460195029579
:103B08000EF03CFA238800226FF345136FF382030B
:103B18006FF3C4032380064B1A7005B0BDE8F08329
:103B28003C1C0020CC3E0020FC3E0020901A0020C7
:103B38001F1C002010B500240548214621F0EFFC89
:103B480008B9044BE0540134402CF5D110BD00BF36
:103B5800161C0020901A002010B5127804469DF813
:103B68000810DAB1D3B111B10D4921F085FCACB11F
:103B7800082246F64E010B480EF093F921460948F3
:103B880021F085FC0749082246F64E000EF083F91D
:103B980005480449BDE8104021F08FBC10BD00BFA6
:103BA800C82E0020141A0020851A002030B5064BB4
:103BB80004781D7824EA05040C7001781B7823EA40
:103BC8000103137030BD00BF2C1A002038B50A4D10
:103BD800002415F8013F2D2B09D0532B07D0542B67
:103BE80005D0462B03D00548214621F08DFC013431
:103BF800402CEED138BD00BFAF2D0020461C002060
:103C080010B50F4821F030FC00240E48214621F061
:103C180086FC80B10C4BE31893F88030482B06D013
:103C280003D82D2B03D0462B00E0542B03D1044896
:103C3800214621F05EFC0134402CE6D110BD00BFC6
:103C4800D21A0020461C0020302D0020094A0A4BB9
:103C5800117831B1997801F00F01814201D000212A
:103C680011709A7860F303029A705A7842F08002D1
:103C78005A707047D11A0020821A00202DE9F043AB
:103C88001F4685B07B4BDDF83090154604461A7800
:103C980088460023784911F8231011F0010F03D04A
:103CA8000121994022EA01020133082BF2D1734B1A
:103CB8001A70002C00F0878014F0010F0CD001213D
:103CC800FF230026009352200B460A4601960296CF
:103CD8000EF054F96A4B1E7014F0020F0DD0FF233A
:103CE80001210093FF3B019302930A460B465320A0
:103CF8000EF044F9624B01221A7014F0040F0DD033
:103D0800FF2301210093FF3B019302930A460B46D0
:103D180054200EF033F95A4B02221A7014F0080F8F
:103D28000DD0FF2301210093FF3B019302930A4624
:103D38000B4655200EF022F9514B03221A7014F04D
:103D4800100F0DD0FF2301210093FF3B0193029335
:103D58000A460B4656200EF011F9494B04221A70F8
:103D680014F0200F0DD0FF2301210093FF3B019396
:103D780002930A460B4657200EF000F9404B0522E5
:103D88001A7014F0400F0DD0FF2301210093FF3B60
:103D9800019302930A460B4658200EF0EFF8384B71
:103DA80006221A7014F0800F0DD0FF230121009312
:103DB800FF3B019302930A460B4659200EF0DEF8AA
:103DC8002F4B07221A70B8F1000F1CD02C4B092278
:103DD8001A7000243846214621F0A1FB60B1FF2368
:103DE8000093FF3B0193631C1BB2012102935A20ED
:103DF8000A460B460EF0C2F821463846013421F037
:103E080083FB402CE6D1CDB100244846214621F061
:103E180086FB80B1012D0ED104230093631C1BB2D5
:103E28000826029374202B462946032201960EF099
:103E3800A5F8134B1E700134702CE6D10F481149B8
:103E4800114AFFF7B3FE114B00221A70013200929B
:103E580006320192F83202920A490B4A074809F0E1
:103E680019FE0B4B3C2251201A7005B0BDE8F043F7
:103E78000EF05ABC2C1A0020411A0020081E0020FF
:103E8800F1670020F11E0020E41E0020CD1D002057
:103E9800611A002037B5FFF709F904460E4821F0EA
:103EA80011FBD0F1010538BF00250C480E211CF08C
:103EB8002DFA10B114F4807F03D124B95DB12246E4
:103EC80002E0012200E00022044B2046009329462C
:103ED800014BFFF7D3FE3EBD231B00201C1A002018
:103EE800054B03EBD00393F8903100F0070053FA29
:103EF80000F000F001007047302D002010B50F4B86
:103F080004461B7813F0010315D0FFF7E1FC28B92C
:103F18000B4B1B1993F88030462B0DD10EF018FB74
:103F280018B92046FFF7DCFF30B10648214621F0DA
:103F3800E0FA012010BD184610BD00BF3C1C00204F
:103F4800302D0020231B0020024B1878003818BFA2
:103F580001207047611A002010B5034C04EB83035D
:103F680058709970DA7010BD411A002010B50024FD
:103F78000948002100190E220E34FCF70BFAB4F59B
:103F8800E07FF5D1054A00231370054A00219952B4
:103F98000233AA2BF9D110BD00160020FB15002012
:103FA800661F0020044B187800F02400A0F10403D9
:103FB800584240EB030070473C1C00207FB5474B3C
:103FC80004461B780E46AA2B78D04548214621F096
:103FD800A6FA0546002871D12046FFF78FFF002872
:103FE8006DD14048214621F09AFA50B93E48214601
:103FF80021F095FA054620B92046FFF7A5FA0028D2
:104008005DD13A4B1B7823B9394B1B7813F0010F5C
:1040180009D1384BDB7803F02003DBB21BB9364BF0
:10402800032283F84020012E05D82E48214621F08E
:1040380076FA40B142E0022E07D12B48214621F002
:104048006EFA10B13AE0274800E02748214621F0EF
:1040580050FA2A48214621F057FA022E15D1012597
:10406800294603222B4600964A2066190195029696
:104078000DF084FF2046FEF77BF800230246314608
:1040880018200093FEF73CFB19E0012E09D102230A
:104098000093631C02930196122031460322334693
:1040A80009E07EB90121022300936318029301916C
:1040B800112003220B460DF061FF03E0002528467E
:1040C80004B070BD2046FEF753F8024601200023D5
:1040D800211800930125FEF713FBF0E71E1C0020B2
:1040E800851A0020311A00209E1C00202C1A00205E
:1040F800611F0020083B0020901A00204E1C002061
:104108002DE9FF4704460D467548214621F007FA78
:104118008146002840F0DF802146714821F0E9F906
:104128007048214621F0F0F96F4E0DBB01274FF082
:104138000208E31902934246032039463B46CDF86C
:10414800008001970DF01AFF327862B10EF000FA84
:10415800024630B1337840461E33009321462A4642
:1041680004E0009000E00092404621463B4628E0EB
:10417800012D2BD15D4B04F5E440C1301F5D0DF0DE
:104188007FFE07F00F07874209DA631C02220293B9
:104198000E2029462B46009201950DF0EFFE32784D
:1041A80092B10EF0D5F9024638B14F4B0D201B786D
:1041B80021461E330093002202E000900D20214684
:1041C8000123FEF79DFA5EE00092F7E7022D0BD17E
:1041D80001230193E3180293142049462A464B46CB
:1041E80000950DF0CBFE4EE0032D4CD101272A4659
:1041F8004FF0020804EB070A4D2039463B46CDF83C
:1042080000800197CDF808A00DF0B8FE35783DB3D1
:104218000EF09EF9024630B1337840461E330093C3
:1042280021464A4602E00090214640463B46FEF7BA
:1042380067FA0EF08DF9671C054648B12046FDF770
:1042480097FF337802461E3300931A2039462CE034
:104258002046FDF78DFF0095024639461A202DE0CD
:1042680021462A463B4640460095FEF749FA204635
:10427800FDF77EFF514602462B461A200095FEF7B1
:104288003FFA384628E03578EDB10EF061F904F1CF
:104298001C06054658B12046FDF76AFF124B024638
:1042A8001B7830461E330093611C002307E020462C
:1042B800FDF75EFF009502463046611C2B46FEF76F
:1042C8001FFA012008E02046FDF752FF009502463C
:1042D80004F11C00F1E7002004B0BDE8F08700BF3E
:1042E800461C00204E1C0020A61C00202B1B002072
:1042F800064B1B1893F84001492804D0452814BFE1
:104308000320022070470120704700BF302D002095
:104318002DE9F041244F00243C702448214621F027
:10432800FEF8E5B2224B002837D01E5D3B789E424E
:1043380000D303B93E70002E30D131461C484022CC
:10434800FCF728F81B4B1C4803EBD50393F888812E
:1043580004F0070348FA03F8214608F0010821F0A1
:10436800DEF868B9B8F1000F02D02846022101E052
:1043780028463146FFF7C4FE28460EF0D5F90DE071
:10438800B8F1000F0AD12846FFF7B2FF0B4BDB78D4
:1043980003F02003DBB20BB9094B18550134402C4C
:1043A800BBD1BDE8F08100BFA61C0020721A002016
:1043B8005E1C0020302D0020461C0020083B0020F9
:1043C800901A00202DE9F04F914B8BB01B7813F019
:1043D800010F06D08F4B1A786FF386121A7001F00E
:1043E80032BB8D498D4A0B7810788D4D984218BF95
:1043F8008C49137018BF0B706B7803F00803DBB29D
:104408004BB143F6CF200DF03BFD864B18702B883F
:104418006FF3CB232B80844B1B78AA2B08D18349BD
:10442800AA3B0B702B8843F080032B8000F02CBF35
:104438006A787B4B02F01002D2B27D4CA2B11A8886
:104448006FF30C321A807B4B1B7823B97A4B1B789D
:1044580013F0010F08D1E37803F02003DBB21BB996
:10446800764B032283F840202368754F6FF3186357
:1044780023603A7802F00202D2B232B96B494A7824
:104488001AB16B4A43F080731360E67816F00106A0
:1044980048D05D20FFF7A6F900285AD16B78DFF8DD
:1044A800808103F00203DBB22BBB5D30FFF74CF8D1
:1044B800064600BBB8F80030012143F40073A8F8A1
:1044C8000030042303220093019302900B460D2031
:1044D8000DF054FD45200EF027F9314601223346F0
:1044E8000D200096FEF70CF90920314632460123CB
:1044F8000096FEF705F96B7803F00203DBB243B3CD
:104508004C4B1B7823B94C4B1B7813F0010F20D16F
:10451800E37803F02003DBB2DBB9484B032283F8CE
:10452800402016E06B7803F00203DBB26BB1314632
:10453800324601230A200096FEF7E2F88D20314624
:10454800012233460096FEF7DBF82B886FF34923E8
:104558002B802368354A6FF35963236093787BB1C6
:10456800D37823B93B7813F00C0F05D108E03B78DA
:1045780003F00C03042B03D0236843F0007323607B
:10458800E17801F00201C9B200295BD05E20FFF793
:1045980029F9002865D16B78214F03F00403DBB2B9
:1045A800EBB95E30FEF7D0FF0646C0B93B88012163
:1045B80043F480633B800423009301330322019377
:1045C80002900B4617200DF0D9FC45200EF0ACF8F0
:1045D8000D203146012233460096FEF791F86B789C
:1045E80003F00403DBB2002B3BD0124B1B7823B93A
:1045F800114B1B7813F0010F33D1E37803F020033C
:10460800DBB273BB0D4B032283F8402029E000BFC7
:10461800091E0020783F0020281C0020291C0020AB
:104628003C1C0020A71C00201E1C00202C1300206E
:10463800083B00202C1A0020611F0020901A00203F
:104648002E2D00206B7803F00403DBB22BB18D20F4
:1046580001220B460091FEF753F82B886FF38A234B
:104668002B8023684FF05F0B6FF3DF732360002606
:1046780096E00698F9B21BF087FE002875D04FF433
:1046880036637343342202FB0733A749A8F15E0A55
:10469800CB1803F108021B7A5FFA8AFA13F00103B8
:1046A8004DD02368404643F0004323600592FFF74E
:1046B80099F8059A002864D1937813F0040F20D153
:1046C8004046FEF741FF059A8146D0B9937801210B
:1046D80043F00403937004230093DB18032201932F
:1046E80032200B46CDF808A00DF048FC4A200EF009
:1046F8001BF80C20514601224B46CDF80090FDF7DF
:10470800FFFF4FF436637343342202FB0733864AB4
:10471800D3189B7A13F0040F33D0844B1B7823B93A
:10472800834B1B7813F0010F2BD1E37803F02003A0
:10473800DBB233BB7F4B032283F8402021E0927821
:1047480012F0040F05D08C20514601220093FDF78A
:10475800D7FF4FF436637343342202FB07337249A1
:10476800CB189A7A6FF382020AE04FF436637343E8
:10477800342202FB07336C4AD3189A7A60F3820218
:104788009A72013708F10108382F5FFA88F87FF428
:1047980070AF01360BF1380B022E5FFA8BFB04D099
:1047A800F3B20693D846002763E72368624923F0EB
:1047B80080636FF39E7323600B79002B00F02B84CA
:1047C8005E4ADFF87CB106924FF0CF0800271BF84D
:1047D800011F3E460137002952D0236808F1710AAB
:1047E80043F080635FFA8AFA23605046FEF7FAFFC7
:1047F80000285CD129237343DFF8489119F8032076
:1048080012F0100F23D150460593FEF79DFE059B2D
:104818008246E0B919F80320012142F0100209F894
:10482800032004230093023301933BB20322029333
:104838000F200B460DF0A2FB45200DF075FF0D2053
:10484800514601225346CDF800A0FDF759FF292310
:10485800734319F8033013F0100F28D0334B1B782B
:1048680023B9334B1B7813F0010F20D1E37803F001
:104878002003DBB2DBB92F4B032283F8402016E07C
:1048880029237343DFF8BC9019F8033013F0100F95
:1048980005D08D2001220B460091FDF731FF292319
:1048A800734319F803206FF3041209F80320069ADA
:1048B80012F8011F0692002946D02368404643F0AB
:1048C80080432360FEF78EFF002854D14FF029095A
:1048D80009FB06F9DFF86CA01AF8093013F0200F6D
:1048E80049D14046FEF730FE0646002843D11AF863
:1048F8000930012143F020030AF80930042300930A
:10490800033301933BB2032202934B200B460DF075
:1049180035FB50200DF008FF19203146012233469F
:104928000096FDF7EDFE26E0D04200202C1A00206C
:10493800611F0020901A00202C1300203B3D00200E
:10494800673D0020793D002029237343DFF8AC92AE
:1049580019F8033013F0200F05D0992001220B46D7
:104968000091FDF7CDFE29235E4319F806306FF359
:10497800451309F8063008F10108082F5FFA88F88E
:104988007FF425AF984ADFF878B206924FF05008C6
:10499800083F1BF8011F3E460137002952D0236803
:1049A800A8F16E0A43F080635FFA8AFA23605046E2
:1049B800FEF718FF00285CD122237343DFF84492E6
:1049C80019F8032012F0400F23D150460593FEF743
:1049D800BBFD059B8246E0B919F80320012142F08E
:1049E800400209F8032004230093023301933BB2E9
:1049F8000322029369200B460DF0C0FA45200DF002
:104A080093FE0D20514601225346CDF800A0FDF734
:104A180077FE2223734319F8033013F0400F28D090
:104A2800724B1B7823B9724B1B7813F0010F20D1FE
:104A3800E37803F02003DBB2DBB96E4B032283F883
:104A4800402016E022237343DFF8B89119F80330A9
:104A580013F0400F05D08D2001220B460091FDF781
:104A68004FFE2223734319F803206FF3861209F8C7
:104A78000320069A12F8011F0692002935D02368F0
:104A8800404643F080432360FEF7ACFE002843D144
:104A98004FF0220909FB06F9DFF868A11AF8093076
:104AA80013F0200F38D14046FEF74EFD064698BB5E
:104AB8001AF80930012143F020030AF809300423C9
:104AC8000093033301933BB20322029310200B4659
:104AD8000DF054FA50200DF027FE1920314601221E
:104AE80033460096FDF70CFE16E022237343DFF8E9
:104AF800149119F8033013F0200F05D099200122E2
:104B08000B460091FDF7FCFD22235E4319F80630A1
:104B18006FF3451309F8063008F10108072F5FFA0B
:104B280088F87FF436AF344ADFF8DCB006924FF0ED
:104B38005708073F1BF8011F3E460137002967D079
:104B48002368A8F1790A43F080635FFA8AFA236040
:104B58005046FEF747FE002871D122237343DFF841
:104B6800AC9019F8032012F0400F23D1504605935A
:104B7800FEF7EAFC059B8246E0B919F803200121FB
:104B880042F0400209F80320042300930233019302
:104B98003BB20322029367200B460DF0EFF9452044
:104BA8000DF0C2FD0D20514601225346CDF800A05C
:104BB800FDF7A6FD2223734319F8033013F0400FC5
:104BC8003DD00A4B1B7823B9094B1B7813F0010F12
:104BD80035D1E37803F02003DBB283BB054B032216
:104BE80083F840202BE000BF0B3B00202C1A00204C
:104BF800611F0020901A00206B3B0020793D0020A7
:104C0800253D0020383C00205F3B00208C3B0020E5
:104C180022237343DFF8B89319F8033013F0400FD9
:104C280005D08D2001220B460091FDF769FD222356
:104C3800734319F803206FF3861209F80320069AC4
:104C480012F8011F0692002935D02368404643F028
:104C580080432360FEF7C6FD002843D14FF02209A8
:104C680009FB06F9DFF868A31AF8093013F0200FDA
:104C780038D14046FEF768FC064698BB1AF809305A
:104C8800012143F020030AF8093004230093033379
:104C980001933BB2032202931F200B460DF06EF9DD
:104CA80050200DF041FD192031460122334600966F
:104CB800FDF726FD16E022237343DFF8149319F855
:104CC800033013F0200F05D0992001220B460091E4
:104CD800FDF716FD22235E4319F806306FF34513DE
:104CE80009F8063008F10108042F5FFA88F87FF404
:104CF80021AF4FF000084FF05B094FF0D70A464646
:104D0800AA4B08F10108F15CA94F002949D0236892
:104D1800484643F080632360FEF764FD002852D1C3
:104D280024237343FA5C12F0200F22D148460593DE
:104D3800FEF70AFC059B8346D8B9FA5C012142F0CC
:104D48002002FA5404230093023301930FFA88F3E4
:104D58000322029320200B460DF010F945200DF098
:104D6800E3FC0D20594601225B46CDF800B0FDF763
:104D7800C7FC24237343FB5C13F0200F23D08D4B17
:104D88001B7823B98C4B1B7813F0010F1BD1E378E8
:104D980003F02003DBB2B3B9884B032283F8402029
:104DA80011E024237343FB5C13F0200F05D08D2002
:104DB80001220B460091FDF7A3FC24237343FA5C00
:104DC8006FF34512FA547E4BF15C002933D0236807
:104DD800504643F080432360FEF704FD00283ED18F
:104DE800242303FB06735A7812F0200F37D150465C
:104DF8000593FEF7A9FB059B834680BB5A780121E2
:104E080042F020025A7004230093033301930FFAEF
:104E180088F3032202934C200B460DF0AFF8502084
:104E28000DF082FC1920594601225B46CDF800B0EE
:104E3800FDF766FC13E0242303FB06735B7813F08D
:104E4800200F05D0992001220B460091FDF758FC50
:104E5800242303FB06735A786FF345125A70594B93
:104E68002422F35C002B3CD07243BB5CC3F3801B51
:104E7800BBF1000F1DD154490978D1B143F040036B
:104E8800BB5404230093DB18012101930FFA88F324
:104E9800032202932F200B460DF070F847200DF0E7
:104EA80043FC0920414601225B46CDF800B0FDF7DE
:104EB80027FC24237343FB5C13F0400F22D03D4BA7
:104EC8001B7823B93C4B1B7813F0010F1AD1E378F8
:104ED80003F02003DBB2ABB9384B032283F8402040
:104EE80010E07243BA5C12F0400F05D089204146A9
:104EF80001220093FDF704FC24237343FA5C6FF34B
:104F08008612FA5401360AF1010A09F10109022E42
:104F18005FFA8AFA5FFA89F97FF4F2AEDFF8B4A093
:104F28004827023E1AF8013FB04601362BB9274BF5
:104F3800F31813F8011C002950D02368384643F0B1
:104F480080432360FEF74EFC002860D14FF03709FC
:104F580009FB08F9DFF880B01BF8093013F0200FBF
:104F680055D13846FEF7F0FA804600284FD11BF895
:104F78000930012143F020030BF809300423009382
:104F88000333019333B20322029313200B460CF030
:104F9800F5FF50200DF0C8FB192041460122434679
:104FA800CDF80080FDF7ACFB31E000BF393D0020B3
:104FB800183B00202C1A0020611F0020901A0020A6
:104FC8002D3D0020713B0020783B00201F3C002035
:104FD8008C3B00202F3C0020AC3F0020372303FBF4
:104FE80008F3DFF8BC9119F8033013F0200F05D04F
:104FF800992001220B460091FDF782FB372303FB22
:1050080008F819F808306FF3451309F80830013724
:10501800082EFFB286D1A67806F00806F6B2002E52
:1050280040F03281584A06925FFA86F8B8F1000FCC
:105038000CBF4023702347F69B510993079149F60B
:105048009E69002447464FF4E07A0AFB06FA4E4A66
:105058002146524410465FFA84F8089220F05FFA1D
:1050680048B949480AF1700A5044214620F057FAD5
:10507800002800F0F680444B4FF4E07A0AFB063A29
:105088000AF1E00A5046214620F049FA002840F08B
:10509800E8805046214620F02CFADFF808A10FB925
:1050A800484600E007980CF0EBFE8AF800009AF8F2
:1050B8000000DFF8F0B0002800F0D3800138C0B25B
:1050C8008BF800000BF0B8FA002840F0CA809BF873
:1050D800000000F56A507C300CF0D2FE2B49C0B2BB
:1050E80008701FB92A4B19F803A003E0069A131990
:1050F80093F850A100EA0A0ABAF1000F00F0B18053
:105108000898214620F00BFADFF890B000B31E4B48
:105118004FF4E07000FB06302146703020F0FFF9B4
:10512800B0B91C49012F0B784AEA030A8BF800A092
:1051380054D13823B8FBF3F203FB12834FF43661E2
:105148004A43DBB2342101FB0323134AD3183FE05F
:105158000D4B4FF4E07000FB06302146703020F014
:10516800DEF938B10898214620F0D9F910B9094973
:105178000B7804E0074A13781AEA030F14D023EADD
:105188000A0A8BF800A029E0A8290020A21E002006
:10519800528FFF1F2C1A0020D0420020081E00202A
:1051A800AC3F0020221B00204AEA030A012F8BF89B
:1051B80000A013D13823B8FBF3F203FB12834FF49A
:1051C80036614A43DBB2342101FB0323A049CB18E3
:1051D80093F8302042F0200283F830209D489E4901
:1051E8009E4AFEF7E3FC9C4B1B781BB1FDF75EFF64
:1051F800002836D198489A4913F09AF868B10DF00A
:10520800A7F970BB964808F0B9FC50BB0123944835
:105218009449914A0093FEF79FFC00230093924A19
:105228000133019313788B4802938B498B4A8D4B3A
:1052380008F030FC012F14D13823B8FBF3F203FB3C
:1052480012884FF436635A435FFA88F8342303FB15
:1052580008237F49CB1893F8312042F0010283F8E4
:1052680031200134079A0999E3B205328B4209F1DA
:1052780001090792FFF4E7AE069A013602F5E072DB
:10528800022E06927FF4D0AE784E73786FF3C71370
:1052980073702B7803F08002D2B2002A00F00A81E2
:1052A80073490C78002C40F0058103F02403042B8B
:1052B8000BD1FEF7ABFBFF230093402021460122D0
:1052C8002346019402940CF059FE2B8800246FF3B6
:1052D800C7136FF3820364F3451364F3410364F364
:1052E8000003644A64F3492364F38A2314702B800F
:1052F800614B1A7842F0C0021A705A7864F3C302FC
:105308005A70FEF763FC5D4820F0AEF85C4820F068
:10531800ABF85C4820F0A8F85B4821464122FBF72F
:1053280039F829236343594A0134D15C082C01F028
:10533800DF016FF30411D154F3D1002322225A4321
:1053480053490133885C072B00F0DF006FF38610A8
:105358008854F3D14F4B1A786FF345121A7093F8AB
:1053680037206FF3451283F8372093F86E206FF3D8
:10537800451283F86E2093F8A5206FF3451283F841
:10538800A52093F8DC206FF3451283F8DC2093F80E
:1053980013216FF3451283F8132193F84A216FF311
:1053A800451283F84A2193F881216FF3451283F857
:1053B8008121394B1A7802F0DF026FF386121A70D6
:1053C80093F8222002F0DF026FF3861283F822207E
:1053D80093F8442002F0DF026FF3861283F844202A
:1053E80093F8662002F0DF026FF3861283F86620D6
:1053F8002A4B5A786FF345125A701A7802F0BF0296
:105408006FF345121A7093F825206FF3451283F84D
:10541800252093F8242002F0BF026FF3451283F889
:105428002420002311E04FF436615943342000FB57
:1054380002111B48013209188878382A6FF3820054
:105448008870F0D10133022B2CD00022EBE700BF8B
:10545800D0420020081E0020F11E0020E41E00207B
:10546800391A0020CD1D0020A21E0020821A00201B
:105478002C1300201F1C0020783F00209E1C0020B9
:10548800311A0020721A0020901A0020793D00205D
:10549800383C0020AC3F00208C3B0020183B00200B
:1054A800D8420020082273480021FAF773FF724B94
:1054B80000221A70714C2378002B4DD12978704A3C
:1054C80001F00201C9B201B36E49487863F3820062
:1054D80048706D481188477863F34D3163F3C3070B
:1054E80041F0800147701180CA2020F03DFEC6209F
:1054F80020F03AFE20F086FE644A13780BB90DF0CE
:105508009FF9FEF703F8FEF731FD614A2B88117801
:105518006FF341036FF300016FF3000311705D48EF
:10552800002140222B80FAF735FF5B481FF09CFFD3
:105538005A481FF099FF5A481FF096FF59481FF024
:1055480097FF08224B480021FAF724FF4A4A002314
:105558001370554A13706AE02F7807F00203DBB224
:1055680093B917F001070FD14B481FF07DFF23783F
:10557800F8B23B4113F0010F03D0FEF763F90CF0CA
:10558800DDFF0137082FF2D12B783D4F13F0010FC3
:1055980025D0FEF77FFC3B8843F002033B80FEF7F3
:1055A800F3F9354B93F80080B8F1000F14D1CA20F5
:1055B80020F0DAFDCD2020F0D7FD3B883B4868F38A
:1055C80000033B80324B1A7842F001021A701FF038
:1055D8004BFFFDF79BFF02E00120FEF737FB2B781E
:1055E80003F00202D2B212B32F4A12782AB113F092
:1055F800010F02D10220FEF729FBFEF789FE2C4994
:1056080026481FF04FFF254925481FF035FFFEF7B4
:10561800F7FA224927481FF02FFF274925481FF08E
:1056280036FFFEF787FA1F481C491FF046FF20493E
:1056380022481FF021FF15490B780BB9FEF708FA2D
:10564800737803F08003DBB2002B3FD1FEF7AAFC8E
:1056580030B143F6EC200CF013FC08B1062033E01F
:10566800FEF772FC08B105202EE00DF0D3F938B32F
:10567800032029E0621A00202A1A00202C1A002090
:105688003C1C0020933F0020783F00202C13002072
:10569800301A00205E1C002075320020161C0020E5
:1056A800721A0020561C0020A61C0020231B002074
:1056B800851A0020461C0020D21A00206A1A0020F1
:1056C80001F08AF810B10420FEF7C0FA6C4B1B7881
:1056D8001BB173786FF3C71373706A4A137813B1E9
:1056E800694B1B78CBB12B78684E03F04403402BF1
:1056F80013D10021BF3300933F200B4602220191B2
:1057080002910CF03BFC338843F6CE2043F00403AF
:1057180033800CF0B5FB5E4B18705A495D4E0B7820
:105728009BB1594B197881B92A78584B02F040023D
:10573800D2B252B11A8861F382021A80337823B93F
:1057480043F6CE200CF09CFB30702A78DFF83C81C1
:1057580002F00400C0B2504B00287FD002F02000B5
:10576800C0B24B4F90B11A78002042F0C0021A70B4
:10577800FDF7B0FD3B78002B76D1B8F8002063F335
:10578800820263F34512A8F800206DE0D20052B2FD
:1057980019789211D2B241F0C00112F0010F1970BC
:1057A80003D0C9B260F3C711197012F0020F03D009
:1057B8001A786FF386121A701B78374A03F0400381
:1057C800DBB273B9537843F008035370237843B1BD
:1057D8002B8843F400532B80304B5A7842F0040254
:1057E8005A700120FDF776FD43F6CD200CF048FBFA
:1057F800C0B20128307002D1264B02221A703C78C0
:10580800002C31D1FEF702F9FF230122009340203A
:1058180021462346019402940CF0B0FB2B8843F6F2
:10582800CD2043F020032B800CF02AFB184B1C4A98
:105838001870154B14701A780AB1013A1A70197851
:1058480091B9104A13787BB1FF23009341200222BB
:105858000B46019102910CF091FB05E01A7842F099
:10586800C0021A70FDF736FD0DF084F80D481FF0E0
:1058780029FE0D4BD0B91A7860F3820219E000BFF7
:10588800165D0020281C0020A71C00203C1C0020BE
:105898001F1C00208F1A0020783F0020933F002013
:1058A8002C130020DA1A0020301A00201A7842F04F
:1058B80004021A706A78654812F001011A780CBF60
:1058C80061F3410242F002021A7061491FF0F5FDCE
:1058D80060495E481FF0DBFD5C485F491FF0D7FD5B
:1058E8003378012B40F0AF802B8800246FF34923D5
:1058F8006FF38A232B80594B21461C70412258484C
:10590800FAF748FD57481FF0AFFDFEF75FF9514819
:105918001FF0AAFD50481FF0A7FD29236343524AF0
:105928000134D15C082C01F0DF016FF30411D1546C
:10593800F3D1002322225A434C490133885C072BB8
:1059480000F0DF006FF386108854F3D1484B1A78C3
:105958006FF345121A7093F837206FF3451283F8E6
:10596800372093F86E206FF3451283F86E2093F872
:10597800A5206FF3451283F8A52093F8DC206FF378
:10598800451283F8DC2093F813216FF3451283F84E
:10599800132193F84A216FF3451283F84A2193F8AB
:1059A80081216FF3451283F88121324B1A7802F076
:1059B800DF026FF386121A7093F8222002F0DF02DA
:1059C8006FF3861283F8222093F8442002F0DF0256
:1059D8006FF3861283F8442093F8662002F0DF0202
:1059E8006FF3861283F86620234B5A786FF34512BB
:1059F8005A701A7802F0BF026FF345121A7093F8C2
:105A080025206FF3451283F8252093F8242002F00F
:105A1800BF026FF3451283F82420002311E04FF4EE
:105A280036615943342000FB021114480132091829
:105A38008878382A6FF382008870F0D10133022BFE
:105A480001D00022EBE70BB0BDE8F08FFA3600205A
:105A5800461C0020311A00209E1C00208F1A0020AE
:105A6800901A0020721A0020793D0020383C00204E
:105A7800AC3F00208C3B0020183B0020D84200207F
:105A88002DE9FF4104460D460CF09EFFA04B1A1964
:105A980092F880709F4A98461278AA2A0AD1A7F1EC
:105AA8004F03DAB20B2A00F2AD819B4A5BB29A40EF
:105AB80040F1A881994B0C2202FB04335A7A08332F
:105AC800AA42C0F09F81FF2A00F09C81FF229A70B1
:105AD800934808EBD403214693F888511FF01FFD23
:105AE8000646002840F08E8104F007031D41502F20
:105AF80005F0010500F0268114D8462F00F0F28049
:105B080009D8412F00F09E80452F00F01B812D2FD2
:105B180040F0768134E0482F00F0C5804F2F40F0E8
:105B28006F810EE0542F67D006D8522F00F08A807C
:105B3800532F40F065811CE0A7F15903012B00F2B7
:105B48005F81784821461FF0EAFC0646002840F0AD
:105B580059815A2F01D1744802E0592F04D1734852
:105B680021461FF0C6FC54E121466F481FF0C1FCD6
:105B7800F5E76F4821461FF0D2FC002800F042816B
:105B88006C4821461FF0CBFC8046002840F03A8143
:105B9800214668481FF0ADFC674821461FF0B4FC59
:105BA8000227012655B1A419142041463A46434616
:105BB8000097019602940CF0E1F92AE129463A4649
:105BC800334604F101080A2000970196CDF80880B1
:105BD8000CF0D4F92046FCF7CBFA414602462B4696
:105BE80013200095FCF78CFD384629462A46334693
:105BF8000095FCF785FD0CE14E4821461FF08FFC0F
:105C08000746002840F00581012602223146334626
:105C1800A5193E200092019602950CF0AFF9204696
:105C2800FCF7A6FA294602463B4614200097FCF7E3
:105C380067FD21463F481FF05CFC21463E481FF0A7
:105C480063FCE6E03A4821461FF069FC0646002856
:105C580000F0DF80374821461FF061FC064628B96E
:105C68002046FDF771FC002840F0D380002D40F05D
:105C78008E802046FEF742F9002840F0C580204675
:105C8800FEF736FB2D4BDB7803F02003DBB20BB9B4
:105C98002B4B1855412F00F08880522F40F0B080D0
:105CA8002046012183E0234821461FF038FC28B90B
:105CB8002046FDF749FC002840F0A480002D66D15D
:105CC8002046FEF71BF9002840F09E801B4BDB782E
:105CD80003F02003DBB2002B67D1194B032283F8B2
:105CE800402062E0134821461FF019FC064628B9F7
:105CF8002046FDF729FC002840F08B802046FEF75F
:105D0800FDF800287ED1002D41D1204603214EE028
:105D1800302D00201E1C002000003080042F0020A1
:105D2800851A0020882A0020A8290020182A002087
:105D3800161C0020461C00204E1C0020083B00209A
:105D4800901A0020354821461FF0E9FB0646002836
:105D58005FD02046FDF7D0FD20B1214630481FF026
:105D6800C8FB4FE0502F28D12E4B1B782BBB204669
:105D7800FDF7AEFD08BB2C4821461FF0D0FB0646B8
:105D880020B92046FDF7E0FB002842D115B1204696
:105D980002210CE02046FEF7ABFA244BDB7803F037
:105DA8002003DBB20BB9224B185520460021FEF721
:105DB800A7F9061E18BF01262BE02046FDF788FD2F
:105DC8000546F8B91B4821461FF0A9FB0646D8B975
:105DD8002046FDF7B9FB0746D8B9164821461FF0FB
:105DE80088FB154A135D8BB910494E7806F02006DA
:105DF800F6B26EB908EB040393F80031135508E0C6
:105E0800012606E0002604E02E4602E03E4600E0B9
:105E18001E46304604B0BDE8F08100BF161C0020C5
:105E2800231B0020A61C0020461C0020083B002045
:105E3800901A0020721A00205E1C0020032210B560
:105E480005490648FAF77CFD054806490222BDE8DF
:105E58001040FAF775BD00BF032700200402002098
:105E6800090200200127002070B5834B1B7813F02E
:105E7800010F0AD00CF074FB38B100207F4902F002
:105E88008DFE7F4B7F48197847E07F4D2B78002B9C
:105E980048D00CF06BFB002844D07C4B1B7863B9CE
:105EA8007B4B5B7813F0010F07D00CF051FB20B946
:105EB800FEF778F808B10320BEE0764C207870B180
:105EC8000020754902F06AFE21780122734802F029
:105ED8008BFE00201021621C07F0C4FA02E0704912
:105EE80002F05CFE6F4C684807F0E2FA2378002B5A
:105EF80000F018810CF034FB002800F013816A4987
:105F08006A481022FAF71CFD68485B21FAF7C0FAC4
:105F1800002800F00781217801308322BDE8704015
:105F280002F062BE624C237803F00503012B5DD1B9
:105F38000020604902F032FE202110225E48FAF764
:105F480029FA601D5D490322FAF7A4FC40BBE01C56
:105F58005B490222FAF79EFC30B95A48FAF76AFC04
:105F68005849024654480BE0E01C57490222FAF708
:105F780091FC40B95548FAF75DFC544902464E4831
:105F8800FAF7DEFC0EE0E01C51490222FAF782FC27
:105F980030B95048FAF74EFC4E4902464648EFE7FA
:105FA800FFF74CFF6278303AD3B2092B00F2BA807F
:105FB8003F4B9B78303BDBB2092B00F2B3800A21C0
:105FC80001FB0231C9B2002900F0AC80374BFF2237
:105FD8000C291A7740F2A68010295A7740F2A2803D
:105FE80013299A7740F29E80DA7770BD3A4C23786D
:105FF80003F00203DBB213B1002038498EE0234ED0
:106008003378EBB9224B5B7813F0010F18D00CF002
:106018009FFAA8B932481FF055FA60B12268314B8F
:1060280002EA03033BB919F0CBFA20B9E37803F08D
:106038004003DBB223B10020BDE8704009F0D0BDB9
:10604800337863B90CF084FA48B1274B1B7803F016
:106058000603042B03D02B780BB90120ECE7FDF7DE
:1060680073FF10B10020214958E0214B1D78002D05
:1060780042D0204952E000BF3C1C0020F53F0308F5
:106088002A1A0020000200202C1A0020A01E00203E
:10609800611F0020EA1D00200815030805020020E2
:1060A800C6140308A61C0020E7140308F401002006
:1060B800FE2600200F1A03080402002030A303085C
:1060C80034A30308721A030837A30308511A0308F4
:1060D8003AA30308301A0308083B0020662903087E
:1060E800DA1A00203000000F301A00209827030821
:1060F80031130020291503080B4802F0FEFC0A485A
:1061080002F0F2FC094802F0EFFC1DF07DFEE37896
:1061180003F02003DBB22BB105492846BDE87040E7
:1061280002F03CBD70BD00BFF41E0020141E00200C
:1061380021140308054B1B78D8019B015BB2DB11C6
:1061480040B243EAE070C0B2704700BF3C1C002078
:1061580070B50E4686B041000122054601F5E97189
:1061680005A80BF09EFE0021012E8DF815104FF0AA
:10617800FF0205F1010305D1009201910293092064
:10618800FB3A04E00092019102931E2004220B4680
:106198000BF0F4FE05A83D49FAF700FA50B105A83E
:1061A8003B49FAF7FBF928B105A83A49FAF7F6F995
:1061B800002867D105A83749FAF7F0F9364B0446A5
:1061C800F8B95A78214642F010025A70FF23022289
:1061D80000930190FE3B02903D200BF0CFFE4D2036
:1061E8000CF0A2FA691C0122234612200094FCF745
:1061F80087FA12202146224601230094FCF780FAF0
:1062080003E05A786FF304125A700024E0B2552163
:1062180016F052FA38B12846214616F0EEFB10B1B6
:10622800204616F0D9FB0134112CEFD13EBB1B4898
:106238001B491C4AFDF7BAFC19481B4912F078F8AB
:1062480068B10CF085F950B9174807F097FC30B9D8
:10625800012315481549124A0093FDF77DFC144B9C
:106268000F491D700023009305330193114B0D4A0C
:106278001B780A4802930D4B07F00CFC02E00E4B0A
:1062880000221A7005A806B070BD00BFC1A303089C
:106298003DA30308CDA50308783F0020081E002071
:1062A800F11E0020E41E0020391A0020CD1D002018
:1062B800973F0020A21E0020611A002007B5410068
:1062C800012201A801F5E9710BF0EBFD002301A8FB
:1062D80004498DF80530FAF761F9D0F1010038BFAB
:1062E80000200EBDC1A3030807B54100012201A883
:1062F80001F5E9710BF0D5FD002301A804498DF8DB
:106308000530FAF74BF9D0F1010038BF00200EBD77
:106318008AA5030870B5154B04461B1893F88050DE
:10632800B1B1134821461FF0FAF888B9114821463F
:106338001FF0DFF8A5F15903DBB2012B0CD94F2D63
:106348000AD0542D08D021460B481FF0D2F807E098
:10635800084821461FF0D8F8074821461FF0D4F80E
:1063680004480649BDE870401FF086B8302D00206B
:10637800851A0020DA1A00207A1A0020561C0020FC
:10638800024B1878C0F38000704700BF301A002015
:10639800024B1A8860F308221A8070473C1C0020C0
:1063A800034B5878C00140B2C011C0B2704700BF5B
:1063B8003C1C0020014B1878704700BF2C1A0020A5
:1063C80030B5457800230021C218917055FA03F1C1
:1063D80011F0010F08D0064959188C7C017804EA9D
:1063E8000101A14208BF91700133042BEBD130BDEC
:1063F800EA1D002046F6295104220BF052BD000088
:1064080070B5104C0546112220460021F9F7C2FF4D
:10641800002004F8010C2A78103414F8011FC3B2C4
:1064280091420BD152B10849013301F8013B1122C5
:1064380046F67973BDE8704002F0FCBA01300428D2
:10644800EBD170BDEB1D0020EA1D00201FB520B167
:10645800134B1A8842F480521A80124B00245A783F
:10646800214642F010025A70FF23022200933D2079
:10647800FE3B019402940BF081FD4D200CF054F981
:1064880040210122234612200094FCF739F91220FA
:106498002146224601230094FCF732F91FBD00BFB4
:1064A8003C1C0020783F00202DE9F3412D4C0722A9
:1064B800E37849F6346702FB0030C0B200F51E40AD
:1064C80055300BF0DDFC257964795FFA80F80026F9
:1064D80048FA06F313F0010F3AD03946042201A80E
:1064E8000BF0DFFC9DF804009DF805309DF80610C0
:1064F8009DF8072000282BD0002929D0002B27D071
:10650800002A25D0934204D19C4221D185421FD331
:106518000FE09A4210D99C421AD3944218D89C4250
:1065280001D994421AD39C4201D1854216D2944291
:106538000ED18D420CD811E09C4201D185420DD27A
:10654800944201D18D4209D99C4207D8944205D37F
:1065580001360437082EBBD1002000E00120BDE839
:10656800FC8100BF845A002010B5044649F68D60AE
:1065780000EBD4000BF084FC04F00704C0B2204107
:1065880000F0010010BD70B5C30849F68D655D19AE
:10659800044628460E460BF073FC04F00704C0B20C
:1065A800012126B9A14040EA0101C9B202E0A14097
:1065B80020EA01012846BDE870400BF057BC0000F6
:1065C800F0B57D4B95B0DD78082200EBC505EDB23E
:1065D800E90001F50A4104A8BC310BF062FC774BD5
:1065E800774E1A78002304A9C95C312905D13039BE
:1065F800994041EA0202D2B205E0302903D12F398D
:10660800994022EA01020133082BECD132706C4820
:106618006C496D4AFDF7CAFA6A4B1B7813B96A4B85
:106628001B78F3B16748694911F082FE68B10BF035
:106638008FFF50B9654807F0A1FA30B901236348C4
:106648006349604A0093FDF787FA002300930233F9
:106658000193FD3302935A485A495B4A5C4B07F051
:1066680019FA05EB0511002401F50C41347004A852
:106678007C3111220BF015FC2646E0B2542116F0AD
:106688001BF8002838D004AB1B5D312B03D1204602
:1066980016F0A8F838B104AB1B5D302B2CD120467E
:1066A80016F0A0F840B34EB9FF23009334203146CA
:1066B80004223346019602960BF060FC04AE305D6E
:1066C8002146303816F09CF8335D0126312B4FF007
:1066D800030306D10093A3191BB201960293352038
:1066E80005E00093631C1BB201960293362000213B
:1066F80004220B460BF042FC0134112CBDD1A90138
:1067080001F5104104A8343140220BF0CAFB113CBA
:1067180004AD274615F8013BE6B20134302B03D10E
:106728003046FFF721FF38B115F8013C312B2CD149
:106738003046FFF719FF40B34FB9FF2300933420C9
:10674800394604223B46019702970BF017FC15F8CF
:10675800011C30463039C9B2FFF715FF15F8013C66
:106768000021302B4FF0FF0305D1009323B2019194
:106778000293372004E0009323B20191029338205A
:1067880004220B460BF0FAFB0127402CC2D1114D15
:106798006B7803F00403DBB263B1403C2046FFF79B
:1067A800E3FE38B90134E4B2402CF7D16B7860F3DA
:1067B80082036B7015B0F0BD845A00202C1A00209B
:1067C800081E0020F11E0020E41E0020391A0020B7
:1067D800CD1D0020783F0020014B1878704700BF7E
:1067E800311300202DE9F04F4E4B00221A704E4A0B
:1067F80085B01678002E40F091804C4B4FF4B46869
:10680800DA78997808FB02F24FF03C0808FB012877
:106818005A78474F90441FFA88F8BA466CE03AF81D
:1068280015303C24DAB2544304EB13244C44A4B28C
:10683800042CEEB207D842F25A73984503D904F5EE
:106848001C546034A4B2444511D949F654600BF085
:1068580017FBC8EB0403834209DC364B1A787B1913
:1068680093F87030934302D02E4901230B702F4ABE
:10687800D378B34232D142F26073B4FBF3F203FB34
:1068880012439BB2434523D12B4B9B7813F0090F3E
:1068980044D12A4B5B7803F08003DBB2002B3DD157
:1068A800274B5B7803F00203DBB2002B36D1254B74
:1068B8001A781BEA020F11D10199009841EA0202E5
:1068C8001A70FFF7F1FD48B90098FFF779FE05E067
:1068D8001C4B02991A7801EA02021A70013509F56F
:1068E800B469072D1FFA89F999D1039E0737013634
:1068F800082E0AF10E0A11D04FF0010B0BFA06FB15
:106908005FFA8BF301936FEA0B03F2B2DBB24FF03D
:106918000009009202934D46039680E705B0BDE852
:10692800F08F00BF31130020AD1C0020845A0020D6
:10693800AE1C00202C1A0020083B0020873F0020B6
:10694800F2340020AC1C002073B50C4601EBC001EA
:10695800C9B2C90001F50A41054608226846BC319A
:106968000BF09FFA104B002003EBC402121B5219C4
:1069780082F870001DF80020312A0AD101218140D7
:1069880003EBC402121B521992F87060314382F86B
:10699800701001300828EDD16946312230231EF0ED
:1069A800C6FDC0B27CBD00BFAE1C002000B501EB27
:1069B800C001C9B2890191B001F5104134314022BA
:1069C80068460BF06EFA40206946312230231EF0EB
:1069D800AEFDC0B211B000BD7FB501EBC001C9B2B8
:1069E80001EB011101F50C417C31112201A80BF0DA
:1069F80058FA112001A9312230231EF098FDC0B2A7
:106A080007B000BD2DE9F843002634462BE02146A7
:106A18002846FFF799FF214681462846FFF7C6FF1B
:106A2800214640EA09092846FFF7D6FF5FFA89F9A7
:106A380049EA000010F0FF0F05D04046394602220F
:106A48000BF02FFA03E04FF0FF33A8F800300135C0
:106A5800EDB20237072D08F10208D8D10134E4B2AB
:106A68000E3E082C07D0054BC6F50A47C6EB0308AF
:106A78004C370025CBE7BDE8F88300BFAE1C0020EB
:106A880010B523F073FA4FF4803023F08FFA23F017
:106A9800A7FB0128044628D1102023F089F90220F9
:106AA80023F07AF9002023F0C1FA002023F0D2FA6B
:106AB8004FF4806023F0C4FA4FF4404023F0D4FA36
:106AC8004FF480304FF4E01123F08CFA204623F085
:106AD80095FA392023F070FB0028FAD0022023F021
:106AE80093FA23F09BFA0828FBD17C20012123F09C
:106AF8002DFB46F60120012123F028FB0C4801213B
:106B080023F030FB0B48012123F02CFB042001214A
:106B180023F028FB7E2023F04FFB38B123F076FBCF
:106B2800054B04211A7861F344021A7010BD00BFA6
:106B38000340060020080818F95C002010B50C4630
:106B4800014620B110220C48F9F7FAFE04E00A4881
:106B580020211022F9F71EFC34B1084821461022E2
:106B6800BDE81040F9F7ECBE044820211022BDE82A
:106B78001040F9F70FBC00BFF40100200402002008
:106B880010B5FF2B1446029A03D0421802F8013CB4
:106B980008E06FF07F439A4204D013144370131235
:106BA8008370C2701CF042F802E07F2023F04AFE96
:106BB8001CF028F80028F8D1ACB10B4890F8201048
:106BC800163001F00F011CF031F802E07F2023F0AD
:106BD80039FE1CF017F80028F8D1044B93F86930F7
:106BE80013F0010FE9D110BD580C0020145C0020EF
:106BF80010B50A4B002203EBC003013B10460849BD
:106C080051184C7813F8011F8C4205D10130C0B2DD
:106C18000C320828F3D1F73010BD00BF16A90208BE
:106C2800042F002070B50D4C05460E464FF4007237
:106C380000212046F9F7AEFB2A46314604F50070DC
:106C4800F9F700FB642024F8035C1DF0AFFB002378
:106C5800A4F82D33024B64221A6070BD7D5D0020BC
:106C68000827002010B5054C002120464FF400727B
:106C7800F9F790FB0023A4F82D3310BD7D5D0020AB
:106C8800164B2DE9F0415D8A07462846FAF748FF7A
:106C98001349FBF751F8134B134E1860D723B5FB74
:106CA800F3F5EDB2822229460446F01901F09CFF63
:106CB8002846FAF739FF01462046FAF77FFE0B49C6
:106CC800FAF786FFFBF74AF90337BE19C1B28122EA
:106CD8003046BDE8F04101F087BF00BF40320020D8
:106CE80000005743581D0020F401002000002041F7
:106CF80070B54B4D2868FAF71FFB45A3D3E900236D
:106D0800FAF7BAF9FAF706FEFAF716FB42A3D3E93F
:106D18000023FAF765FB3EA3D3E90023FAF78AFCC0
:106D2800FAF7F8FDFAF708FBFAF712F9FAF7F2FDA5
:106D38003C4906462860FBF7F3F820B13046FBF7DC
:106D48000DF9C4B25EE030463649FBF7FDF850B1A4
:106D580030463549FBF7E4F828B13046FBF7FEF832
:106D6800C0B2441C4EE030462F49FBF7EDF850B155
:106D780030462E49FBF7D4F828B13046FBF7EEF839
:106D8800C0B2841C3EE030462849FBF7DDF850B11C
:106D980030462749FBF7C4F828B13046FBF7DEF840
:106DA800C0B2C41C2EE030462149FBF7CDF850B1E3
:106DB80030462049FBF7B4F828B13046FBF7CEF847
:106DC800C0B2041D1EE030461A49FBF7BDF850B1A9
:106DD80030461949FBF7A4F828B13046FBF7BEF84E
:106DE800C0B2441D0EE030461349FBF7ADF848B178
:106DF80030461249FBF794F820B13046FBF7AEF85D
:106E0800C0B2841D0A202146BDE870400BF02EB8A0
:106E1800736891ED7CFF7F400000000080842E4164
:106E28005C1D0020000010410000F04100004842B5
:106E380000008E420000B8420000E0420000F2422A
:106E48002DE9F04FA1B01BF087FE09201DF04AFC88
:106E58001DF030FA4FF461401DF080FC09201DF050
:106E6800FDFC0022A3484FF4804123F006F8A24815
:106E7800002123F0CFFBA14904224B78DFF8A0E2E0
:106E88006FF300034B709E4B9E4C1A705A715A70E8
:106E98009A70DA701A719A71DA719B4B033A1A7008
:106EA8009A4B00201F328EF8000020705A7105900E
:106EB8000546069006467F2023F0C4FC23780E2B57
:106EC80001F2B681DFE813F00F004F009500E000F3
:106ED8007902DE0330048504EA06DC07EF07580868
:106EE800B108D00882098A4E8A48317801F00F012A
:106EF800013149014118FFF721FE337813F00F03E0
:106F080008D1854A92F80123012A41F09181834AE8
:106F1800138024E0012B03D17F4B93F819330BE046
:106F2800022B04D17C4B93F80D33032B05E0032B84
:106F380006D1794B93F80D33012B41F079810EE09E
:106F4800774901220A7077484FF4007122F095FFC3
:106F5800754BC8221A6033786FF30303BFE33378A5
:106F68005A1C01F05FB8704B1A6822B96D484FF48B
:106F7800007122F082FFDFF898816C4898F80010C1
:106F880001F00F01013149014118FFF7D7FD36B172
:106F980098F800305A1C62F3030388F800305F4BFE
:106FA80000221A8098F8001001F00F02022A03D17B
:106FB8001A7842F010020AE0042A03D11A7842F043
:106FC800040204E0052A05D11A7842F040021A703A
:106FD80001F02EB9062A04D14D4B6FF30301197045
:106FE8007EE301F00F01012212FA01F1198001F08C
:106FF8001FB9474E4E48317801F00F010131490160
:107008004118FFF79BFD96F8008008F00F08B8F1CB
:10701800070F27DC18F0010F464B02D000205880DC
:1070280002E04FF0FF3159804FEA6809062209F162
:10703800010902FB09394FF0FF32A9F80220404646
:10704800FFF7D6FDFF2806D03B4B03EB4000582343
:10705800437401F0EDB80023A9F8023008F10108E3
:1070680001F08AB8002110221BA8F9F793F917A894
:1070780000211022F9F78EF9237801332370337831
:107088006FF3030301F07BB8DFF884A09AF800805F
:1070980018F00F0840F03F81284E337803F0400382
:1070A800DBB2F3B926486FF07F43817A012200935F
:1070B80001F00F01FF23FFF763FD224B93F86920CE
:1070C80012F0400F08D093F86C3013F0040F03D07F
:1070D800337843F0400333707378142262F3C703A4
:1070E8007370737813F0F80F30D0174800F120014F
:1070F800A7E300BF00180140002C014062320020C5
:10710800302D0020621D00202F130020793D002023
:10711800611D002056A90208042F0020783F002096
:1071280038270020000C014008270020F6A9020893
:10713800D6AA0208FE3E0020F4010020F33A0020FF
:10714800580C0020145C0020F6AB0208BC4B1B78DE
:1071580003F04003DBB2002B00F0D980DFF8048392
:10716800DFF8049398F8003013F00C0B30D1B54ECB
:107178006FF07F4396F82B1006F12100009301F081
:107188000F0101220523FFF7FBFC96F84C104FF482
:10719800860A06F1420001F00F010122FF23CDF813
:1071A80000A0FFF7EDFC96F84110FF2306F1370029
:1071B80001F00F015A46CDF800A0FFF7E1FC0423C7
:1071C80089F8003098F8003043F0080301F02EB831
:1071D80003F00803DBB2002B39D099F800A0BAF10C
:1071E800000F03D0984800F1400138E0954E6FF049
:1071F8007F4B717D06F10B0001F00F010122FF2387
:10720800CDF800B0FFF7BCFC96F82B1006F1210072
:1072180001F00F0101220723CDF800B0FFF7B0FC01
:1072280096F836104FF48603009306F12C00FF23DE
:1072380001F00F015246FFF7A3FC98F800306AF3FB
:10724800C303DBB243F0040388F800305AE099F82E
:1072580000C0BCF1000F08D07B4800F16001FFF7C7
:107268006DFC99F80020303208E2764E6FF07F40CE
:10727800717DFF23009001F00F0106F10B00012240
:10728800CDF80CC0FFF77CFC9AF80030DFF8C4B1E9
:1072980003F0100A5FFA8AFADDF80CC0BAF1000FA1
:1072A8000CD098F800206CF3820288F800205A1C51
:1072B80062F303038BF8003000F0BABF96F82B1086
:1072C8006FF07F42009206F1210001F00F010122C8
:1072D8000C23FFF755FC96F836104FF486030093FD
:1072E8005246FF2306F12C0001F00F01FFF748FC7E
:1072F8009BF8003083F01002C2F3001262F304130B
:107308008BF80030042389F8003000F091BF4E4814
:1073180000F1800195E2B8F1010F3CD14A4800F133
:10732800A001FFF70BFC002E00F082879AF80030CE
:10733800444E5A1C62F303038AF8003096F82B1067
:107348006FF07F4906F1210042460F2301F00F013B
:10735800CDF80090FFF714FC96F82B1006F12100E9
:1073680042460E2301F00F01CDF80090FFF708FC0C
:1073780096F82B1006F12100424601F00F010F2369
:10738800CDF80090FFF7FCFB30488021424622F000
:1073980074FD00F04DBF2C4800F1C001FFF7CEFB93
:1073A800002E00F045872A4B96221A609AF8003082
:1073B8006FF303038AF8003092E1264E317811F01A
:1073C8000F0A16D1244800F12001FFF7B7FB204B24
:1073D8001B68002B40F02C871BA8F9F72BFA4022DA
:1073E800134601461BA801F023FA3378012200F066
:1073F80019BEBAF1010F39D112486FF07F4390F8E6
:10740800201000220093163001F00F01FF23FFF730
:10741800B7FB01F077FA002800F00A8733780222D8
:1074280062F3030333700D4B1A7842F080021A702E
:107438000B4B5A7842F002025A7000F0F9BE00BFB6
:10744800F33A0020580C0020F6AB02080010014067
:1074580008270020611D0020D6AC0208F83A002059
:10746800F2410020986300201F65002001F00F0101
:1074780001F10E0303F00F03012B44D89B48490187
:107488004118FFF75BFB9A486FF07F4390F8201094
:1074980000221630009301F00F01FF23FFF770FB65
:1074A8001CF050FD337803F00F03022B13D118F0B2
:1074B80053F8002800F0BC868E4B1A7842F0400240
:1074C8006FF304121A705A786FF345125A703378B2
:1074D800032200F0A7BD18F029F878B118F0C8F811
:1074E80017F080FF844B00201A7858816FF3C71279
:1074F8001A703378042262F3030333707F4B1A78CF
:107508006FF3000263E5BAF1040F4DD1DFF8DC91A7
:107518004901DFF8108249444846FFF70FFB98F805
:107528000010774B01F00402D2B27AB941F004019D
:107538006F4883F800A088F8001090F836104FF4D0
:10754800860300932C3001F00F01EEE293F800A0BF
:10755800BAF1000F40F06C8665486FF07F45417DB9
:1075680001220B3001F00F01FF230095FFF708FB04
:1075780064480122817AFF2301F00F010095FFF78B
:10758800FFFA98F8003005226AF3820388F8003081
:107598003378484662F30303337009F1A001FFF71B
:1075A800CDFA554600F044BEDFF84481FF2398F831
:1075B800201000226FF07F4908F1160001F00F013A
:1075C800CDF80090FFF7DCFA2BB2072B18D13378EF
:1075D80008F121006FF3030333702378012201338C
:1075E800237098F82B100E2301F00F01CDF80090AE
:1075F800FFF7C6FA44488021002222F03EFC00250D
:10760800424E96F86B3013F0040F00F0118698F88C
:1076180057106FF07F43002200933D48FF2301F08D
:107628000F01FFF7ADFA96F86B303A4A03F00F03F3
:10763800012B137003D1002D08BF01250CE0022B8C
:1076480004D12BB2012B08BF032505E0032B03D17E
:107658002BB2032B08BF0725ABB213F0010F02D0E2
:107668002D4A3121517713F0020F02D02A4A3221D4
:10767800917713F0040F00F0DB853322264BDA777D
:1076880000F0D6BD1948254E00F1C001FFF756FAA3
:1076980096F80090DFF85C8019F00F090CD117F00C
:1076A800BBFD98F8003069F3000388F800303378A0
:1076B8005A1C62F30303337017F040FE98F8003049
:1076C80013F0010F00F0B48500221548802122F044
:1076D800D4FB0A4B00225A70337862F303033370E9
:1076E80023780133237000F0A3BD00BFD6AC020895
:1076F800580C0020F2410020F83A00206A4100208E
:107708001F6500200100002000100140145C0020CB
:10771800A50C0020F23A0020F4010020611D002091
:1077280000180140986300208648874E00F1E00168
:10773800FFF704FA17A8F9F77DF817A90246834856
:10774800F9F7FEF800218248B18090F8C5106FF073
:107758007F4300220093BB30FF2301F00F01FFF7A6
:107768000FFA7C4A92F86B1092F86C30327843EA40
:10777800012312F0010FB38010D0A3F1EB0292B2F3
:107788000A2A04D9A3F5E6739BB2282B02D8F388FA
:107798000133F38033786FF3000333707378002B71
:1077A80040F04685684AD2887AB16B4A1FA811789A
:1077B80063F30301117022788DF87F300132227053
:1077C80028228DF87C2022F077FB0022F28000F03E
:1077D8002FBD624EDFF8ACA1337803F004085FFADE
:1077E80088F8B8F1000F15D111A841461522F8F70D
:1077F800D1FD5B4BCAF800801B684546CDF8473081
:107808003368474643F004033360564BA3F8368386
:1078180000F00EBD03F08003DBB2002B67D1DAF86D
:107828000010002940F004854F48FFF787F94F48BA
:107838004FF4805122F017FB012806D04A4800F186
:10784800A001FFF77BF900F0F3BC4649B1F83623F5
:10785800002A43D009314648013AF9F771F8444BF8
:1078680003F1100113F8012B0D2A01D00A2A02D1C5
:10787800202203F8012C8B42F4D13E4B4FF03C08F8
:1078880008FB073808F11E084046F8F7D3FF4146C1
:1078980002463948F8F7FEFFD8B9022F03D13368FA
:1078A80043F0100304E0032F03D1336843F040038F
:1078B8003360327853005BB203EAC263DB17326885
:1078C800DBB263F3C71232601BB1FFF7CBF900F0EC
:1078D800AFBC0137FFB2042F08BF0227254B3C2657
:1078E80006FB07363046F8F7A5FF314626E0DAF8FA
:1078F8000080B8F1000F40F09B84737803F02002F9
:10790800D2B2002A40D11D4B11A81A889B781C4975
:107918008DF84630ADF84420F8F796FD114B5B7AA8
:10792800302B07D1FFF79EF9336843F400533360D7
:1079380000F07EBC11A8F8F77DFF11A9FFF772F9D6
:1079480000F076BCD6AC02086A410020080200208C
:10795800580C0020145C0020611D00200C2700201A
:107968003FA30308745D0020D6AD0208000801405B
:10797800040200200C0000207D5D002044A30308C1
:1079880048A303080827002003F04003DBB2002BBC
:1079980040F08980B14800F16001FFF7CFF8B048A6
:1079A800F8F748FF8046AE49AE484246F8F772FFFE
:1079B800002873D1AC4B43445B7A302B6ED1FFF770
:1079C80051F93368DFF8D09243F48043336099F873
:1079D8002B106FF07F43009309F12100082301F079
:1079E8000F010122FFF7CCF86423CAF800307F208A
:1079F80022F028FFDAF80030002BF8D1984699F8E1
:107A08008E10D633994E89F886304B3B6FF07F4AFB
:107A180089F88730964801F00F0142467433CDF853
:107A280000A0FFF7ADF896F8B91106F5D670033047
:107A380001F00F014246FF23CDF800A0FFF7A0F8A0
:107A480096F8C41106F5DD7001F00F014246FF23D8
:107A5800CDF800A0FFF794F896F8CF1106F5E2707C
:107A6800013001F00F014246FF23CDF800A0FFF7D7
:107A780087F896F8DA1106F5E87001F00F0142462A
:107A8800FF23CDF800A0FFF77BF899F89910794803
:107A9800CDF800A001F00F01424646E07648F8F71D
:107AA800C9FE75494AE796F802B0DFF8EC910BF089
:107AB800020B5FFA8BFBBBF1000F3AD199F820104B
:107AC800FF236FF07F4809F1160001F00F015A46B5
:107AD800CDF80080FFF754F8684B93F86B3003F04B
:107AE8000803DBB2002B00F0A38399F82B100122C6
:107AF80009F1210001F00F010323CDF80080FFF701
:107B08003FF83368554843F4003300F1800133608F
:107B1800FFF714F855485A4690F8E51100F5EC704F
:107B2800CDF80080033001F00F01FF23FFF728F89C
:107B38007EE3CAF8008099F820106FF07F43009325
:107B48004246FF2309F1160001F00F01FFF718F86C
:107B58002AB241F211139A421DD1434B5B7A302B62
:107B680013D1FFF77FF83368454668F3514368F34C
:107B78008E3368F34D333360414B1A7868F3030250
:107B88001A7023780133237052E33E48F8F752FE07
:107B98003C49FFF747F8394E96F86B3013F0040F5D
:107BA80000F0468325B9384820211022F8F7F2FB67
:107BB8007F2022F047FE99F857106FF07F4300228C
:107BC80000933248FF2301F00F01FEF7D9FF96F822
:107BD8006B202F4B02F00F020D2A1A7005D125B920
:107BE8002C4A412191754FF480551A78062A08D1FC
:107BF8002AB2B2F5805F04D1264A3621D1754FF4F6
:107C080088551A78082A08D12AB2B2F5885F04D1B3
:107C1800204A3821117641F210151B780B2B09D117
:107C28002AB241F210139A4204D11A4B2A225A76E8
:107C380041F211150D486FF07F4390F8F0110022C2
:107C4800009300F5F370FF2301F00F01FEF798FF92
:107C580096F86B3013F0010FAAD0E9E2D6AD02080E
:107C68001A0100207D5D0020745D002001000020C5
:107C7800DC0C0020E70C0020FC000020145C002035
:107C8800611D00203801002004020020A50C0020FE
:107C9800F23A0020F4010020580C0020A34B1A7877
:107CA80042B300221A700F20FAF7CEF906460A20CE
:107CB800FAF7CAF99E4B9F4958824A7812F0010F89
:107CC80018D06436301A58839B4B1A78642A01D12D
:107CD8009B321A701B78984EFF2B0BD00A21B3FBEE
:107CE800F1F1964B19311980954822F093FC3378BD
:107CF80001333370DFF8648298F8003013F00F0610
:107D080012D18E4B19228B481A804378192143F0DF
:107D1800010343708A4822F07DFC8A4800F1200163
:107D2800FEF70CFF04967CE2012E68D1804B5A8B3B
:107D3800A2F1690189B2112908D8049911F0010F3B
:107D480004D141F00101C9B204910592049A12F0DC
:107D5800020F0DD15B8A7C4A1380A3F5C263023BF4
:107D68009BB2D72B04D8049840F00203DBB20493EB
:107D78001B20FEF785FF0599744B0AB2632A05DDBF
:107D8800642192FBF1F230321A7401E0092A0CDD09
:107D9800059A11B2642291FBF2F002FB10120A203C
:107DA80012B292FBF0F230325A74059802B2642093
:107DB80092FBF0F100FB11210A2209B291FBF2F0CB
:107DC80002FB101230329A745B4B1B78FF2B08D1E0
:107DD80058495B484B786FF300034B70002122F041
:107DE80019FC049A032A40F0238252480021437860
:107DF8006FF300034370524822F00CFC11E2022E8C
:107E080003D1534BC8221A600BE2032E16D1504BF4
:107E18001B68002B40F00C824A4800F14001FEF735
:107E28008DFE1B20FEF72CFF414B5B8AA3F51E63DA
:107E38000F3B9BB2542B00F2FB81F2E1042E0CD1D4
:107E48003B4B988A0FF078FE002840F0F1813D48BE
:107E580000F16001FEF772FEE3E1052E07D1344B15
:107E6800988A0FF069FE032840F0E281D9E1062ED6
:107E780040F0D78122786FF3030301322270D5E1F5
:107E8800344800F12001FEF759FE334B1B78002BD4
:107E980000F0CE81237801332370304B1A786FF3CA
:107EA8000302FFF794B82D4EDFF8A480337813F05F
:107EB8000F021AD12A4800F12001FEF73FFE294897
:107EC800F8F7B8FC274902462748F8F7BBF92548D0
:107ED800F8F7B0FC254BA3F8160233785A1C62F366
:107EE800030333701CF0E4FC91E0012A16D1D8F8A2
:107EF8000030002B40F09C811CF006FD012840F06A
:107F080097811B48F8F796FC194902461948F8F773
:107F1800C1FC002840F08C8111486FE0D8F800209F
:107F2800002A40F085810B217BE000BF321300203E
:107F38004032002062320020701D0020540C0020C6
:107F4800002C014096AE0208641D0020F4010020B8
:107F58000827002016AF0208601D0020611D0020C0
:107F680056AF020874010020E03800201861002094
:107F78009201002019610020874E337813F00F0812
:107F88000CD186484146FEF7D9FD33785A1C62F376
:107F980003033370824BA3F8028049E1B8F1010F63
:107FA80018D18048042121F05EFF002800F04081AC
:107FB8007A4800F12001FEF7C1FD33784FF0FF3118
:107FC8005A1C62F303033370774B64221A60744BB4
:107FD80059802DE1B8F1020FDFF8CC811BD1D8F818
:107FE8000030002B40F024816E48042121F03BFF33
:107FF800002840F01D816A4B5880684800F1400114
:10800800FEF79CFD33785A1C62F303033370642334
:10801800C8F800300CE1D8F80020002A40F00881A8
:108028000C21217062F30303A9E0604910234FF487
:108038000052CB700D3B8B700A805D4821F0C4FE66
:108048000A2200215B48F8F7A5F9802021F020FEDC
:10805800237801332370504B1A786FF303021A7098
:10806800514BC8221A60E3E05348DFF848A100F1F9
:108078002001FEF763FD9AF80030002B00F0D8804D
:108088004E48DAF80020444E0260BAF80420828094
:108098009AF806208271317811F00F0159D1DFF872
:1080A8000881D8F80010002940F0C2809AF804101E
:1080B800A2F5A6524FF0640B103A0BFB01229AF876
:1080C80005004FF00A0909FB00200393F9F728FD82
:1080D8003B49F9F731FE02469AF80200039BA0F5E6
:1080E800A65010380BFB030B9AF80100354B09FB1F
:1080F80000B018600392F9F713FD039A0146104681
:10810800F9F75EFC304B1860F9F716F91EA3D3E9AE
:10811800002382468B46F9F7E9FB002800F08880A7
:10812800504659461AA3D3E90023F9F7D5FB00288E
:108138007ED0FEF7DDFD337848465A1C62F3030310
:108148003370C823C8F8003009F09AFEC0B207900F
:108158006EE001296CD10D300799832200F044FDAF
:10816800114BD3F80080B8F1000F61D1404621F0DF
:108178008FFD237801332370337868F3030333705A
:1081880056E000BFAFF30080736891ED7CFF7F403D
:108198000AD7A3703D008040611D0020B6AF0208D9
:1081A800FE3E0020000C0140082700205E3200201F
:1081B80000100140781D002016B0020804020020BB
:1081C80000007A44741D00205C1D00208448854E00
:1081D80000F12001FEF7B2FCF37913F0010F27D06C
:1081E800DFF8488298F8009019F00F0920D17E4BEB
:1081F8000A2259781878103902FB0011B1701979E0
:10820800D878103902FB00117170D9799B7910392F
:1082180002FB0312327019F093FCF37969F300033F
:10822800F37198F800305A1C62F3030388F80030A1
:10823800DFF8FC9199F8006016F001063EF43BAEB9
:108248006A4B01221A701BF0F1FA2378092B01D02E
:108258000D2B28D10120664912F0EEFC654B664AC9
:108268005B7803F01F03D35C644A522B137002D16E
:10827800634B01221A70634B634A03F1200153F8E0
:10828800040B8B4242F8040BF9D1002109A812F023
:1082980011FD09A80D211CF0A7FA5C4B1A780132D0
:1082A80002F003021A7099F8006006F00206F6B2AE
:1082B800002E00F08B800FF09BFE14F02BFA06982E
:1082C8000322431C93FBF2F202EB42029B1ADBB23D
:1082D8000693002B79D1DFF8488198F84960C246A7
:1082E800002E4DD0022E03D198F80130312B49D001
:1082F80023780E2B13D1464846490522F8F7CAFAC7
:108308008246002840D1B21F37484349F8F718FB86
:10831800344B5646DA7942F00102DA7135E00D2B1A
:1083280003D13E483A49072227E0032B22D13C4B90
:10833800002713F8012F2C2A03D00137FFB2B742C8
:10834800F7D11BA832493A46F8F7FAFA7B1C07E03E
:108358000AEB03025278303AD2B2092A03D8013321
:10836800DBB2B342F4D30AEB0701FA4317A8023190
:10837800D21802E0264911A8721EF8F7E1FA03E0C4
:10838800069E02E0012600E000261E4B204A03F16B
:10839800100153F8040B8B4242F8040BF9D1214B1E
:1083A800214A03F1100153F8040B8B4242F8040BE5
:1083B800F9D1402388F811301C3B88F82230023B61
:1083C80088F84B301BF098FF00E0002699F8003041
:1083D80003F0F5036FF3000389F80030FEF76BBD77
:1083E80056B00208845A0020661D0020321300206F
:1083F800B5600020B460002048E702081C3C00205B
:10840800601D0020F4010020483D0020173B00209B
:10841800235D00204BA30308285D0020781D002061
:10842800225D002004020020345D0020611D002030
:10843800FC5C0020AFF3008010B5044640181146DC
:10844800F8F79AF92046F8F7F5F9C0B210BD42548A
:108458000131C8B27047000010B50D4B0D4A1B78AA
:108468000C460E2101FB0323997A39B10139052302
:10847800594301F56E51443189B201E043F6C431E4
:108488000019042209F00DFD201DC0B210BD00BF67
:1084980039630020C817002010B5054B0C46197821
:1084A80000190131042200F09FFB201DC0B210BD4D
:1084B8003963002000F5364008B54B3009F0E0FC80
:1084C80010F0FF0F14BF0020012008BD10B50A46A8
:1084D80000210446FFF7B0FF01462046FFF7DCFF06
:1084E800114A01462046FFF7A7FF232201462046EE
:1084F800FFF7ADFF01462046FFF7AEFF5B220146BE
:108508002046FFF7A4FF232201462046FFF79FFFDE
:1085180001462046FFF7A0FF7C2201462046BDE821
:108528001040FFF794BF00BF51A3030810B55D22A8
:108538000446FFF78CFF0D2201462046FFF787FF10
:108548000023235410BD38B51D460C4640182C197D
:1085580011461A4600F048FBE0B238BD2DE9F0415B
:1085680018490446FFF7B2FF174F0E263B78174D00
:1085780073430146EA5A20460423FFF7E4FF20220A
:1085880001462046FFF763FF3B78014606FB03538D
:1085980020469A7A0223FFF7D6FF2022014620467A
:1085A800FFF755FF3B78014606FB035520466A7ADC
:1085B8000323FFF7C8FF01462046BDE8F041FFF757
:1085C800B5BF00BF54A3030839630020C8170020B3
:1085D8002DE9F047264E0E223378264F534337F9BC
:1085E8000380FA1824494FF47A73044698FBF3F889
:1085F800157AFFF76BFF4E2201462046FFF727FF4B
:108608001E4B1C2202FB05355FFA88F8B8F1030FF0
:1086180001460CBF05F1120205F108022046FFF7DA
:108628000BFFA1468046002519E019F8013BA32B52
:1086380007D133780E2202FB0373204629465A7A63
:1086480008E0242B09D133780E2202FB03739A7AAF
:10865800204629460223FFF776FF0135EDB245454E
:10866800E3D120462946BDE8F047FFF75FBF00BFCA
:1086780039630020C81700205EA3030868E70208D2
:10868800074B187800F00400C0B240B11A686FF3C5
:1086980082021A60034B00221A70034B1878704745
:1086A800083B00209C1D0020841D0020054B002154
:1086B8001970054B05481A6861F382021A60122284
:1086C800F7F768BE9C1D0020083B0020841D002091
:1086D80038B5084C084922780546F7F7B3FD2378E2
:1086E8000021E954054B1A6861F382021A60207868
:1086F80038BD00BF9C1D0020841D0020083B0020C1
:10870800064A07491378112BC85401D8013313704E
:10871800044A136843F00403136070479C1D00204B
:10872800841D0020083B0020054B1B7813F0010F27
:1087380005D1044B181810F8010CFFF7E1BF70477A
:108748009D1D002096B002082DE9F041334C00230E
:1087580014F8101094F82A2001F00F0161F30302B5
:1087680084F82A2004EB400084F8293084F8283063
:108778004378DFF8B88063F30712638C4FF4D2773D
:10878800E38498F800302A267B4306FB0133244D06
:108798002448E95A84F82A2021F03AFF98F8003052
:1087A80094F82A207B4302F00F0206FB0233EB18F1
:1087B80059881C48013989B221F02EFF01210A4647
:1087C800184821F0F5FE0121164821F0E2FE98F83C
:1087D800003094F82A207B43120906FB0233124822
:1087E800E95A21F015FF98F8002094F82A305743E9
:1087F8001B0906FB0376AD1969880B48013989B254
:1088080021F008FF01210A46074821F0D1FE064859
:108818000121BDE8F04121F0BCBE00BF9E1D002033
:10882800A2B002080008004000340140CA1D002020
:1088380030B5164C94F82B50A38445F0010500235D
:1088480084F82B50628484F8211084F8203019E0D1
:10885800C55CA5F13002D2B2092A08D9A5F14102B6
:10886800D2B2052A9ABFA5F13702D2B22A46084DDC
:10887800013305EB420292F8495392F848232570D8
:1088880062700234DAB28A42E2D330BD9E1D002003
:10889800A2B00208124B10B59A8C0024DA8483F82F
:1088A800294083F82840224601210E4821F080FE05
:1088B80064210C4821F0ACFE32210A4821F0ACFEBC
:1088C80001212246084821F073FE6421064821F060
:1088D8009FFE05483221BDE8104021F09BBE00BF35
:1088E8009E1D0020000800400034014010B5002102
:1088F8002C220348F7F74EFDBDE81040FFF7CABF2A
:108908009E1D002070B5214C2378042B39D8DFE850
:1089180003F0030D152A30001D4B012093F82B306E
:1089280013F0010F30D02070013870BD184B93F848
:108938002000FFF709FF0223237022E0144DEE8C7C
:10894800FEB9FFF7A7FF95F8203095F821200133ED
:10895800DBB29A4285F8203001D8042300E00323D3
:108968002370304670BD0A4BD88C50B90123237050
:1089780070BD074BDD8C35B9FFF7B8FF25700120B6
:1089880070BD002070BD002070BD00BFCB1D002051
:108998009E1D0020044B00225A701A709A7842F0EB
:1089A80001029A70704700BFF41E0020202102487F
:1089B8000A46F7F7EFBC00BFF401002038B50446BB
:1089C80008460D46F7F736FF98B10319202B094BD7
:1089D800C8BFC4F120001C19002308E014F8012BBB
:1089E800E02A14BFEA5C202204F8012C01338342F8
:1089F800F4DB38BDF40100200D4B46F6E9421B6854
:108A08009B6893420FD043F6FC2293420BD0122B63
:108A180009D0B3F5E97F08D046F68D501B1A5842A5
:108A280040EB03007047012070470120704700BFEA
:108A3800041E0020F0B51F4687B006460C460846BF
:108A480000211546F7F7A6FC244B07B19F80B3F920
:108A5800041005A801EB8601042209F022FA002679
:108A680005AB9B5D013BDBB2B92B34D81D2B4FEA1C
:108A7800031208D8D31803F528416846FE3111229D
:108A880009F00FFA0BE01649D3185B186A4603F190
:108A98001007186859680833BB4203C2F9D1204649
:108AA800F7F7C8FEC7B26846F7F7C4FE3818A842F9
:108AB80003D8E0196946F7F75FFE6846F7F7BAFE8C
:108AC8007B1C1B18AB4203D2E0190649F7F7BCFC24
:108AD8000136042EC4D107B0F0BD00BFF41E00203B
:108AE8008C7E030876A3030810B500216C22044687
:108AF800F7F750FC0123A37010BD002343700370E7
:108B0800837843F001038370704700002DE9F0413A
:108B18009378804613F0010F0D4614463AD06FF350
:108B2800000393701BF0C0FB6378002B32D12378CD
:108B38000BB90A336370A378174F6FF30003A37060
:108B48001BF0B2FB217807EB0806611807313046A5
:108B58002A46F7F7F5FE3046F7F76CFEC6B2AE4286
:108B68000DD80AD20023237006EB08000A3363707D
:108B780038182021AA1BF7F70DFCAE420AD122783B
:108B8800A3181B7A1BB101322270BDE8F081237053
:108B98000A236370BDE8F081F4010020054B1A78C0
:108BA8000AB100221A701B7846F68A4202FB0311AA
:108BB800FFF704BFE71D0020F8B505460C46081866
:108BC800002109F053F9013CE4B26719384609F06D
:108BD80057F9C6B2202E03D83846002109F046F9C5
:108BE8000CB1202EEFD9F8BD02F00F03032B22F0B1
:108BF8007F0230B5D2B20CD94FF47A7491FBF4F4F9
:108C08002025E4B2057002B114B13034047000229A
:108C18000130B1F57A7F05DB4FF47A7491FBF4F5F6
:108C280004FB1511022B0BD9642491FBF4F42025C5
:108C3800E4B2057002B114B130340470002201307E
:108C4800632904DD642491FBF4F504FB1511012B61
:108C58000AD90A2391FBF3F32024DBB2047002B192
:108C68000BB1303303700130092904DD0A2391FB6D
:108C7800F3F203FB12113031017030BD13B5104B04
:108C880001461B689A899C7B12F0100214BF0220CF
:108C9800012034B10B4C9B7C2478634303FB001107
:108CA80009B23AB10DF10600022209F0FAF8BDF84E
:108CB800060002E0084609F0E3F800B21CBD00BF58
:108CC800041E0020931E002010B50F4B1B689A89C4
:108CD8009C7B12F0100214BF0221012134B10B4C0D
:108CE8009B7C2478634303FB010000B22AB1084946
:108CF8000222BDE8104009F0CEB8054B1968BDE85E
:108D0800104009F0B3B800BF041E0020931E0020D5
:108D1800AC1E00203038C0B2092894BFFF200020C4
:108D280070470000024B1A786FF300021A70704700
:108D3800E31E002070B5FFF7F5FF884B1A781E2A4E
:108D480001D91E221A70864C2678254606F0F006B0
:108D5800202E72D109F0FCFB00286ED1814B1B78C4
:108D680033B92378C3F30312013262F307135EE0C9
:108D78007D4B1B7803F08003DBB2002B59D07B4876
:108D8800F7F758FDC5B27A4CBDB12046794932464D
:108D9800F7F7D6FD0A2D0BD82A4620467349F7F770
:108DA800CFFD60193146C5F10A02F7F7F3FA04E07E
:108DB80020466E490A22F7F7C3FD6F4B1B7813F064
:108DC800010F01D0472300E02023E372684C0422FE
:108DD80004F10C00A521F7F7DDFA684B1A7852B1B7
:108DE800FF23012A237306D9022A637303D0032AB7
:108DF800A37318BFE373624C257815F0600502D1A0
:108E080094F8A33013B95F485F4902E05D4804F164
:108E1800A3010622F7F794FD5C4B1B78452B40F025
:108E28008D81002D40F08A81237843F080032370E0
:108E380070BD4F485649324675E12C7804F0F0046D
:108E4800102C3FD109F084FB00283BD12022514946
:108E58004748F7F775FD46484E492246F7F770FD33
:108E68004D4B1B7813F0010F06D04C48F7F7E2FC86
:108E78004A4902464A4805E04A48F7F7DBFC4949AF
:108E880002464748F7F75CFD364B1B781BB9464846
:108E98004649102247E1444845491022F7F750FD5A
:108EA800314B1B7803F08003DBB22BB13B48F7F75B
:108EB800C1FC02463F484FE03A48F7F7BBFC024680
:108EC8003C4842E02B7803F0F003302B7ED109F0C8
:108ED8003FFB00287AD1264C202237492046F7F755
:108EE8002FFDA521052204F10B00F7F753FA334BA8
:108EF8001B78042B02D9FF23E37300E002D1FF2380
:108F0800A37301E0032B02D1FF23637301E0022B5B
:108F180002D1FF23237300E00BB1FF23E372284B38
:108F28005B7813F0600F05D03F23E37223736373FC
:108F3800A373E373234B1B7803F02003DBB233B135
:108F48001848F7F777FC02461F481649EBE0134824
:108F5800F7F770FC02461C481049E4E0EF1E0020B9
:108F6800E31E0020382700200C27002010270020AF
:108F7800F40100207844030830630020062800200C
:108F8800412700200E020020931A0308CC1D002060
:108F9800364403087B7A0308F2410020C57B0308A6
:108FA80001020020E67B0308040200204880030831
:108FB8009C7A030811020020381B03082F2D00207B
:108FC80068320020083B00200F0200202B7813F0A5
:108FD800F0030CD120225A495A48F7F7B1FC5A4BF2
:108FE800584819888322BDE87040FFF7FDBD602B03
:108FF8001ED109F0ADFAD8B9544920225148F7F7E3
:109008009FFC5348F7F716FC514902465148F7F7B9
:1090180097FC5148F7F70EFC4F4902464F48F7F7BF
:109028008FFC4F48F7F706FC4D4902464D487AE059
:109038002B7803F0F003102B06D109F089FA18B148
:109048004048494920226EE02B7803F0F002402A7C
:1090580002D0502A6BD10AE0444920223948F7F758
:109068006FFC0FF043FD04460FF05EFD09E0404938
:1090780020223448F7F764FC0CF068F904460CF039
:1090880089F9FF2806D13B48F7F7D4FB394902464E
:10909800394817E0FD2806D13848F7F7CBFB3749A0
:1090A800024635480EE0022806D13548F7F7C2FBDC
:1090B80033490246304805E03248F7F7BBFB3149EF
:1090C80002462D48F7F73CFC202107222E48F7F7E7
:1090D80061F9FE2C06D12748F7F7ACFB2549024673
:1090E800294820E0012C06D12848F7F7A3FB274997
:1090F8000246254817E0022C06D12548F7F79AFBC7
:109108002349024620480EE0042C06D12148F7F7EF
:1091180091FB204902461C4805E01F48F7F78AFBE7
:109128001D4902461848BDE87040F7F709BC1B4ABC
:109138006FF3071313701A4B00221A6070BD00BF3B
:10914800D51A0308F4010020E21D0020B41A030810
:10915800B4130308F8010020BE1303080802002016
:10916800B91303080F020020171B0308BD7A030870
:10917800DE7A0308077C0308FD010020287C030829
:10918800837B0308C57B03080D020020FF7A0308D0
:10919800207B0308417B0308627B0308E31E002051
:1091A800041E0020204B70B5F022204D1A702B7839
:1091B80013F0010F0BD01E4C207810F0010006D1DF
:1091C8001C49FFF7EBFC237843F0010323701A4E88
:1091D8003378532B0ED1164C237813F0010F07D098
:1091E80000201649FFF7DAFC23786FF30003237099
:1091F800FFF798FD3378232B14D10D4B1B7813F010
:10920800010F0FD1FFF78EFD2B780D4A43F00603AF
:109218002B701378013BDBB213700A4A52F82320F3
:10922800094B1A6070BD00BFEF1E0020E31E00202E
:10923800091E00204C700308CC1D00202B70030869
:10924800C31E0020D01E0020041E00202DE9F0417E
:109258005E4BF0225E4D1A702A7802F01003DBB2E2
:10926800002B2DD15B4963F347120B601C462A7013
:10927800594A9A5C2D2A01D00134E4B20133112BEA
:10928800F6D1564E3A213046F7F702F938B1801B2D
:10929800C0B20130301821460222FFF7A5FC504B1E
:1092A8001B78452B40F08F8000242046013413F0B2
:1092B80089FA112CF9D12B7843F010032B703CE07C
:1092C800484C237813F0010F17D1424E4648FFF758
:1092D8000BFC424F3168384601310222FFF784FC0B
:1092E8002D23BB70307846F6157340496522FFF789
:1092F800A1FB237843F00103237003200D213A4A90
:10930800FFF704FC2D78324E15F0E00545D110200A
:109318003749FFF743FC324B1B78442B11D12D4AB8
:10932800136801331121B3FBF1F101EB01115B1A51
:109338002949C95C2D29F4D01360BDE8F041FFF735
:10934800F1BC532B0DD132784E3B63F34712327088
:10935800204A28491268062000FB02125380BDE803
:10936800F081232B2FD11B4B1D60337803F0EF03C3
:1093780065F347133370FFF7D5FC23781E4A43F093
:10938800060323701378013BDBB213701B4A52F8B3
:1093980023201B4B1A60BDE8F081104C102019499E
:1093A800FFF7FCFB04F110002821F7F771F850B122
:1093B800001B3178C0B20130201849098022BDE86D
:1093C800F041FFF711BCBDE8F08100BFEF1E00209F
:1093D800091E0020AC1E0020CD3E0020F401002014
:1093E800CC1D0020E31E0020F41E0020FB1E0020E0
:1093F800C86F0308FE3E0020C31E0020D01E0020B8
:10940800041E0020E96F0308454B2DE9F041F022C6
:10941800444E1A703378444D43F0010333702B687F
:10942800424C9B7C022B06D1414B1B7803F0400336
:10943800DBB23BB10FE0012B0DD13E4B1B7813F093
:10944800010F08D109F0FCF9236800206FF3555388
:109458002360394944E0A378344F03F02003DBB29A
:10946800C3B909F0EDF9F87800F02000C0B288B966
:109478002968324B897C1A7861F301021A703B68BB
:109488002D4943F400133B60FFF788FB2C4B8022E7
:1094980083F843200DF000FF804678B12B689B7C51
:1094A800012B08D1234B5B7803F01003DBB213B117
:1094B8000020244914E00020234911E00DF01CFF8E
:1094C800074610B1404621490AE00DF05DFF10B192
:1094D80038461F4904E01A4B93F8433013B91D4925
:1094E800FFF75CFB1C4B1B78232B16D1FFF71AFCEC
:1094F800337843F00603337009F0A2F923686FF359
:10950800555323600CF082FD144A1378013BDBB2FB
:109518001370134A52F823302B60BDE8F08100BF66
:10952800EF1E0020E31E0020041E0020083B002040
:109538000C270020F24100206D700308F74100203D
:109548008D220020AF7003088E700308F1700308A5
:10955800D070030812710308CC1D0020C31E002020
:10956800D01E00202DE9F341704B714DF0221A7086
:109578002B68704C9B7C1BB9637843F0020302E0B4
:10958800637843F001036C4E6370337843F0010352
:109598003370238823F4FF739B059B0DB3F5007F7D
:1095A80007D0664B1B787BB1624B5B7813F0010FD9
:1095B8000AD0237800206FF3861361492370FFF7E0
:1095C800EDFAF8F77DFD84E023785A4F03F0400365
:1095D800DBB2FBB9BB78EBB95A4B93F8008018F0B3
:1095E800010817D1F8F76CFD3B7843F040033B7056
:1095F8002B68B3F91030022B3B780CBF43F0800383
:1096080068F3C71300213B70082001220B46009124
:10961800F9F776F8A378474A032B28D003D8012B0B
:109628000BD00DD806E0052B2DD0117825D3FF2BB4
:1096380032D12BE00020424949E00020424946E06F
:109648004248F7F7F7F8DFF83C81C7B23F4908F11D
:1096580010003A46F7F774F90F2F3AD807F11000BF
:1096680040442021C7F11002F6F794FE31E0384B50
:10967800187800282DD1374929E06FF38611117029
:109688000020354923E00020344920E06FF386119B
:109698001170002032491AE0053BDBB26FF38611E6
:1096A800022B117002D100202E4910E0012B02D1AB
:1096B80000202D490BE0032B02D100202B4906E0A6
:1096C800052B02D100202A4901E02A490020FFF792
:1096D80065FA237803F04003DBB20BB9F8F7F0FC26
:1096E800254B1B78232B1ED1FFF71CFB33782278E0
:1096F800617843F00603337001F0FE01002302F0A5
:10970800BF0263F3C71263F34101A3702270617053
:10971800F8F7D6FC194A1378013BDBB21370184AE4
:1097280052F823302B60BDE8FC8100BFEF1E0020FB
:10973800041E002030630020E31E002002370020B2
:109748006D70030836630020B06C03083F63002087
:1097580034630020D16C030875710308556D030844
:10976800B86D0308F26C0308136D0308346D030821
:10977800766D0308976D0308CC1D0020C31E0020DA
:10978800D01E0020F40100207B4B2DE9F341F0228C
:109798007A4E1A7033787A4D43F0010333702B6890
:1097A800784C9B7C022B11D1774B1B7803F040033C
:1097B800DBB293B1754B1B7803F02003DBB2BBB16E
:1097C800A37803F04003DBB23BB111E0012B0FD1CA
:1097D8006F4B1B7813F0010F0AD1F8F771FC23685F
:1097E800002023F480036FF3D753236069498FE087
:1097F800A778DFF8908107F04003DFB2002F34D15B
:10980800F8F75EFC2968644B897C1A78384661F35E
:1098180001021A70D8F800305E4943F4800367F3F8
:10982800D753C8F80030FFF7B9F92B68198A21B95E
:109838000091082001220B4615E00BB2022B0CD137
:1098480001223B46082039460097F8F759FF534B49
:109858001A7842F008021A7007E0012B05D1009728
:109868000E2039463A46F8F74BFF0DF015FD07462E
:1098780078B12B689B7C012B08D1454B5B7803F0B2
:109888001003DBB213B10020454941E000204549EF
:109898003EE0414B3946187800F00300F8F74AFDDE
:1098A800FF280FD13D4B1B7803F01803182B31D03C
:1098B800A07800F08000C0B210B138463A4927E0DD
:1098C8003A4925E00DF018FD8046E0B1334B187891
:1098D80000F008085FFA88F8B8F1000F0AD1F8F725
:1098E8007FFEC0B2022801D840460AE0062811D8F7
:1098F800404604E000F01000C0B210B138462C49D0
:1099080006E02C4904E00DF03FFD18B12A49404615
:10991800FFF744F9294B1B78232B29D1FFF702FACB
:10992800337843F006033370F8F7CAFB236823F44F
:1099380080036FF3D7532360184B1A786FF3C30271
:109948001A701F4A1378013BDBB213701D4A52F894
:1099580023302B60104B1B7803F00303022B02D13A
:109968000DF070FC20B102B0BDE8F0410CF04EBB28
:1099780002B0BDE8F08100BFEF1E0020E31E00200A
:10998800041E0020083B00200C270020412700204F
:10999800F24100206D700308F74100201C200020D0
:1099A800AF7003088E700308757103089671030879
:1099B8005471030833710308D0700308CC1D0020CC
:1099C800C31E0020D01E002010B5FFF7ABF90A48CF
:1099D8002523C377094B0A4A1B6824219B7C1C302A
:1099E80001FB03235B781A3903F00F0359438322E1
:1099F800BDE81040FFF7F8B8F4010020041E00206D
:109A0800183B00202DE9F047514D524F2B78F0229A
:109A180043F001032B70504BDFF878911A703B68C4
:109A28009C6847F67313E21A544244EB020424215B
:109A380061434A4A565C5318C6F300065FFA86F833
:109A48009246B8F1000F23D140464549FFF7A6F8E2
:109A580099F80030232B79D1FFF764F92B78414A24
:109A680043F006032B701378013BDBB213703E4AB8
:109A780052F823303B603D4B1E703D4B1E703D4BF2
:109A88001E703D4BC3F800803C4B1E70BDE8F0874C
:109A980099F80020232A21D19A786FF300029A704E
:109AA8000EF052FBFFF73EF92B782E4A43F00603DF
:109AB8002B701378013BDBB213702B4A52F823301A
:109AC8002A4A3B6000231370294A1370294A1370ED
:109AD800294A1360294A1370BDE8F087532A13D125
:109AE8009A7812F001010FD172206043244D42F0A0
:109AF80001022E5C61F300062E549A701E4B01225F
:109B08001A60204617F016FA242303FB04A39B7857
:109B180013F0010F02D000201A4913E0164B1B68FE
:109B280073B9382102221848FFF75EF8204616F06C
:109B380081FC014615480222BDE8F047FFF754B8FA
:109B480013490020BDE8F047FFF728B8BDE8F087C3
:109B5800E31E0020041E0020EF1E0020183B0020FA
:109B680003290308C31E0020D01E0020E91D002081
:109B7800121E0020931E0020AC1E00209E1E0020F6
:109B880090590020A6730308120200200D0200203D
:109B980085730308CC1D00202DE9F0412D4E2E4F72
:109BA800307800F5E640713008F06AF93B78C4B2C5
:109BB80013F0010F26D0294D2B78552B0AD1EC2C08
:109BC80001D0013CE4B23078214600F5E64071301E
:109BD80008F04CF92B78442B0DD1A4F11403DBB217
:109BE800D72B01D90134E4B23078214600F5E6409C
:109BF800713008F03BF92B78532B03D1FFF792F81B
:109C08000EF0A2FA164B1B7803F08003DBB253B1B7
:109C18003B7813F0010F06D0124820210422BDE83A
:109C2800F041F6F7B7BB14F0800F0F4805D12B238E
:109C38000A2103746143113006E02D230374373B76
:109C48005C43113004F520610322BDE8F041FEF7C2
:109C5800CBBF00BF931E0020E31E0020CC1D0020B8
:109C6800083B002004020020F40100201FB5204B0F
:109C780020491A781AB1087840F00100087009786C
:109C88001C4C11F0010F31D01B490978532901D020
:109C98000AB103E082B901221A700DE023290BD121
:109CA800002018701549FEF779FFFFF73BF8237875
:109CB80043F00603237019E01B78012B16D12021ED
:109CC8000A460F48F6F766FB0E4B68461B681022DB
:109CD800996808F0E6F8002409491DF8040001EB2A
:109CE800440101341BF036FC102CF5D11FBD00BF18
:109CF800931E0020E31E0020CC1D0020BE76030822
:109D0800F4010020041E0020034B1B78532B01D1C3
:109D1800FFF708B8704700BFCC1D0020084BFF288C
:109D28001A68936807D1917B41B10649927C0978FA
:109D380001FB023302E0927C02FB003318467047B5
:109D4800041E0020931E00204328F8B504460D4643
:109D5800174608D1114B0A261A7891FBF6F66FF3CD
:109D6800C3021A7000E00E462046FEF7D3FF90B1FA
:109D78000A4B303C1A780A2602F00801C9B20029B9
:109D880018BF002506FB05466FF3C30236B21A70EA
:109D9800BE42A8BF3E4630B2F8BD00BFE31E002059
:109DA800614B2DE9F3411A689846157C977C5F4C06
:109DB8002DB15F4821780222FEF716FF00E02570DA
:109DC800FF01237807F51E47E83707EB4307594E8D
:109DD8000BB90DB10FE015B901A8394601E001A88A
:109DE800B91E022208F05DF89DF80430F3759DF85D
:109DF8000530337605E006F117003F210222F6F719
:109E0800C9FA5B23B375023373764B4B1B7813F097
:109E1800010F5DD0494B1B78A3F13002D2B2092A59
:109E280031D822780AB9002D3CD1454A1178964696
:109E38009942444A01D00021117043481178A3F196
:109E4800300490F800C004EB840404EB010802A875
:109E580001318444C9B23D48641810F80880005D97
:109E68000CF8048C117008B1032901D90021117074
:109E78008EF800300DB9384600E0B81E01A902225C
:109E880008F009F817E0232B04D12F4B1A7892B960
:109E9800013205E02A2B05D12B4B1A785AB1013A29
:109EA8001A7008E0532B06D1294A533B1370264AEF
:109EB8001370FFF729FF274B1B7803F08003DBB2F1
:109EC800002B2FD0204B1B78F6182023F37529E0A0
:109ED80045B31A4B1878A0F13003DBB2092B10D820
:109EE8001B4A137803B92370013303F0010313707D
:109EF800D8F800302178B3F91020FFF725FF20703B
:109F080005E0432803D1124B1B7803B92370114B8A
:109F18001B7803F08003DBB223B10548202102221D
:109F2800F6F738FABDE8FC81041E0020131E002055
:109F380002020020F4010020E31E0020CC1D0020B6
:109F4800E61D0020121E0020E41D002010B40208A7
:109F58009E1E0020083B0020F7B5384E384D337858
:109F6800384C6FF34103337019F090FFFFF7CCFEC4
:109F780002238DF807302B7883B1334AD17941F029
:109F88000101D171314A207802EBC3035F6B93F86A
:109F980039203978FFF7D8FE38700DE0337813F0A0
:109FA800010F06D02378303BDBB2062B9CBF264A34
:109FB800D37003238DF80730337813F0010F12D0D4
:109FC800234B1B7803F08003DBB263B129781F4B66
:109FD800204803EBC10393F838309DF80720C018D8
:109FE8002021F6F7D7F92378232B09D11A4A2B78A1
:109FF8001268927C013A934202DA114A01331370D3
:10A0080023782A2B04D12B7813B10D4A013B137006
:10A018002378532B0FD117F093FD0B4B0021297098
:10A02800DA7961F30002DA71FFF76EFE0B4B9A7969
:10A0380042F004029A7100232370FEBDE31E002043
:10A048009E1E0020CC1D0020845A002010B4020857
:10A05800083B0020F4010020041E002010200020EE
:10A068002DE9F74F864E874C3378874D232B874F42
:10A0780025D12368986843F6F123984217D1DFF871
:10A088003482296898F8000000F56A50713007F0AA
:10A09800EDFE98F80000013000F0010088F800009B
:10A0A80000F56A50713007F0EBFE286007E000B257
:10A0B800FEF7E4FD28603B7843F008033B703378F3
:10A0C800532B40F06E81236849F695629B68934252
:10A0D80002D12A686E4B15E04BF23662934202D1E8
:10A0E8002A686C4B0EE04BF2B352934202D12A68B5
:10A0F800694B07E049F6E662934204D12A68674B48
:10A1080002B101221A7023689A6843F6DD239A4245
:10A118000AD1634B29681A7861F300021A7008F0B3
:10A1280017FA08B108F032FA236843F6E0229B6870
:10A13800934206D15A4B29681A7861F3C7121A70EC
:10A1480019E043F6EA22934206D1554B29685A781A
:10A1580061F300025A700EE043F6E72293420AD1F7
:10A168002968504B19B11A6842F0005202E01A6887
:10A1780061F35D721A6023689A684BF2CC639A4265
:10A188000AD12968484B19B11A7842F0040202E052
:10A198001A7861F382021A7023689A684BF259732D
:10A1A8009A4202D128781AF0D9FB236843F6DA22BA
:10A1B8009B68934202D12A683C4B05E043F6DE22B5
:10A1C800934203D12A683A4B1A7008E049F69E6216
:10A1D800934204D12B6813B92B4B01221A602368D0
:10A1E8009A684BF25A739A420BD1324A2B6812780A
:10A1F8003149032B8B5404D1304B5A7942F0100269
:10A208005A71236849F6DE629B68934202D1296835
:10A218002B4A05E049F6E162934203D12968294AAD
:10A22800117016E049F6E262934203D12968264A82
:10A23800117015E049F6E462934203D12968234A74
:10A2480011704DE049F6E562934202D12A68204B2D
:10A2580013E043F60852934202D12A681D4B0CE0E2
:10A268004AF6EC02934202D12A681B4B05E04BF2F6
:10A278004A62934234D12A68184B1A703BE000BFF7
:10A28800CC1D0020041E0020AC1E0020E31E002070
:10A2980038270020F03A0020E7340020CA1D0020AB
:10A2A800611F0020083B002030630020125D002061
:10A2B800783B0020931E0020C0170020E0260020D5
:10A2C800C4420020C2420020F5410020694100201C
:10A2D80090200020FE150020AD1C0020821D0020CB
:10A2E80049F69662934206D12A68A04B01201A705B
:10A2F80001460EF063FD2368986843F6F1239842FF
:10A308000DD1DFF87482296898F8000000F56A50CA
:10A31800713007F0ABFD002388F8003002E000B28E
:10A32800FEF7D2FC23689A6843F698139A4236D10E
:10A338002968DFF840B2DFF848A20BEBC1031B79AC
:10A34800DFF83482C3F34113012BDFF8389221DDA3
:10A3580098F8000000F56650203007F087FD98F85F
:10A368000030DAF8001009EB030211720BEBC1029E
:10A378001279C2F34112032A0CD17D4A12689068FF
:10A388001030C01807F072FD98F80030DAF8002095
:10A398004B441A7498F800302A6809F80320FFF72C
:10A3A800B3FC3B78DFF8E08113F0010F00F0EE809A
:10A3B800216843F698128B68934240F081806D4A79
:10A3C8002B68914602EBC3010979C1F341110129B8
:10A3D80006DD694A1278072A02D9FEF7A3FCE1E0F4
:10A3E8003278442A36D15FFA83F82DE008F1010863
:10A3F800604B5FFA88F803EBC8031B79C3F341137A
:10A40800012B06DD5D4B1B7823BB5B4B1B78072BB1
:10A4180020D8DFF864A19AF800303F2B08D808F05C
:10A4280097F870B109EBC8031B7913F0100F08D126
:10A438009AF800303F2B07D909EBC8031B79DB09D1
:10A4480002D0C5F8008005E009EBC8031B7913F0BA
:10A45800080FCBD03378552B40F0A4802E782CE011
:10A46800013EF6B209EBC6031B79C3F34113012B76
:10A4780009DD424B1B78002B40F094803E4B1B7843
:10A48800082B00F28F80DFF8F08098F800303F2B1F
:10A4980008D808F05DF870B109EBC6031B7913F012
:10A4A800100F08D198F800303F2B06D909EBC603E6
:10A4B8001B79DB0901D02E6074E0002ED0D171E049
:10A4C8004BF25A7293420AD005DCA3F536424A3A57
:10A4D800012A0ED803E04BF2B772934209D13378C0
:10A4E8002F2B5FD9B1F91020303293425ADC303B20
:10A4F80030E043F6F122934207D11F4B1B7823B17A
:10A508003078B5F900103B222CE008F021F818B398
:10A51800236843F6C4219A688A4203D047F281210E
:10A528008A4204D13078B5F900102D221AE0A2F53C
:10A538006A516139052903D943F6E9218A4201D1D3
:10A54800012307E043F6E0218A4202D00A318A4219
:10A5580003D100232B6025E023683078B5F900107B
:10A56800B3F91020FFF7F0FB28601BE0863F0020BE
:10A57800041E002014040020931E00204A0D002011
:10A58800AC1E0020302D0020E31E00202368B3F904
:10A598000800FEF773FB286098F8003043F00803C2
:10A5A80088F80030FFF7B0FB236843F6D22298689A
:10A5B80090420BD12B6813B99C489D4901E09B48F8
:10A5C8009C490222F6F7BCF90226B0E14BF2B772B9
:10A5D80090420AD12B6813B99748984913E0012B88
:10A5E80095480CBF964997490DE04BF25A72904234
:10A5F80018D12B68012B02D18F48934903E0022B15
:10A6080005D18D4891491022F6F79AF98EE1032B6E
:10A6180002D189488E49F6E7042B87480CBF8D493B
:10A628008D49F0E74BF24A6290420AD12B6813B980
:10A6380081488A49E7E7022B7F480CBF8849894946
:10A64800E1E74BF24B6290420AD12B6813B97A4882
:10A658008549D8E7012B40F0698177488349D2E7DB
:10A6680049F6E362904203D043F6EE2290420ED1BF
:10A6780028680A21B0FBF1F201FB12017C4B303152
:10A68800D97730322E2199775A7703264FE143F64E
:10A69800F12290423ED1774B1B78E3B90222296818
:10A6A8007548FEF7A1FA43F6F220FEF7E7FA022210
:10A6B80001465E48FEF798FA3B7813F0010F00F068
:10A6C80086816E4B1B7803F08003DBB2002B00F011
:10A6D8007E81694819E0FEF7D1FA022201466648F0
:10A6E800FEF782FA022251482968FEF77DFA3B7884
:10A6F80013F0010F00F06B81604B1B7803F08003AF
:10A70800DBB2002B00F06381484820210222F5F7D4
:10A7180041FE5CE143F69812904240F0F5802B68C8
:10A72800574EDFF8508156F8331010224248F6F79A
:10A7380007F90DF1060298F800000DF1070110F075
:10A7480019FC4246334620B316784E49895D0329E1
:10A758001FD0296803EBC1010979C1F3411101290F
:10A7680017D1072E15D948490B224848F6F7E8F8BB
:10A778004748711C0222FEF737FA9DF80710454832
:10A7880001310222FEF730FA9DF8061042480131E5
:10A7980018E02E68157803EBC601097903EBC606A5
:10A7A8003679C1F34111012906F00706C8BF05F043
:10A7B8000705012E0ADC394934480B22F6F7C0F8A0
:10A7C8003348691C0222FEF70FFAAFE0022E0BD1C4
:10A7D80033490B222D48F6F7B3F832462C48691C4A
:10A7E800FEF702FA0E36A2E0032E0BD12D490B22FA
:10A7F8002648F6F7A5F82648691C0222FEF7F4F960
:10A808000D3694E0042E51D127490B221F48F6F744
:10A8180097F81F48691C0222FEF7E6F91D4805F162
:10A8280009010222FEF7E0F90C3680E0120200204E
:10A8380074B4020876B4020804020020A262030875
:10A84800E4620308C3620308796103089A61030894
:10A85800BB610308DC610308586103084763030808
:10A868008963030868630308CB630308EC63030880
:10A87800F4010020931E00200F020020083B002056
:10A8880014040020302D0020307D0308F901002039
:10A89800FA010020FE01002001020020EE7C0308DE
:10A8A800497C0308CD7C03088B7C0308052E11D155
:10A8B80048490B224848F6F743F84848691C0222E1
:10A8C800FEF792F9464805F109010222FEF78CF9D4
:10A8D8000B362CE0062E29D142490B223E48F6F7CA
:10A8E8002FF83E48691C0222FEF77EF93C4805F124
:10A8F80009010222FEF778F93B4805F1110102220D
:10A90800FEF772F90A3612E0B3F91060092E04DD79
:10A91800632ECCBF0326022600E0012633482968AF
:10A92800801B46F08002FEF75FF900E010263B78B6
:10A9380013F0010F0BD02E4B1B7803F08003DBB212
:10A948002BB12A482021801B3246F5F723FD294EDA
:10A95800B37803F00203DBB2002B38D0FEF74CF8D3
:10A96800254D034628B92878F11D6522FEF762F8BF
:10A9780008E0B2792978B388F01D01FB023109B2E9
:10A9880007F08FFA236847F281229B68934213D01D
:10A9980006DC43F6C42293420ED043F69E5209E0E9
:10A9A80047F20132934207D049F69E62934203D0A0
:10A9B80047F2C12293420AD105200B210D4AFEF726
:10A9C800A5F829780D4801310222FEF70DF9BDE8F6
:10A9D800FE8F00BF6A7C0308F9010020FA010020FD
:10A9E800FE010020AC7C03080202002014020020B3
:10A9F800083B0020F41E0020931E0020F5010020D3
:10AA0800F0B5114B1F78114B303F1E680DE0D6F89A
:10AA180014C01CF803C00133644501D112E00023BF
:10AA2800DAB28242F3D301350D70094B0622094987
:10AA380002FB07330D785B1993F86840002CEED1C0
:10AA48000C70F9321046F0BDCC1D0020041E002009
:10AA580010B40208121E00202DE9F74F964C974EAD
:10AA680023689A6843F609539A4203D133780BB99D
:10AA7800013333702368924F99689B7C3A78B3F11D
:10AA8800010848BF03F106084FEAE808337808F1DF
:10AA9800010812F0010F03FB08188A4D00F0AD8081
:10AAA800894B1A789946432A4DD128780FFA88FAA3
:10AAB8000AEBD00007F0E4F92268844B916846F667
:10AAC80048029142186001D12A783AB12A780121C6
:10AAD80002F0070211FA02F250401860287819783B
:10AAE8000AEBD00007F0C2F9236847F261329B688D
:10AAF800934209D1734B1A78754B03EBD203734A0F
:10AB0800126883F8A0211EE046F62952934205D127
:10AB18003178002001310EF0CBFC14E046F63F1AE4
:10AB28004FF0000B23689B68534504D101200BEBC1
:10AB380000010EF0BDFC0AF1080A46F67F139A459B
:10AB48000BF1010BEED199F80030232B10D12268BC
:10AB58002B78927C013A93420ADA5A4A01331370ED
:10AB68005C4B9B7803F00203DBB20BB1FDF712FFDD
:10AB780099F800302A2B0CD12B7853B1514A013B5C
:10AB88001370544B9B7803F00203DBB20BB1FDF753
:10AB980001FF99F80030552B14D12368997C0F29AF
:10ABA80010D92A7808398A42464B01DA083200E07F
:10ABB80000221A70474B9B7803F00203DBB20BB1FB
:10ABC800FDF7E8FE99F80030442B42D123689A7CBF
:10ABD8000F2A3ED929783B4B072902D90839197021
:10ABE80001E0083A1A703B4B9B7803F00203DBB292
:10ABF800002B2ED0FDF7CEFE2BE049F65563994287
:10AC08000ED1314B1B78A3F13101C9B2072907D8FE
:10AC180042F006023A7007225343284A573B137002
:10AC280023689A6843F609539A4212D133781B2B4A
:10AC380008D9284B46F615629A809A7842F00202A3
:10AC48009A7006E05901C918234B0020C918FDF76E
:10AC5800A5FFFFF759F8214A2B78117893469942B6
:10AC680088BF137012780F32934202DD1B4A0F3BE4
:10AC7800137023684FF0000A93F81290B9F10F0F80
:10AC88009ABFC9F120095FFA89F94FF010099BF8BA
:10AC980000004FFA8AF318180FFA88F202EBE00066
:10ACA800019307F0EDF89BF80020019B5FFA80FC08
:10ACB8009B1803F007032AE0041E0020931E0020BF
:10ACC800E31E00209E1E0020CC1D0020AC1E00208C
:10ACD800302D0020F41E0020FC650308951E00207E
:10ACE8004CFA03F06549013300F0010000280CBF5D
:10ACF800A520DB20DBB201F809000AF1010A09F1FD
:10AD08000109082B5FFA8AFA5FFA89F903D0B9F1C9
:10AD1800200FE5D109E0B9F1200F06D023684FFADA
:10AD28008AF19B7C89189942B1DB3B7813F0010FBB
:10AD380015D0236852499B7C09780F2B01F08001BC
:10AD480098BFC3F11003C9B294BFDBB2002331B17D
:10AD5800297810318A1A4949CB185F219954DFF8AC
:10AD6800288198F80230474603F00203DBB2002B33
:10AD780064D0FDF741FE034600BB226846F6295120
:10AD880092688A4206D024318A4203D043F6E511FC
:10AD98008A4204D130783B496522002309E043F612
:10ADA80009518A4208D130781C38C0B208F107012D
:10ADB8006522FDF73FFE18E02878F7E7236846F696
:10ADC800E9429B68934203D043F6FC22934202D1A6
:10ADD800BA79317801E0BA792978BB88294801FB2A
:10ADE8000231BA7909B207F05CF823689A7C102A14
:10ADF80002D905200B211EE09B6846F6E9429342E2
:10AE08000ED006DC43F6E512934209D043F6FC2245
:10AE180004E046F62952934202D02432934201D1EB
:10AE2800102007E043F60952934202D10020102176
:10AE380001E000200721144AFDF768FE226846F663
:10AE48008D5193688B4216D046F647418B4212D0FB
:10AE580043F6ED218B4202D1084BDB219977937C95
:10AE6800102B08D9297809480131022203B0BDE81E
:10AE7800F04FFDF7B9BE03B0BDE8F08FF401002034
:10AE8800083B0020FB1E0020F41E0020F5010020D6
:10AE9800114B002270B50D461A7118B11B7803B911
:10AEA80020234370BDB10D48F5F7C4FC0446681C67
:10AEB8005CB10A492246F5F7C5F9022C0BDC601C87
:10AEC80028182021C4F1030201E020210322BDE853
:10AED8007040F5F75FBA70BD801E0020811E00200B
:10AEE80038B50546002408E0601906F0C9FF303877
:10AEF800C0B2092808D80134E4B2044B1B78303BAF
:10AF08009C42F1DB012038BD002038BDE81D00203F
:10AF180008B506F0B5FF0023C0B2064AD25C8242EB
:10AF280001D1202804D10133082BF6D1002008BD17
:10AF3800012008BDB4B4020870B506460D460024C9
:10AF48000DB12D232B55A0190021013406F08EFFD9
:10AF5800062CF5D170BD00002DE9F04F954C964EAA
:10AF6800226896F80090936892F8128099B208FBCC
:10AF7800091848F6BC20834287B01FFA88F80BD11D
:10AF88008E490878497800F00700C1F3420101EBC7
:10AF9800C00108EBC10825E048F67C4083420CD18B
:10AFA800864908784D7800F0070088214843C5F3A2
:10AFB8004205773901FB05010DE049F2340083426F
:10AFC8000BD17E490878497800F00700C1F34201A7
:10AFD80001EBC0018901884404E0B3F5E97F08BFAB
:10AFE80001EB4908764F774D397811F0010F52D1AE
:10AFF80047F28912934204D046F68972934240F090
:10B008004681714A12782A2A3CD1704A92F800A0E7
:10B018000AF1010A0AF0010A82F800A0BAF1000F49
:10B028001BD046F68972934208D1694B46F61562E1
:10B038009A809A7842F002029A7028E12021102220
:10B048006448F5F7A7F94FEA49139944624B002081
:10B0580009EB0301FDF7A2FD19E15D48FDF744FD89
:10B06800236850469A6846F689739A420CBF5B4932
:10B078005B49FDF793FD31785A4801310222FDF70B
:10B08800B3FD04E1552A02D0442A40F000814F4B19
:10B0980000221A70FBE05069F5F7CCFB4A4B834657
:10B0A80093F800A09946BAF1450F02D14E4B002201
:10B0B8001A705046FDF72EFE00284FD04B4B5FFA12
:10B0C8008BFB1A7852450ED15846FFF799FCFF289A
:10B0D80004D15846FFF794FCFF283FD0444B1A7818
:10B0E80001321A7015E0DFF808A100228AF8002062
:10B0F80058460593FFF784FCFF28059B04D09AF86F
:10B10800002001328AF8002099F80020FF281A70E0
:10B1180024D02168374A4B6910601B5C886847F265
:10B12800891188421360924610D1562B01D0542BB6
:10B138000CD13378123BDBB2022B07D82B780FFAED
:10B1480088F0C01806F09CFECAF800002B780FFAA9
:10B1580088F0C018DAF8001006F088FE99F8003078
:10B16800552B17D12368997C0F2913D92A780839C8
:10B178008A42144B01DA083200E000221A70144B9C
:10B188009B7803F00203DBB20BB1FDF703FC184B0D
:10B1980000221A7099F80030442B3AD123689A7C1F
:10B1A8000F2A36D92978074B072925D90839197064
:10B1B80024E000BF041E0020931E0020991E0020DA
:10B1C800E31E00209E1E0020CC1D0020EE1E002045
:10B1D800F41E0020F40100201F5E0308305C030801
:10B1E800725C0308F5010020E41D0020E61D002024
:10B1F800121E0020AC1E0020083A1A70964B9B784D
:10B2080003F00203DBB20BB1FDF7C4FB934B002242
:10B218001A7099F80030432B0DD123680FFA88F083
:10B228005B6919788E4B19602B78C01806F01EFEE2
:10B238008A4B00221A7099F80030232B13D1226808
:10B248002B78927C013A93420DDA864A01331370C7
:10B25800824B00221A70804B9B7803F00203DBB20A
:10B268000BB1FDF797FB99F800302A2B0FD12B78FB
:10B278006BB17C4A013B1370784B00221A70764BF5
:10B288009B7803F00203DBB20BB1FDF783FBFEF7FB
:10B298003BFD754A2B7811789246994288BF137006
:10B2A80012780F32934202DD6F4A0F3B1370236806
:10B2B8004FF0000B93F81290B9F10F0F9ABFC9F134
:10B2C80020095FFA89F94FF010099AF800000FFA7F
:10B2D80088F318185844059306F0D2FD634A02F81B
:10B2E800090009F101095FFA89F9B9F11F0F059BF6
:10B2F80005D821680BF1010B897C8B45E5DB397892
:10B3080011F0010F17D021685948897C00780F295E
:10B3180000F0800098BFC1F11001C0B294BFC9B25B
:10B32800002140B128789AF800C010305218CCEBB0
:10B3380000005F211154226890684AF6EA029042A0
:10B348000AD14C4B1B78532B30D106F099FD4A4B50
:10B35800187006F08FFE29E0B0F5E97F26D1454A3E
:10B368001278532A22D11846FFF7D2FD8046E8B951
:10B378003378DA00D31A03F11200FFF7B1FD68B190
:10B38800FF2300933D4BCDF804801B7879200133CF
:10B39800029341460422434606F0F0FD337800212B
:10B3A800DA00D31A03F11200FFF7C6FDDFF8A89000
:10B3B80099F80230C84603F00203DBB2002B68D0CC
:10B3C800FDF71AFB034688B9226849F234019268EE
:10B3D8008A420BD046F689718A4214BF28783078A1
:10B3E80009F107016522FDF725FB12E0236898F8AB
:10B3F80006209B682248B3F5E97F0CBF317829788D
:10B40800B8F8043001FB023198F8062009B206F0BA
:10B4180048FD23689A7C102A13D89B6848F6BC22FA
:10B4280093420BD13B7813F0010F01D010202CE090
:10B43800202107221348F4F7ADFF2AE0B3F5E97F8E
:10B4480002D105200B2121E046F6897293421BD1D7
:10B45800002010211AE000BFF41E0020121E002058
:10B46800AC1E00209E1E0020951E0020F401002026
:10B47800083B0020CC1D0020E81D0020931E002062
:10B48800FB1E00200402002000200721094AFDF7C6
:10B498003DFB23689B7C102B08D92978064801318D
:10B4A800022207B0BDE8F04FFDF79EBB07B0BDE82C
:10B4B800F08F00BFF41E0020F50100202DE9F04FA9
:10B4C800794E8BB033689D6893F81290122D01D095
:10B4D8000B2D09D1754A122D92F80090A9F1300967
:10B4E8005FFA89F915D01DE04BF267739D4203D0CE
:10B4F80028339D4240F053836D482821F4F7C8FF54
:10B508008046002800F04E8301302821F4F7C0FF60
:10B5180048E39F7B37B9674BB846D879FEF7FEFBFF
:10B52800044615E00027B846FF20FEF7F7FB4BF26C
:10B5380058539D4204460BD14BF2376006F0A0FCED
:10B54800C0B2099020B15B4B9B790BB1FDF7EAFBC8
:10B558003368594D9A68122A1AD19B7BC3B12B784C
:10B5680013F0010F08D12046FFF7BAFC534B10B176
:10B5780001221A7000E018704E4B9B7943B12046A7
:10B58800FFF7AEFC20B14D4B1B780BB1FDF7CAFBA2
:10B598002978DFF844A111F0010100F087819AF8B9
:10B5A8000030DFF838B118460793FDF7B3FB079B67
:10B5B800002800F0B5804249002008704148424AFE
:10B5C80090F800C013609C45404940F0898033687A
:10B5D8009B8903F00F03032B1ED13D4BACF1300CBC
:10B5E80018784FF00A0E05903A480EFB0C00DDF86B
:10B5F80014E000EB0E0C0EF1010E5FFA8EFE7044A3
:10B608009CF8ADC090F8AD00C2F800C083F800E027
:10B61800002872D1187070E0082B2CD12C4BACF19B
:10B6280030001B7800EB800C0CEB030E294BDFF885
:10B63800A0C013F80E3008930BB98CF800309CF8B2
:10B6480000E000EB8000059070440EF1010E5FFAF7
:10B658008EFE8CF800E01F4BDDF814C01B5C0890D0
:10B668000CEB0E00DFF86CE013601EF80030002BC6
:10B6780043D1174811E0072B11D1BCF1300F10D17D
:10B688001348037823B14FF02B0EC2F800E001E015
:10B69800C2F800C0013303F0010303702DE0062B4C
:10B6A8002BD10B78013327E0041E0020E81D002071
:10B6B80004020020A21E0020E31E002033130020F5
:10B6C800175D0020E61D0020AC1E00209E1E0020F5
:10B6D800121E002010B40208CC1D0020E91D002015
:10B6E800DFF898E203709BF800304FF0010C8EF8F9
:10B6F80000C013B10B7863440B7040238BF8003003
:10B708000B784B4503D39B4B09F1FF301870087831
:10B718001168201806F0AAFB2B7843F004032B705D
:10B728009AF80030232B2FD1924B09F1FF311A7868
:10B738008A4229DA72B932684BF2677192688A4292
:10B7480008D028318A4205D02046079306F098FB96
:10B75800079BC8B118780130C0B21870201806F0DD
:10B768008FFB28B9834B20211878201806F07EFB20
:10B77800814B40221A702B78804A43F004032B70C7
:10B7880000238BF8003013709AF800302A2B10D160
:10B79800784B1A786AB1013A1A70774B40221A70BE
:10B7A8002B78764A43F004032B7000238BF8003083
:10B7B80013709AF80030432B1FD16E4B1878484508
:10B7C80005D220182021079306F050FB079B9BF811
:10B7D80000203AB91B7809F1FF32934202DA654A30
:10B7E800013313702B78644A43F004032B70002351
:10B7F8001370624A8BF8003013709BF8003013B155
:10B808005F4A013B13709BF80030012B0ED1594B56
:10B818001A784A4501D201321A70584A0023137027
:10B828002A7842F004022A708BF800302B7803F053
:10B838000402D2B2002A71D0524A6FF38203137005
:10B84800002111225048F4F7A5FD504A494B1178C0
:10B858001B78994288BF137011780F318B4202DD33
:10B868004A490F3B0B70117847481022611806F0BF
:10B8780018FB4548F4F7DEFF33684BF267719B68A5
:10B88800C2B28B4202D028318B4205D122B940483E
:10B89800F4F7D0FF421CD2B20F2A3FD83A482021F1
:10B8A8008018C2F11002F4F775FD37E0DFF8D8B060
:10B8B80011225846F4F76EFD33684BF267729B68A5
:10B8C800934202D02832934209D1214604222E48BD
:10B8D80006F0E7FA40463946FFF7DAFA1EE0214655
:10B8E8001022584606F0DDFA5846F4F7A3FF024640
:10B8F8002021C2F110025844F4F74CFD21464A4673
:10B90800244806F0CEFA244A1020937882F806904C
:10B9180043F0020393700146FDF7F8F89AF80030F7
:10B92800532B75D133689A684BF258539A4208D111
:10B93800204606F0A5FA20B14BF23760012106F047
:10B9480095FA3368DFF838A09B68122B40D120465F
:10B95800FFF7C6FA8346002830D0104BFF2219782B
:10B968000F4BF9B9009201911B78782001330293AB
:10B97800FB3A1FE09E1E0020175D0020121E0020CB
:10B98800E91D0020E31E0020801E0020951E0020D7
:10B99800811E00201B1E0020141E002033130020CF
:10B9A800931E00200021009201911B787A20013318
:10B9B800029304220B4606F0E1FA09E08AF8000037
:10B9C8007D492046FFF7B8FA7C4B83F800B0EFE0DA
:10B9D80020464946FDF7F0F8794B00201870336887
:10B9E8008AF800009B684AF6FE02934202D1009052
:10B9F800013005E04BF27A52934206D101230093BD
:10BA08000146024603460DF07FFD6E48FDF76CF8CF
:10BA1800FEF77AF92B7813F0010F17D033684BF241
:10BA280067729B68934202D02832934204D1404601
:10BA38003946FFF72DFA09E05F4B634A03F110011D
:10BA480053F8040B8B4242F8040BF9D133689A6817
:10BA5800122A1ED19B7BE3B12046FFF741FAC0B101
:10BA68002B7813F0010F14D1584B9A7922B9DA794F
:10BA7800574B1B789A420CD0564B1A780023303A11
:10BA880005E055492A20C91801330874DBB29342EE
:10BA9800F7DB326893680B2B01D0122B0AD14A4B83
:10BAA800991D13F8010B202802D10D3003F8010C61
:10BAB8008B42F6D192684BF258539A4214D1434BB9
:10BAC8009B798BB1099878B14FF0000909EB040014
:10BAD80006F0D6F918B1404B2A224B441A7409F1E2
:10BAE8000109B9F1100FF1D12B7813F0010F25D00E
:10BAF8003A4B1B7803F08003DBB2FBB133689A68DA
:10BB08004BF267739A422D4B03D04BF28F718A42E6
:10BB18000CD11B7833B9B8F1000F0FD05F3388F818
:10BB280001300BE057B15F22FA5407E0244A1B7832
:10BB3800127810339B1A284A5F21D154284CA378D5
:10BB480003F00203DBB2002B32D0FCF755FF20498B
:10BB5800034628B908786522E11DFCF76BFF12E05F
:10BB68003068B4F90430A27984680978122C01FB92
:10BB7800023105D1807B18B91449C97902FB01311A
:10BB8800184806F08EF933689B68122B10D10820EC
:10BB9800134A01460BB0BDE8F04FFCF7B7BF0027CA
:10BBA800B84600E0074609F1FF395FFA89F9BBE4B6
:10BBB8000BB0BDE8F08F00BF801E00209E1E002045
:10BBC800951E0020141E002004020020A21E002042
:10BBD800931E0020E81D0020F4010020083B0020EF
:10BBE800F41E0020FB1E002024282DE9F0411446F5
:10BBF80026D16B4B43F63C321B686A4D9B686A4EF4
:10BC0800934206D12B7813F0010F0ED024386749E0
:10BC180009E04BF28F7293420AD12B7813F0010F8F
:10BC280003D063490020FCF7B9FF2978490800E0F0
:10BC38002978301901310222FCF7D6FF0234AAE034
:10BC4800E72809D1574B5848197880180131032241
:10BC5800FCF7CAFF03349EE0A3282AD1514D2B7864
:10BC68003F2B15D810465349FCF798FF5148F4F775
:10BC7800E1FD2A2124184C48E4B2F4F709FC002815
:10BC880000F08A80297802220131FCF7ADFF83E0B9
:10BC98005901494DC918691801F582411046DF312B
:10BCA800FCF77CFF05F59240FE30F4F7C3FD24183D
:10BCB80071E0F22821D13B4F3B4D3978072605EB3F
:10BCC8000208B1FBF6F1404601310222FCF78CFF75
:10BCD80039782D23B1FBF6F688F80230F3009E1B65
:10BCE8008B1B364FDBB207EB83031988E21CA95282
:10BCF8009B78A818837006344DE025280BD1304B6B
:10BD080046F615629A8045229A719A78053842F06B
:10BD180002029A703CE05E280BD1294B46F6157258
:10BD28009A8045229A719A783E3842F002029A70B7
:10BD38002EE07C280BD1224B46F248129A80112221
:10BD48009A719A785C3842F002029A7020E0EC28E6
:10BD58000BD11B4B46F659729A8045229A719A78F4
:10BD6800CC3842F002029A7012E0A7280BD1144B8B
:10BD780046F679729A8045229A719A78873842F005
:10BD880002029A7004E0E02801D1541C03E018B1C3
:10BD9800054B18550134E4B22046BDE8F08100BFD8
:10BDA800041E0020931E0020F4010020845603087E
:10BDB80042560308FE5D030800140308794003088F
:10BDC800F41E002038B50A4B46F68A451B78002435
:10BDD80005FB030507E0074B22461978FFF704FF28
:10BDE800041B2D190446287808B11F2CF3D938BD37
:10BDF800E71D0020931E002070B5002543F620643F
:10BE0800204606F03DF8064604F1080006F038F82A
:10BE180016F0FF0F06D020F07F0010F0FF0F01D0C2
:10BE28000135ADB246F23F139C4201D00934E7E731
:10BE3800284670BD70B5B0F900500E4605EBC50533
:10BE480005F578552835284606F01AF8C3B213F0D8
:10BE5800800F064C08D03EB922882846013A03F0E4
:10BE68007F01228006F002F8208870BDE21D0020C4
:10BE7800454B2DE9F74F1B88444A044689461788E5
:10BE8800DFF80C8123B14FF0000A0AE09A4608E077
:10BE98000529FBD198F8003043F0040388F80030F6
:10BEA80070E098F8003013F0030F0BD013F0010F77
:10BEB80002D0B4F1FF3F05D103F00203DBB21BB19E
:10BEC800012C01D03F19BFB23BB2B3F1FF3F04D000
:10BED800B3F57A7F08BF002701E040F2E7370FFA91
:10BEE80087FB0BEBCB0303F5785303F12000019399
:10BEF80005F0C6FF10F0FF0F019B16D0B9F1050F32
:10BF080009D103F1280005F0BBFF20F07F0010F0F5
:10BF1800FF0FC6D022E0B9F1000F1FD003F12800AF
:10BF280005F0AEFF00F07F0618E00AF1010AB4F14F
:10BF3800FF3F1FFA8AFA04D198F8003043F0010352
:10BF480005E0012C05D198F8003043F0020388F889
:10BF58000030BAF57A7F0DD03D46A2E74E4505D0B0
:10BF6800B9F1000F02D0B9F1050F9AD1BAF1000F5B
:10BF780005D000E03D46054A2DB2156002E0034BAE
:10BF8800C3F800B0BDE8FE8FE21D0020AC1E002003
:10BF9800B01E00202DE9F041037890465A1ED2B217
:10BFA800792A9AB00F4600F2CA805E01654AF318F2
:10BFB8009B18654A46F68A461278457806FB02368B
:10BFC800E7213046F4F764FA0446F0B930467C219C
:10BFD800F4F75EFA0446C0B930462521F4F758FA5A
:10BFE800044690B930462421F4F752FA044660B961
:10BFF80030464021F4F74CFA044630B93046F9216E
:10C00800F4F746FA0446002878D0A41B0FB14F482D
:10C0180000E0404631462246A619F4F791FC304626
:10C02800E721F4F735FA30B128466946652246F625
:10C038005973FCF7FFFC30467C21F4F729FA50B11C
:10C04800691EC9B201EB011101F5C24168464831C8
:10C05800112205F026FF30462521F4F719FA38B1E8
:10C06800681EC0B26946652246F61563FCF7E2FC15
:10C078003046F921F4F70CFA38B1681EC0B26946A7
:10C08800652246F61573FCF7D5FC30464021F4F7D7
:10C09800FFF950B1691EC9B201EB011101F5EA417E
:10C0A8006846BB31112205F0FCFE30462421F4F726
:10C0B800EFF958B117B12548201801E008EB040042
:10C0C80029460222FCF790FD02340CE017B11F4804
:10C0D800201801E008EB04006946F4F74DFB6846B8
:10C0E800F4F7A8FB0419002F29D0194A93781419DA
:10C0F80043F0020393700023E37116E03046F4F72F
:10C1080099FB05461FB9404631462A4615E01028D6
:10C1180010DD2A460D483146F4F712FC0C4A937894
:10C12800551943F002039370EC7110200146FCF797
:10C13800EDFC04E0074831461022F4F701FC1AB080
:10C14800BDE8F081E3450308E71D0020FB1E002041
:10C15800F41E0020040200200C4B1A7812F0010390
:10C1680002D000200A4905E002F00200C0B218B16E
:10C1780008491846FCF712BD02F00402D2B20AB10F
:10C188000549F7E705480121FFF704BFB01E002065
:10C19800BC1B03089B1B0308DD1B0308E51E0020CE
:10C1A80070B5124D124C00201249FCF707FC2846C6
:10C1B800A1780222FCF718FDE81CE1780222FCF7BE
:10C1C80013FD05F1080021790222FCF70DFD05F1A8
:10C1D8000B0061790222FCF707FDA17905F10E0039
:10C1E8000222BDE87040FCF7FFBC00BFF40100204C
:10C1F800E51E002021B502082DE9F341544F554CA6
:10C208003B689D7C237813F0010F33D1022243F65B
:10C218001E610DF1060005F044FE4F4EBDF80630D4
:10C228004FF0FF3033602946FFF722FE237843F0B2
:10C2380001032370494B1B7813F0030F18D1B6F98B
:10C248000010474801EBC10101F57851203109225E
:10C2580005F027FE434B1B883BB1434B304619780A
:10C26800C1F34001FFF7E6FD10B90020FAF790F896
:10C27800FFF796FF3D4E3378552B0DD1DFF8DC8064
:10C288003B48FCF731FC98F800304FF0FF306FF373
:10C29800410388F800300DE0442B2FD1DFF8BC8033
:10C2A8003348FCF721FC98F8003001206FF30003B5
:10C2B80088F800302946FFF7DBFD98F8003013F0C6
:10C2C800030F19D1244D2648B5F90010092201EBB6
:10C2D800C10101F57851203105F0E3FD214B1B88A0
:10C2E8003BB1214B28461978C1F34001FFF7A2FD65
:10C2F80010B90020FAF74CF8FFF752FFFFF72CFFB0
:10C308003378232B22D1154B194E1A7802F0FC02F0
:10C318006FF382021A70FCF705FDB3786FF34103DF
:10C32800B370144B1D7835B9FCF734FB3046FCF775
:10C33800DBFB3D600AE02278013DEDB242F00602E7
:10C3480022701D700C4B53F825303B60BDE8FC8112
:10C35800041E0020E31E0020AC1E0020B01E00209A
:10C36800E51E0020E21D00205B680020CC1D002097
:10C37800F41E0020C31E0020D01E00202DE9F0412D
:10C388001646104A0F4653780E21C3F342034B4317
:10C39800117803F50A434C330B4D01F007010446AD
:10C3A80003EB4101022205F07CFDE8192178022205
:10C3B800FCF71AFC6178A8190222BDE8F041FCF7E5
:10C3C80013BC00BF991E0020F4010020044B022278
:10C3D8005978044BC1F3420118180131FCF704BC29
:10C3E800991E0020F401002010B5074B074C1B785C
:10C3F800074A03F0070304EB83031C88111814523F
:10C408009B788B7010BD00BF991E002079400308EF
:10C41800F4010020084B1B789B0902D0012B06D1A0
:10C4280002E01020054904E01020054901E0054913
:10C438001020FCF7B3BB00BF991E00205E2803083C
:10C448007F280308A02803082DE9F041DFF8688059
:10C458000F4698F80010174DC1F38201044616469E
:10C4680005F1080001310222FCF7BEFB98F8001024
:10C47800042201F01C0101F51E413431204605F06B
:10C4880010FDE81921780222FCF7AEFBF81C2818E9
:10C4980061780222FCF7A8FBA819A1780222FCF710
:10C4A800A3FBF01CE17828180222BDE8F041FCF754
:10C4B8009BBB00BFF4010020E51D0020064B1B7844
:10C4C80003F08003DBB233B1435C04482021C01879
:10C4D8000222F3F75FBF7047083B0020F4010020F9
:10C4E8002DE9F743654D664C2B6821789B6802223D
:10C4F80003EB41010DF1060005F0D3FC2B68A946BA
:10C508009A6843F6F4239A4208D100205D49FCF763
:10C5180045FBBDF806804FF4B46303E0BDF8068020
:10C528004FF46163B8FBF3F103FB11883C221FFA57
:10C5380088F8B8FBF2F302FB1388CFB2DEB202220E
:10C5480051483946FCF750FB5FFA88F802224F48F9
:10C558003146FCF749FB02224D484146FCF744FBB3
:10C568004C4B1B7813F0010F6ED04B4B4B4D18788A
:10C57800232804D12B78012B62D8013305E02A281F
:10C5880005D12B78002B5BD0013B2B7058E0A0F134
:10C598003003DBB2092B01D943284BD12B7873B96F
:10C5A800D9F8003039B29A6843F6F4239A4201D197
:10C5B8000A2200E01122FDF7C7FBC7B216E0012BE3
:10C5C8000ED1D9F8003031B29A6843F6F4239A4272
:10C5D80001D1172200E03B22FDF7B6FBC6B205E009
:10C5E80041463B22FDF7B0FB5FFA80F8D9F80030EE
:10C5F8009A6843F6F4239A4209D13C235E434FF4E8
:10C60800B46303FB0767B844ADF8068006E0384614
:10C618003146424610F02DFAADF80600D9F8003040
:10C6280020789B680DF1060103EB4000022205F01B
:10C6380032FC05E0532803D100232B70FDF764FB7F
:10C6480017482978FFF73AFFD9F800309A6843F677
:10C65800F4239A4210D02078124965220023FCF76F
:10C66800E9F905200B21104AFCF750FA21780F4808
:10C6780001310222FCF7B8FABDE8FE83041E00204F
:10C68800931E0020835A0308040200200A02002097
:10C6980012020020E31E0020CC1D00209E1E002058
:10C6A80032B50208FB1E0020F41E0020F501002010
:10C6B80073B5994B994D1A7812F0010F05D12A7864
:10C6C80012F0380204BF2A706A701A78924E42F04B
:10C6D80001021A702B78914C13F038023ED1904920
:10C6E8000978552904D113F0070F2FD0DA1D0AE075
:10C6F80044290CD103F0070201323D3992FBF1F1D4
:10C70800C800411A521A62F3020323701EE053292B
:10C718000AD1C3F3C201013161F3C5032370637801
:10C7280062F34303637011E023290FD1FCF7FAFA8F
:10C7380033787C4A43F0060333701378013BDBB24D
:10C748001370794A52F82320784B1A6000207849F0
:10C75800FCF724FA1C20FFF747FEDBE0082A2CD15F
:10C7680074490020FCF71AFA0620FFF72FFE0C2068
:10C77800FFF73AFE1521182201A8FFF7FFFD684BC5
:10C788001B78552B06D1637803F0FE03C3F34202EE
:10C79800013A07E0442B09D1637803F0FE03C3F3A1
:10C7A8004202013262F343036370B3E0532B28D093
:10C7B800232B40F0AF802378A6E0102A51D15D49A1
:10C7C8000020FCF7EBF90620FFF700FE0C20FFF72E
:10C7D8000BFE1521182201A8FFF7D0FD61785648F5
:10C7E80001F00101FFF76AFE4D4B1878232801D0AC
:10C7F8002A2804D16378DA4362F30003D4E7532884
:10C8080004D12378C3F3C202013280E0A0F13003DF
:10C81800DBB2092B01D943287CD16B7802AA03F03B
:10C8280001033B21D41883F001024B43172606FB72
:10C83800023214F8041CFDF787FA04F8040C6B782C
:10C848000E22C3F342035343287803F50A434C33BB
:10C8580000F0070003EB400001A90C3A05F01BFBB0
:10C8680058E0182A4DD133490020FCF797F90620E3
:10C87800FFF7ACFD0C20FFF7B7FDFFF7CBFD284B0A
:10C888001B78552B07D1237813F0C00F42D0C3F380
:10C898008112013A06E0442B07D123789A09012A2C
:10C8A80038DC013262F3871333E0232B04D1237879
:10C8B800C3F3C202023A2AE0532B2BD1FCF732FA17
:10C8C80033781E4A43F006033370164B164819781E
:10C8D80040F82120013119702378C3F3C2010131D6
:10C8E80061F3C503C3F381112370104B11B1012902
:10C8F80004D101E01C3202E0114A00E0114A1A603A
:10C9080008E0114A00211170C3F3C202013A62F330
:10C91800C50323707CBD00BFE31E0020991E0020C4
:10C92800CC1D0020C31E0020D01E0020041E0020A5
:10C938001C2803083D28030835B5020838B5020845
:10C9480070B502088CB502089E1E002073B5494BCD
:10C95800494D1A7812F0010F04D12A7812F0030217
:10C9680008BF2A701A78434E42F001021A702B78D9
:10C97800414C13F003022ED1404A1278552A03D1B4
:10C98800C3F38202013A04E0442A06D1C3F38202C7
:10C99800013262F38403237017E0532A03D15A1C2F
:10C9A80062F30103F7E7232A0FD1FCF7BBF93378C9
:10C9B800334A43F0060333701378013BDBB213703C
:10C9C800304A52F82320304B1A6001A810211B224C
:10C9D800FFF73AFD4CE0012A4AD101A810211A328A
:10C9E800FFF732FD254B1878232804D12378C3F3A9
:10C9F8004112013205E02A2807D12378C3F34112F6
:10CA0800013A62F3461323702CE0532804D12378AB
:10CA1800DA1C62F30103F6E7A0F13003DBB2092B5D
:10CA280001D943281ED12B7802AAC3F34113D41885
:10CA38000C215A1C03F001034B4302F001021F268C
:10CA480014F8041C06FB0232FDF77EF904F8040C06
:10CA5800287801A900F01C0000F51E40343004229B
:10CA680005F019FA29780948C1F34111FFF726FDA5
:10CA78007CBD00BFE31E0020E51D0020CC1D00206A
:10CA8800C31E0020D01E0020041E0020A8B50208E6
:10CA9800064B1B7803F08003DBB233B1435C0448D8
:10CAA8002021C0180322F3F775BC7047083B00200B
:10CAB800F40100204328F8B504460D46174606D170
:10CAC800104B00261A786FF3C3021A7000E00E4666
:10CAD8002046FCF71FF990B10A4B303C1A780A2619
:10CAE80002F00801C9B2002918BF002506FB054657
:10CAF8006FF3C30236B21A70BE42A8BF3E4630B2C8
:10CB0800F8BD00BFE31E00202DE9F3416E4F6F4EC4
:10CB18003B7843F001033B70347844B94BF2AF5093
:10CB280005F0AEF96A4B6B491860204617E0012CF6
:10CB380002D10020684912E0022C02D10020674986
:10CB48000DE0032C02D10020654908E0042C02D135
:10CB58000020644903E0052C03D163490020FCF759
:10CB68001DF83178D9B9614B1B78312B01D10131CE
:10CB780001E0302B05D1564B4BF2AF50196005F050
:10CB880075F95B4B1A785B4B02F08002D2B20AB19E
:10CB9800202202E04E4A12683032DA776EE001292C
:10CBA8000BD002290CD003290DD004290ED04BF24A
:10CBB800AB55052918BF00250AE04BF29B5507E045
:10CBC8004BF29F5504E04BF2A35501E04BF2A755F9
:10CBD8002946042201A805F064F9474B474A03F1A6
:10CBE800100153F8040B8B4242F8040BF9D10322CD
:10CBF80043489DF80410FBF7F7FF032241489DF8CE
:10CC08000510FBF7F1FF03223F489DF80610FBF7DC
:10CC1800EBFF3E4803229DF80710FBF7E5FF334B77
:10CC28003B4C1878232804D12378022B22D80133CF
:10CC380004E02A2804D12378E3B1013B237019E0EA
:10CC4800A0F13003DBB2092B01D9432812D194F8A3
:10CC5800008002AA904418F8041CFF22FFF72AFF5C
:10CC680008F8040C207802AA131813F8041C2818D2
:10CC780005F0FCF827482178FFF70AFF1B4B1B78C3
:10CC8800532B1FD1224B00221A7033780133DBB2A9
:10CC9800062B337004D0012B14D10D4B1B688BB1BC
:10CCA800FDF732F8002333703B781B4A43F0060344
:10CCB8003B701378013BDBB21370184A52F82320FB
:10CCC800174B1A60BDE8FC81E31E0020931E00206C
:10CCD800AC1E002009740308327503085375030855
:10CCE8007475030895750308B6750308CC1D0020F4
:10CCF800083B0020F401002068A303080402002078
:10CD080005020020090200200D0200201102002067
:10CD18009E1E0020ACB50208C31E0020D01E0020B5
:10CD2800041E002070B5174C0D460646002120460B
:10CD38004FF4C172F3F72EFBFF2D0AD1B10001F5B4
:10CD4800DC4120461531042205F0ABF823789BB965
:10CD580070BDFE2D01D1173E02E0FD2D02D1013636
:10CD6800267009E0B60006F5DC401530401905F0DC
:10CD780087F8C0B2207020B10248BDE8704019F0B1
:10CD88007DB970BD082100202DE9F04119F0A8F9FE
:10CD980060B110208F49FBF701FF8F4B1B78432BA5
:10CDA80040F0EE81BDE8F04119F0BCB919F0AAF9DC
:10CDB800002826D0894C23786BB110208849FBF7CE
:10CDC800EDFE88482D211030F3F762FB002800F0B3
:10CDD800D781217810E010208349FBF7DFFE8148D6
:10CDE8002D211030F3F754FB0446002800F0C881C9
:10CDF80019F0A0F9014620468222BDE8F041FBF770
:10CE0800F3BE7A4C43F6CC2223689B68934250D0F9
:10CE1800774E744D307803EB800005F031F803222B
:10CE280001467448FBF7E0FE2368986846F6797374
:10CE380098422BD0203B984228D03378013000EB21
:10CE4800830005F01DF80322014605F11500FBF7E4
:10CE5800CBFE236830789B68023303EB800005F033
:10CE68000FF80322014605F11900FBF7BDFE236800
:10CE780030789B68033303EB800005F001F8032248
:10CE8800014605F11D00FBF7AFFE0EE02D21032240
:10CE98005948F3F77FFA2D2103225848F3F77AFA15
:10CEA80057482D210322F3F775FA20232B772B7689
:10CEB8002B75544B1B7813F0010F00F0BD802368CD
:10CEC80043F6CC229B68444D934261D04E4E484F66
:10CED80032783878D31803EB800004F0D1FF4B4B3D
:10CEE8000146186028789846A0F13002D2B2092A83
:10CEF80001D943280FD109B2BA22FCF725FF2368CC
:10CF080032789B680146C8F800003878D31803EBDC
:10CF1800800004F0ABFF2B782A2B04D1337813B1AF
:10CF2800394A013B13702B78232B0ED13378022B0F
:10CF38000BD8226846F6597192688A4205D020318A
:10CF48008A4202D0304A013313702B78552B01D016
:10CF5800442B0FD1236831789B68A3F5DC43B3F1E8
:10CF6800150248BFA3F112023B7803EBA202D0B22C
:10CF7800FFF7D8FE264B1B7803F08003DBB23BB1EA
:10CF88003278184B03EB820320225A749A74DA74AD
:10CF98002B78532B06D023689A6843F6CC239A4201
:10CFA80040F0EE80FBF7BEFE236846F615629B68EC
:10CFB800934203D10E4B0220197806E046F67972A7
:10CFC800934227D10A4B002019780131BDE8F0417E
:10CFD8000CF06EBA385D0308CC1D0020F81500204F
:10CFE8000F5C0308F4010020595D0308041E0020AB
:10CFF800931E002005020020090200200D020020D7
:10D0080011020020E31E00209E1E0020AC1E0020FE
:10D01800083B002046F65972934204D1594B01202F
:10D0280019780918D2E746F61572934240F0A8809D
:10D03800544B03201978C8E723684AF6FE029B6818
:10D0480093423ED14F4E10204F49FBF7A7FD317850
:10D058004E4D01EB011101F52841FE311022284601
:10D0680004F01FFF2B4605F110012A461078474FA0
:10D0780078B94749FBF792FD3846E721F3F708FAF4
:10D0880078B13178401B381801310322FBF7ACFD29
:10D0980007E013F8010B10B9203003F8010C8B429C
:10D0A800E4D13C4D2B782A2B03D13078FD21FFF7B2
:10D0B80039FE2B78432B63D1307823680130C0B216
:10D0C80059E043F6CC229342324E1AD0102032490E
:10D0D800FBF764FD33782A2B52D1304B1B689B68D1
:10D0E800A3F5DC43B3F1150248BFA3F11202254BA7
:10D0F800FF211B7803EBA202D0B2BDE8F041FFF795
:10D1080011BE33781F4D552B04D12B78142B01D128
:10D11800033B2B703378442B05D12B78122B02D18B
:10D12800184B15221A702B78DFF874805901C9182A
:10D13800414401F5944100201F31FBF72FFD08F50C
:10D148009241102017312F78FBF728FD3378112FE3
:10D158008CBF032700272A2B05D12878FE21C01B66
:10D16800C0B2FFF7DFFD3378432B09D12B78173B8B
:10D17800DF1B2368F8B2997CBDE8F04118F098BF2E
:10D18800BDE8F081931E0020175D0308F40100201C
:10D19800273E0308CC1D0020D55C0308041E002090
:10D1A8000014030810B50E4B1B78452B17D10D4BF7
:10D1B8001A7842F006021A700B4A1378032B0ED81D
:10D1C8000A490B4C086844F823000133137083683C
:10D1D8000B60FBF7EBFBBDE81040FBF7A3BD10BDF0
:10D1E800CC1D0020E31E0020C31E0020041E0020CA
:10D1F800D01E002010B50C4B04462146D8790FF0FC
:10D20800FCFB60B1204655210FF056FA48B1204684
:10D218000FF0E8FAD0F1010038BF002010BD02205D
:10D2280010BD022010BD00BFA21E002008B50FF0DF
:10D23800D3FBC0B208BD00002DE9F047634B644C36
:10D248001A78994612F0010F624D65D02078FFF7E1
:10D25800D1FF614A2B181178604F93F8A031604EC6
:10D2680044293870336090460AD12D2B08D038B93C
:10D2780095F8A11101233B7031602078FFF7D6FFA4
:10D2880098F80030552B10D133682D2B0DD03B78F2
:10D298005BB1013B514ADBB21370EB1893F8A01154
:10D2A8004F4B20781960FFF7C1FF98F80030232B07
:10D2B80019D14C4B20781B689B7C013B984212DAB1
:10D2C800434B0130C0B21870FFF794FF387028182C
:10D2D80090F8A0313360444B9B7803F00203DBB233
:10D2E8000BB1FBF757FB98F800302A2B14D12078A4
:10D2F80090B1374B0138C0B21870FFF77BFF387018
:10D30800281890F8A0313360374B9B7803F002035C
:10D31800DBB20BB1FBF73EFB344EFCF7F5FC237890
:10D3280032789A4288BF337032780F32934202DDE6
:10D338002E4A0F3B1370DFF8C48000273078381866
:10D34800C0B2FFF757FF281890F8A0310137102F07
:10D3580008F8013F07D0254B1A78224BBA181B68EA
:10D368009B7C9A42EADB99F8003013F0010F13D046
:10D378001F4B1A781F4B02F08002D2B22AB12278D2
:10D3880031781032521A5F2105E022783178103254
:10D39800521A134909689954134DAB7803F00203E4
:10D3A800DBB25BB12078E91D652246F61573FBF701
:10D3B80041FB05200B212A46FBF7A8FB21780E48E4
:10D3C80001310222BDE8F047FBF70EBCE31E002046
:10D3D8009E1E002010B40208CC1D0020E41D002071
:10D3E800AC1E0020041E0020F41E0020951E002004
:10D3F800083B0020F4010020F50100200302002072
:10D408002DE9F041002480460D46164623460127A3
:10D4180017FA04F298F80010E0B2914206D146F6E5
:10D42800597329463246FBF705FB3B460134082C65
:10D43800EDD1083C0A4AE0B2A218917898F8002089
:10D448008A4207D132B146F6797329463246FBF74C
:10D45800F1FA01230134042CECD11846BDE8F0811F
:10D46800A21E00202DE9F041074610460D4614463D
:10D47800F3F7E0F9C3B28046B3B1AB4214D80B4E10
:10D4880020212A46F019F2F785FF2046F3F7D2F952
:10D49800C8EB05056D08EDB2EF1902462146F019F3
:10D4A800BDE8F041F2F7CEBEBDE8F081F4010020FE
:10D4B800312200230178194111F0010F02D00449EB
:10D4C800C9180A7501330132082BD2B2F2D170475C
:10D4D800F40100202DE9F04F87B09DF840408146C7
:10D4E800072C0D4605929A4637D1073C27462B78DC
:10D4F800234113F0010F2CD0012623B24FF000086E
:10D50800029351203146324633460096CDF80480C6
:10D5180004F034FD1B204146A2194346CDF8008093
:10D52800F5F7EEF837B9112039463A4633460097F1
:10D53800F5F7E6F8534B204613F8242001276FF33C
:10D54800000203F824201199F5F79EFF2046F6F70C
:10D55800A5F90134082CCAD10DE2012C03780CD1AD
:10D568000BB90B7823B3FF2300930021464B01919D
:10D578001B780C200133029316E0022C09D10BB959
:10D588000B78ABB10021FF23009301910291342065
:10D598000AE0062C0CD10BB90B784BB10021FF2304
:10D5A800009301910291652004220B4604F0E6FCE9
:10D5B800BAF1010F99F800302BD13BB1334B002061
:10D5C800D979024653460090F5F79AF82B783BB183
:10D5D8002E4B0120D979002203460092F5F790F8E6
:10D5E8000020F5F707FF99F80030002B5BD0284B97
:10D5F8001978002957D1274B5B78002B53D0FF238C
:10D6080000933A2001220B460191029104F0B6FCE6
:10D6180049E063B1052C4FF0000102D100910F20C1
:10D6280001E000910B200A460123F5F769F82B78F1
:10D6380083B1052C4FF0000106D110200A460123C2
:10D648000091F5F75DF812E00C200A4601230091DD
:10D65800F5F756F8022C25D0032C01D10E4B02E029
:10D66800042C02D10D4B1F781DE0052C01D10C4B69
:10D67800F9E7012C01D1044BF5E7062C0CBFFF2775
:10D68800002710E0411A0020221B0020A21E0020C3
:10D698002C1A002033130020BC200020EF5B002050
:10D6A800973F0020FF2799F80030002B00F0B58045
:10D6B800934B944E1A78984602F02002D2B262B187
:10D6C800317811F0010108D1FF23009328200122AD
:10D6D8000B460191029104F051FC98F8003003F0D8
:10D6E8001003DBB26BB1317801F00201C9B241B964
:10D6F800FF230093292001220B460191029104F097
:10D708003DFC98F8033013F0010F0DD0317801F08B
:10D718000401C9B241B9FF2300932A2001220B4614
:10D728000191029104F02AFC98F8033003F00203F7
:10D73800DBB26BB1317801F00801C9B241B9FF23FE
:10D7480000932B2001220B460191029104F016FC54
:10D7580098F8033003F00403DBB26BB1317801F0C1
:10D768001001C9B241B9FF2300932C2001220B46B6
:10D778000191029104F002FC98F8033003F00803C9
:10D78800DBB26BB1317801F02001C9B241B9FF2396
:10D7980000932D2001220B460191029104F0EEFB2B
:10D7A80011F00EFF68B1317801F04001C9B241B9FA
:10D7B800FF230093492001220B460191029104F0B6
:10D7C800DDFB98F8033003F04003DBB26BB131782E
:10D7D80001F08001C9B241B9FF2300934E20012214
:10D7E8000B460191029104F0C9FB767816F0010608
:10D7F80013D14548314617F092FE58B1FF230093E4
:10D80800731C00211BB20293752001220B46019163
:10D8180004F0B4FB0136702EEBD1119B3B4A19780A
:10D828003B4B51B199F8001011702A781A702B7877
:10D838000BB1542005E0522003E011702A785320E0
:10D848001A7004F071FF119B00261A78314B1A7078
:10D8580099F80030334113F0010F2DD03146059867
:10D8680017F05DFE0122014628B933B201900092FB
:10D878000293104605E0002133B200920191029311
:10D8880024200B4604F07AFBBAF1010F05D1224B94
:10D898008020DA790521013208E0022C07F1010223
:10D8A80002D18020072101E0802006213346F6F7C7
:10D8B80053FB3046F5F7C6FF2B78334113F0010FC1
:10D8C80055D000214FF0010B33B2029302205A4683
:10D8D8000B46CDF800B0019104F050FBDA45DFF8B3
:10D8E8003C801DD118F8263013EA0B0332D10A4ABE
:10D8F8000520D1790093594406EB0B0228E000BFBC
:10D90800083B0020141C00201C1A00208D1A00203F
:10D918008E1A0020321C0020A21E0020411A00206E
:10D9280018F8263013F0010314D1022C0CD1134B34
:10D938001B7803F02403042B04BF114B83F800B0B9
:10D9480000230093072001E000930620791C721C35
:10D95800F4F7D6FE11993046F5F796FD3046F5F7FF
:10D968009DFF18F826306FF3000308F826300136BB
:10D97800082E7FF46DAF07B0BDE8F08F3C1C002087
:10D988002C1300202DE9F04180460E46174646F636
:10D998003F1500243846214617F0C1FD88B12946B5
:10D9A80008220B4804F07DFA0948414617F064FD47
:10D9B800074817F087FD20B90123A34032781343A5
:10D9C800337001340835082CE4D1BDE8F08100BF7C
:10D9D8002A1C00202DE9F04387B08046894604A818
:10D9E80047F26931082204F05CFA002440462146D7
:10D9F800E7B217F094FD002843D03846F4F7B8FB97
:10DA08000025661C0246314611202B460095F4F786
:10DA180077FE012321462A460420FF080095F4F7E3
:10DA28006FFE4BF25F70381804F02AFA04F007030F
:10DA3800C1B2194111F001014FF002024FF0010388
:10DA48000AD00092019336B27720294692182B46C5
:10DA5800029604F093FA14E00092019336B2232060
:10DA680004220B46029604F089FAB9F1000F08D097
:10DA780004A8214617F053FD18B10548214617F0B0
:10DA880038FD0134402CB1D107B0BDE8F08300BFA8
:10DA98006A1A00202DE9F74F9846137805460C4678
:10DAA80017469DF830909DF834B09DF83800DFF89F
:10DAB800C8A073B12A4A51786FF3820151703B783C
:10DAC80000EA03033B7021789AF800208A18D31AD9
:10DAD8002B70237883B123482146F5F78BFE224922
:10DAE800204817F0C9FC1F480121FFF773FF1D48A4
:10DAF80041462246FFF746FF1C4B00261E70297838
:10DB080043F6FB2004F0B2F9494646F64D0004F00E
:10DB1800ADF9204639464A46F5F722FC144B4246F1
:10DB28009E7039464B462046CDF800B00195FFF768
:10DB3800D1FC2846F8F764FC2B780E480E498AF881
:10DB48000030F5F757FE12F089FD88F800603E7046
:10DB580026702E7003B0BDE8F04F04F0EFBC00BF94
:10DB6800933F0020331C0020851A0020E01E00206F
:10DB780033130020161C00202C1A002010B50B4B64
:10DB88000B4C024603CB206061600A48114617F02F
:10DB980094FC2146074817F06FFC064817F092FCE2
:10DBA800D0F1010038BF002010BD00BFC02E0020FA
:10DBB800201C00202A1C002010B50A4C637C4BB1A5
:10DBC80000200949FAF7EAFF084B1B78432B01D1DB
:10DBD800433B6374607C20B90549BDE81040FAF7FF
:10DBE800DDBF10BDCE1D0020693E0308CC1D0020FE
:10DBF800483E0308034B1A7801321A700123037058
:10DC0800704700BFE01E002010B50C48FAF76CFF03
:10DC18000B4A002414700B4A0B4B14700B4ADC702F
:10DC280014700B4A9C7014700A4A1C7114700A4ACA
:10DC38001470FBF777F8094B1C6010BDF41E002028
:10DC4800A21E0020CD1D002033130020E41E00205A
:10DC5800F11E0020081E0020E01E0020041E0020E7
:10DC68002DE9F04F984B994E93F800903368DFF800
:10DC7800AC829C7C964BF0221A7098F800308BB0DE
:10DC88000D2B354647463FD1924B93F803C0BCF164
:10DC9800010F04D9ED3A5A7100208F492FE01AD1AB
:10DCA8000024DC708D4A8E4B8E498F488F4D04704E
:10DCB8001C7014700C70CDF800C001942D7802957A
:10DCC800FFF7E8FEFBF72EF8894834600BB0BDE893
:10DCD800F04FFAF709BF87488249F5F78BFD864B65
:10DCE800864A03CB864B10601B785160532B5FD15B
:10DCF80098F800308349013388F8003000200BB0D1
:10DD0800BDE8F04FFAF74ABF092B0FD17C4B1B78BF
:10DD1800532B3DD17C4B00221A700D2388F800301C
:10DD28007A4B1A7842F006021A7089E20E2B37D124
:10DD3800734B1B78532B2BD175496E4817F09CFBFE
:10DD48006C48FFF71BFF044640B198F800300522E5
:10DD5800013B88F800305F4BDA7071E2082246F622
:10DD68004E01664804F09DF864496A4817F0A5FB1F
:10DD7800012300935D4B01941B785B48029359493A
:10DD8800564A574BFFF786FEFAF7CCFF346057E246
:10DD9800232B40F055820BB0BDE8F04FFFF734BF9E
:10DDA80033B95D4B1A781AB901321A7012F056FC61
:10DDB800631E48BFA31DDB10013303FB09F91FFADB
:10DDC80089F909F5D046A9F59049A9F1A1094F4B60
:10DDD800CDF81C901A784E3612F0010F4A4C00F01C
:10DDE8002081474B1A789946432A40F0C9803B78EE
:10DDF8000D2B40F0C5803F48217817F090FB002894
:10DE080000F0BE803D48217817F089FB002840F0DB
:10DE1800B780079920780FFA81FB0BEBD00004F04C
:10DE28002FF823784FF0010A03F007020AFA02FAE2
:10DE3800DFF8EC805FFA8AFA10EA0A0FC8F80000E7
:10DE480027D0244B5B78002B40F09A80274BD87959
:10DE5800F8F734FA002800F09380D8F80010CAF1D7
:10DE6800FF0A20780AEA0101C8F800100BEBD0007D
:10DE780003F0FCFF20780FFA86FB0BEBD00003F0D1
:10DE8800FFFF00EA0A012078C8F800100BEBD00069
:10DE980061E032B202EBD300059203F0F1FF10EA21
:10DEA8000A0FC8F800003DD140EA0A01059B207816
:10DEB800C8F8001003EBD00003F0D8FF217815480C
:10DEC80017F017FB5CE000BF931E0020041E002023
:10DED800EF1E0020331300200E3F0308E41E00202D
:10DEE800CD1D0020F11E0020081E0020A21E0020CB
:10DEF800F41E0020331C0020C02E0020141A00201D
:10DF0800CC1D0020D43F03089E1E0020E31E0020E5
:10DF18007A1A0020851A002078140020E01E0020BC
:10DF2800AC1E0020924B5B7823B9924BD879F8F756
:10DF3800C5F9B8B92078DDF814C0CAF1FF0A0CEBAE
:10DF4800D00003F09DFF8C4A00EA0A01059B207867
:10DF5800116003EBD00003F089FF2178874817F0A0
:10DF6800D3FA0DE020780BEBD00003F089FF40EAEC
:10DF78000A012078C8F800100BEBD00003F076FFF8
:10DF880099F80030232B10D12A682378927C013A23
:10DF980093420ADA7A4A013313707A4B9B7803F07A
:10DFA8000203DBB20BB1FAF7F5FC99F800302A2B23
:10DFB8000CD1237853B1724A013B1370714B9B7893
:10DFC80003F00203DBB20BB1FAF7E4FC99F8003076
:10DFD800552B12D129682278897C694B08398A42E5
:10DFE80001DA083200E000221A70664B9B7803F0D1
:10DFF8000203DBB20BB1FAF7CDFC99F80030442BE1
:10E008000FD122785E4B072A9CBF2A68927C083A77
:10E018001A705C4B9B7803F00203DBB20BB1FAF782
:10E02800B9FCFBF771FE584A237811789246994259
:10E0380088BF137012780F32934202DD524A0F3BA9
:10E0480013702B684FF0000B93F81280CDF818B0BE
:10E05800B8F10F0F9ABFC8F120085FFA88F84FF09F
:10E06800100839784FFA8BF30D2905D19AF800205A
:10E078009B18DB10454A04E09AF800209B18444A94
:10E08800DB10D35C9AF8002005934FFA8BF39A18AB
:10E098000D2902F007094FEAE20202D13D49895CE5
:10E0A8000691DDF81CC004930FFA8CF0101803F0E9
:10E0B800E7FEC0B2049B08909AF8000032B2181824
:10E0C80002EBE00003F0DCFE39789AF80020049BAC
:10E0D800C0B209919A1846E0059BDDF824C043FABE
:10E0E80009F12D4B01F0010100290CBFA521DB210D
:10E0F800BCF10D0F03F8081014D128494FEAE20CBF
:10E1080011F80C1041FA09F111F0010F08D0DDF8EF
:10E1180018C04CFA09F111F0010F03D0582110E092
:10E128002D210EE0DDF820C04CFA09F111F0010FA5
:10E1380001D0502105E040FA09F111F0010F02D099
:10E14800542103F8081009F101095FFA89F90BF164
:10E15800010B08F101080132B9F1080F5FFA8BFBD6
:10E168005FFA88F81CD0B8F1200FB5D125E000BFC0
:10E1780033130020A21E0020AC1E0020851A0020A8
:10E188009E1E0020F41E0020951E00207A1A0020F2
:10E19800DA1A0020141A0020F4010020331C002091
:10E1A800B8F1200F09D09AF800304FFA8BF2D21844
:10E1B8002B689B7C9A42FFF654AF23490B7813F0E7
:10E1C800010F17D02B68214A9B7C12780F2B02F085
:10E1D800800298BFC3F11003D2B294BFDBB2002310
:10E1E80042B122789AF800101032521A1849CB1806
:10E1F8005F219954174EB37803F00203DBB293B151
:10E20800F11D652246F615632078FAF713FC2B6892
:10E218009B7C102B02D905200B2101E0002007214F
:10E228003246FAF773FC2B689B7C102B08D92178AF
:10E238000948013102220BB0BDE8F04FFAF7D4BC0F
:10E248000BB0BDE8F08F00BFE31E0020083B0020A4
:10E25800F4010020F41E0020F501002088234B4320
:10E26800054A03EBD003D35C00F0070053FA00F033
:10E2780000F00100704700BF4C0D002070B5044647
:10E288001646157839B912E00135EDB2284621460F
:10E29800FFF7E4FF48B9202DF6D970BD013DEDB276
:10E2A80028462146FFF7DAFF08B1356070BD002D1A
:10E2B800F4D170BD064B38211B78032201FB0031D5
:10E2C800044844230370C9B2173BC370FAF78CBCE7
:10E2D8009E1E0020F4010020012802D0022806D149
:10E2E80002E01D20044904E01D20044901E004491E
:10E2F8001D20FAF753BC00BFB5370308943703084D
:10E30800D6370308037809680F4A03EB031040184F
:10E3180002EBC00050F8240C0C4988420FD1882128
:10E3280001FB03239A68A0F59C63063B9A4208D038
:10E33800A0F598600538101A18BF01207047002012
:10E3480070470020704700BF4C0D0020733703084A
:10E3580003780A6803EB0313D318084A053B02EB5A
:10E36800C3035968064A914205D1187A09288CBF17
:10E378000020012070470020704700BF4C0D00208E
:10E38800733703082DE9F04F984B994FF0221A7014
:10E398003B6889B09C6847F67313E11A4C4244EB1A
:10E3A8000104CC3A6243934B9D5C03EB0208C5F32E
:10E3B8000005EEB23A46002E2CD130468E49FAF7C7
:10E3C800EDFB8E4B1B78232B41F0388298F80130F7
:10E3D80066F3041388F80130FAF7A4FC884B1A781E
:10E3E80042F006021A70874A1378013BDBB21370B9
:10E3F800854A52F823303B60844B1D70844B1D7056
:10E40800844B1D70844B1E60844B1D70844B1D70A3
:10E4180001F014BA814D95F80090B9F1000F0CD0B5
:10E428004FF43661614309F1FF30342303FB0013D5
:10E438007C49CB181B798DF81F307B4B1E787EB139
:10E448007A4E2046317811F09FFF002840F05C8416
:10E4580075493070087007460646804600F05BBC78
:10E468006D490B688B46A3F11200032809D9A3F163
:10E478001601032909D9A3F11A01032909D9374635
:10E4880005E037464FF0010805E037460126B84653
:10E4980001E00127B04659490978532940F0D58150
:10E4A800B9F1000F3AD1722262436149885C10F0D9
:10E4B800020F0AD0002B41F0C181013363F38300BE
:10E4C8008854CBF8003001F0B9B95A4B997989B121
:10E4D80020464A4611F040FFFF2801F0AF81013085
:10E4E8002870CBF80090FAF71DFC2046FFF7E2FEF3
:10E4F80001F0A4B9DFF8FCC0242202FB04C2517861
:10E50800204669F3041151704B4A022182F80090A9
:10E51800039311F0C7FE0122039BCDE209F1FF31FD
:10E528002046C9B211F030FF002840F08B80DFF898
:10E5380010B1DFF8EC909BF80020012332B98BF87A
:10E548000030324B89F800201A70E4E305900393F9
:10E55800FAF7E8FB05988BF80000039B89F8003070
:10E56800364A835C9246A3F13001C9B2092904D91D
:10E57800413BDBB2052B01F2618101300A28EFD162
:10E588004FF0000847460AEB480016F0FDFF7B08ED
:10E598000237FFB20A2F294E0AF8030008F10108D2
:10E5A800F1D1304612F0F6FB002801F047813046E1
:10E5B80012F05EF90746002841F040811D4B3046B5
:10E5C800997912F0F6FB002801F03881297833791F
:10E5D80001392046C9B202220097019612F03CFC8C
:10E5E800022389F8003001F029B900BFEF1E00208E
:10E5F800041E0020183B002003290308CC1D00201E
:10E60800E31E0020C31E0020D01E0020E91D0020AC
:10E61800121E0020931E0020AC1E00209E1E00200B
:10E62800951E0020D0420020E01D0020941E0020EE
:10E638009059002033130020E21E0020C41E002041
:10E648009F1E0020DBF80030DFF80893202B27D02E
:10E65800212B23D14FF436626243297834200139C3
:10E6680000FB0122AC489DF81F3012184FF0000B38
:10E6780020460192C9B20322CDF800B012F0ECFB9B
:10E68800FAF750FB2A78A54B013AA5481A701423CB
:10E69800C9F800B085F800B003703CE31E2B03D125
:10E6A8000133C9F8003019E31F2B18D14FF4366233
:10E6B800624329783420013900FB012296484FF043
:10E6C800000B121801929DF81F302046C9B206228D
:10E6D800CDF800B012F0C0FBC9F800B0FEE29A1FF6
:10E6E800062A0ED88F4B1A7819462AB901321A70A1
:10E6F8008D4B1A788D4B00E3012A40F00C830223DE
:10E70800A1E1A3F10D02042A3AD88949D3B291F8BC
:10E7180000C095F800E08048864ABCF1000F1ED082
:10E728004FF0000C81F800C011784FF43662624354
:10E738000EF1FF3E0CF1340C0CFB0E228018C018B1
:10E748004174382000FB04EE5FFA8EF000EB800085
:10E7580000F5FA409B30C01803F088FBDBE24FF06D
:10E76800010C81F800C04FF4366161430EF1FF3EA1
:10E778000CF1330C0CFB0E1E7044C3185B7C59E083
:10E78800A3F112020B2A4CD86B4A2978107800287A
:10E7980045D000201070A3F1120938224B1E02FB4D
:10E7A8000433203ADBB2534303F5FE435FFA89F999
:10E7B800DFF894B1CB3303EB49039BF800101846FC
:10E7C800039303F053FB5D4A4FF4B66C0CFB04FC57
:10E7D80011781A22013902FB01C14F48494400EB64
:10E7E80041019BF80000DFF870B18875039B9BF826
:10E7F8000010581C0492CDF814C003F037FB4F49A1
:10E80800049A0B78DDF814C0013B02FB03C2424BAB
:10E818004A4403EB42029BF80030D3757BE20123A4
:10E8280008E0DFF8209199F800302BB9012289F827
:10E838000020434A13706EE2FAF774FA002389F84D
:10E8480000302046FFF736FD65E243294BD1354AB3
:10E858001278002A40F05F82354A1278002A40F088
:10E868005A82B9F1000F00F05682364A1278002A0F
:10E8780040F05182212B30D01F2B30D02E4B1978ED
:10E88800012919D9B8F1000F02D1002F00F04382F5
:10E898002D4B02391A7852FA01F010F0010F4FF09F
:10E8A800010004D010FA01F122EA010225E210FA6F
:10E8B80001F141EA020220E200F02D8209F1FF3164
:10E8C8002046C9B211F060FD20B9204B1B78002BFF
:10E8D80040F0218200232B7000E2202300E01E2359
:10E8E800CBF80030FAE1232940F096800D4B1B78D5
:10E8F800002B40F010820E4B1978002940F00B8253
:10E90800104BB9F1000F50D01A783AB30C480F2ABF
:10E9180001700F48017042E1D0420020941E00208F
:10E92800E01D0020E21E0020921E0020F01E0020A4
:10E93800AB1E0020601F0020971E00209E1E002096
:10E94800E91D0020931E0020911E00209F1E00201C
:10E95800121E0020AC1E0020E11E002009F1FF312C
:10E968002046C9B211F010FDB0B19A4A13787BB1B4
:10E97800B8F1000F01D0082B08D90EB1012B05D929
:10E98800002F00F0C881042B00F2C281013351E747
:10E998009DF81F000121F6E08F4B1A78511EC9B26D
:10E9A80008296FD801321A706CE0DFF86CC2242194
:10E9B80001FB04C1487869F304104870022120461D
:10E9C8000492039311F06EFC09F0BEFBFAF7AAF962
:10E9D8008249087840F006000870814801780139BA
:10E9E800C9B201707F48049A50F8211011607E4A1C
:10E9F80082F800907D4A82F80090039BCBF8009043
:10EA080083F800907A4B85F8009083F80690794B4C
:10EA180083F8009000F012BF2A2936D1764B1B7874
:10EA2800002B40F07881754B1A78002A40F07381EA
:10EA380073490B784BB16C48012B02706B4802701C
:10EA480040F26981013B0B7065E1B9F1000F00F0FC
:10EA5800628109F1FF312046C9B211F095FC58B125
:10EA68005C4A137823B1012B40F25581013BE1E662
:10EA78009DF81F00002186E0574A1378012B01D921
:10EA8800013B13700022584B37E1442940F08D8038
:10EA9800594A1278002A40F03E81B9F1000F0DD191
:10EAA800534B9A79511EC9B2012901D8013203E0AA
:10EAB800032A40F03081023A9A712CE1504A1278C8
:10EAC800002A40F02881444A1278002A40F0238125
:10EAD8004A4A1278002A58D13E4B1B78012B09D993
:10EAE800002E00F01881474B1A78102A00F2128184
:10EAF8000132AAE019D1B8F1000F0BD0424A032025
:10EB080011789846013191FBF0F000EB4000091AAA
:10EB1800117000E1002E00F0FE803B4A1E4611787D
:10EB2800013101F003011170F5E0314B204699796C
:10EB38004A4611F011FCFF2800F0ED80DBF80030A8
:10EB4800212B00F0E8801F2B00F0E58001302870B1
:10EB58002046FFF7AFFB4FF436626243297834232F
:10EB6800013903FB0123294A9BF80000D31893F8C5
:10EB7800049049468DF81F90FFF770FB0146002866
:10EB880040F0AC804846224AA6E00D2B0BD19DF8F8
:10EB98001F0011F0ABFA30B11E4B1A783F2A00F271
:10EBA800BA800132A9E00120AAE0552940F0B380DB
:10EBB800114A1278002A40F0AE80B9F1000F2DD129
:10EBC8000B4B9A79012A01D9013A75E740F0A380E5
:10EBD800032271E7971E00209F1E0020E31E0020DD
:10EBE800C31E0020D01E0020E91D0020121E002098
:10EBF80033130020951E0020E21E0020AB1E0020CB
:10EC0800931E0020911E0020E11E0020D04200200B
:10EC1800AC1E0020601F0020183B0020894A127893
:10EC2800002A78D1884A1278002A74D1874A127843
:10EC3800002A56D1864B1A78012A08D9002E6AD0A4
:10EC4800844B1A78012A65D9013A1A7062E012D108
:10EC5800814B197811B1013919705CE0B8F1000FD6
:10EC680003D002211970904655E0002E53D003219D
:10EC7800197016464FE0B9F1010F4CD9774BA9F13D
:10EC8800020220469979D2B211F074FBFF2842D0D3
:10EC9800DBF80030DFF8D091212B3CD01F2B3AD085
:10ECA800013028702046FFF705FB4FF436626243B7
:10ECB80029783423013903FB0123694A99F80000B4
:10ECC800D31893F804B059468DF81FB0FFF7C6FA69
:10ECD800014618B958464A46FFF7D0FAFAF722F81B
:10ECE80019E00D2B0BD19DF81F0011F0FFF930B181
:10ECF8005C4B1A78012A0ED9013A1A700BE0FF20F2
:10ED0800584911F011F906E000273E46B84602E0DE
:10ED1800012700E001262978DFF89891002940F0C2
:10ED2800CB8099F8003013F0010205D143F00103BC
:10ED380089F800304C4B1A6000252046294611F00E
:10ED4800BDFD30B172236343484AD15C41F00201F2
:10ED5800D1540135382DF0D13A356543434E735DB2
:10ED680013F0020F43F3400015D03F4C206810B950
:10ED78003F4900F0CFBC00203E49F9F70FFF735D13
:10ED880013F00C0F43F3810540F05885F9F7CAFFDB
:10ED9800256000F053BD314DAB79A3B1012B01D1F2
:10EDA800354906E0022B01D1344902E0032B02D198
:10EDB8003349F9F7F3FEA979204611F017FB02222F
:10EDC80001463048EDE114B920462F4901E02F49AA
:10EDD8001846F9F7E3FE2E4803786BB92D490A2245
:10EDE8002D48F1F7ADFD2D49242303FB04135A7870
:10EDF80042F010025A7004E0274829490A22F1F724
:10EE08009FFD284D3821022205F11E00F9F7ECFE7E
:10EE1800204611F00FFB0222014605F11900F9F70F
:10EE2800E3FE214B00221A70204B1B7803F080036D
:10EE3800DBB2002B00F002851D4B1B88EB8100F034
:10EE4800FDBC00BF931E00209F1E0020AB1E0020AB
:10EE5800971E0020911E0020E11E00203313002081
:10EE6800D0420020601F0020AC1E002090590020D6
:10EE780045290308662903086E2A03088F2A030810
:10EE8800B02A030812020020A82903082C2A030824
:10EE9800E01D0020D12A0308FA010020183B0020B9
:10EEA800F22A0308F4010020951E0020083B0020E8
:10EEB80075A30308E31E002001392046C9B211F0EA
:10EEC80063FA002800F00284954B93F800B03823C9
:10EED8000BF1FF3B03FB04BB99F800305FFA8BFB97
:10EEE80013F0010F03D08F4A1378002B41D08E48BE
:10EEF800F9F7FAFD0BEB0B1101F5EA4110228B48EB
:10EF0800BB3102F0CEFF884B11229A71884B1B68E7
:10EF180013B91020874921E0012B02D1102086491E
:10EF28001CE0022B02D11020844917E0052B02D1E6
:10EF38001020834912E01E2B02D1102081490DE0D8
:10EF48001F2B02D11020804908E0202B02D110206D
:10EF58007E4903E0212B03D17D491020F9F71EFEDD
:10EF680099F800306F4843F0010389F80030002316
:10EF78000370784B1A78002A00F0AB800BEB0B1B60
:10EF88000BF5EA4909F1BB0910227348494602F01A
:10EF980088FF00229346704B995C41B10BF1010B3D
:10EFA8005FFA8BFB0132BBF1100FF4D107E06A491D
:10EFB800C2F1100201EB0B002021F1F7EBF9654AD1
:10EFC800107858450BD90138484402F059FF30B938
:10EFD800604B202118780138484402F047FFDFF8D9
:10EFE80094B19BF8003018460393F9F793FEDC467A
:10EFF800039BDFF878B110B9432B44D101E0432BD0
:10F0080005D100238BF800304FF0200A30E0534838
:10F01800534A90F800E053499E450ED1AEF1300EA8
:10F028000A20137800FB0E1E0133DBB21370734401
:10F0380093F8AD307BB913700DE003709BF8003086
:10F048004FF0000E82F800E02BB1424803780F2BF6
:10F0580001D80133037040238BF8003013789CF8F3
:10F0680000200A20303A00FB0211C91891F8ADA01F
:10F078003849394A08785146013802F800A048440E
:10F0880002F0F4FE0FE0384B1B7803F08003DBB28C
:10F098004BB19BF8003033B92E482F490378FF2233
:10F0A800CB1803F8012C9BF8003013B12F4A013B11
:10F0B80013709BF80030012B10D1264A13780F2BC0
:10F0C80001D801331370264A00238BF800301370DF
:10F0D80004E004200C21144AF9F718FD144A1368B7
:10F0E8009346002B48D14FF4366262432978342482
:10F0F800013904FB01241E4AA4186178164AC1F399
:10F10800C30109B93F2004E0994201D9DB2000E09E
:10F11800A5200133DBB2907501320A2BF1D18DE3C2
:10F128009E1E0020951E0020F41E0020FB1E0020BD
:10F13800AC1E0020EF360308D92B03081B2C03084C
:10F14800E12C0308862D0308A72D0308C82D030802
:10F15800E92D0308931E0020F4010020E61D00207D
:10F16800121E002010B40208083B0020E91D0020F0
:10F17800D8420020CC1D0020012B15D14FF4366356
:10F1880063432A783424013A04FB0234AB4BE41875
:10F19800637813F0070300F0518314215943A848FA
:10F1A8008322F9F721FD49E3022B26D1A54A9DF8D0
:10F1B8001F30882101FB03232978A34AD879013914
:10F1C8000623202502F8015950FA03F515F0010F1E
:10F1D80010D04FF436656543342606FB01559B4E27
:10F1E8007519ED791D4115F0010F01D0DB2500E0FF
:10F1F800A5255570013BE4D220E3032B13D14FF42E
:10F20800366363432A783424013A04FB02348F4B73
:10F218001C19237A13F0010F02D010208C4979E2CF
:10F2280010208C4976E2042B13D14FF436636343E4
:10F238002A783424013A04FB0234844B1C19237ABB
:10F2480013F0020F02D01020834963E21020834993
:10F2580060E2052B15D1162700262B783422013BB6
:10F2680053434FF4366202FB0433784A7C49D3187F
:10F27800985DC919013616F06DF90237052EECD1E3
:10F28800DCE2991F062900F2FF809DF81F206D4FD0
:10F2980002EB0210411807EBC101C968714801F17E
:10F2A800100651F804CBB14240F804CBF9D19E1FA7
:10F2B800F6B202EB02129219013207EBC202507A3F
:10F2C80092F80AC0684A29781378904673B94FF4BF
:10F2D800366363433422013902FB0131634BCA5E52
:10F2E800634B024102EA0C021A7011E0022B0FD1A3
:10F2F800604B01391B784FF0000900932046C9B2D2
:10F3080004223346CDF8049011F0A6FD88F8009049
:10F3180098F80030012B29D1574BDFF8589193F812
:10F3280000A05046F9F7F6FC10B9BAF1430F1AD10C
:10F338000DF11F005149FFF70BF810B1002389F8B0
:10F3480000309DF81F30DBF8002003EB03139B18F7
:10F3580007EBC303504699F8001013F8202CFAF76E
:10F36800F3FC89F8000099F800A003E013B9404BBA
:10F3780093F800A0BAF1090F07D9BAF1630F8CBF4F
:10F388004FF003094FF0020901E04FF001099DF821
:10F398001F3003EB03139E1907EBC607FB685A7B64
:10F3A800E02A02D12E4A202151779A7BE02A02D105
:10F3B8002B4A20219177DA7BE02A02D1284A2021A2
:10F3C800D17798F800200ABB4FF436626243297857
:10F3D8003424013904FB0124184AA418A27812F035
:10F3E800080F1BD05A7BE02A02D11D4A3F215177D2
:10F3F8009A7BE02A02D11A4A3F219177DB7BE02BE6
:10F4080040F01C82164B3F22DA7717E21C4B1B7820
:10F4180003F08003DBB2002B40F010820DF11F00D7
:10F428001649FEF76FFF18B15046FEF755FF05E283
:10F4380014485146C9EB00004A46B2E6D8420020BB
:10F448000F0200204C0D002013020020D0420020A3
:10F458007E2C03089F2C0308442D0308232D030842
:10F46800F401002004020020E21E0020D542002002
:10F47800921E0020F01E0020CC1D0020AC1E002093
:10F48800083B002014020020A3F10D02042A31D801
:10F498009DF81F30D6B2222202FB03639F4A02EB7B
:10F4A80083035F6C3846F1F7C5F9394602469C4834
:10F4B800F1F746FA9B4B1B786BB19B4B1B7803F01B
:10F4C8008003DBB21BB1994820210222FBE0984B54
:10F4D800964819780CE04FF4366363432A7834244D
:10F4E800013A04FB0234934B90481C19A619717C0D
:10F4F800822256E6123B0B2B00F2A0819DF81F20BA
:10F50800DBB2222101FB0231844A163152F8212054
:10F51800834902F110008A4652F804CB824241F82E
:10F5280004CBF9D1DFF84C92DFF84CB22FB199F83F
:10F538000020012A15D1013209E096B199F800207E
:10F54800012A07D97C49097803290AD1013A89F89F
:10F55800002006E005D178490978032908BF8BF80F
:10F56800002099F800209AB94FF4B6614C432A78E4
:10F578001A21013A01FB02446E4AE318083302EBF0
:10F5880043039A798BF80020DA796B4B1A7055E1AE
:10F598006A4C202104F118000822F0F7FBFEB8F1AC
:10F5A800000F00D1AEB1644D2B78012B01D1644A14
:10F5B80001E04BB9634A136823615368CAF8043001
:10F5C800B8F1000F2FD00BE0022B0CBF5E4A5F4A48
:10F5D800F1E75F4A136823615368CAF8043027E1EA
:10F5E8009BF80000554A3121002350FA03F515F025
:10F5F800010F01D0117601E02D2515760133013177
:10F608000132082BC9B2F0D1474B1B7803F08003B5
:10F61800DBB2002B44D099F80030012B40D9E41814
:10F628002023A3753CE0002E00F00281202108224F
:10F638004848F0F7AFFE3D489BF800108222F9F7E2
:10F64800D3FA394B1B7803F08003DBB21BB199F86E
:10F658000030012B02D82B78032B21D12021022244
:10F668003248F0F797FE1BE050FA03F515F0010F4A
:10F6780001D0117701E02D251577013301310132D1
:10F68800042BC9B2F0D1284B1B7803F08003DBB2FE
:10F6980033B199F80030012B02D9E4182023A3765E
:10F6A800214B1B7803F08003DBB2002B00F0C680EF
:10F6B80099F80030012B40F0C180002F40F0BE8047
:10F6C800174820210822F0F765FEB7E099F80030C6
:10F6D800214D13F0010F04BF43F0010389F80030F6
:10F6E8002E78002E4AD12D210A221C48F0F752FE0E
:10F6F80004201B49F9F752FA1A4B1B78012B02D147
:10F708001020194906E0022B02D11020174901E008
:10F7180017491020F9F742FA90E000BF4C0D00207D
:10F7280004020020AB1E0020083B0020120200202B
:10F73800601F0020D0420020E11E0020F4010020BC
:10F74800293603084A3603086B3603088C36030843
:10F75800A53503080C0200209F1E0020C41E0020AF
:10F7680018380308951E0020022D0308C02C030832
:10F77800E12C0308971E0020911E0020314B1C78B5
:10F788002046F9F7C7FA304B304A00282AD0304FC4
:10F7980030493878A04216D130380C782E4E00EB1C
:10F7A80080073C19345D04B90C700F7800EB8000B9
:10F7B800C4190137FFB2C0190F70315C345D59B9F3
:10F7C8002448017008E00120087019783C7019B1CC
:10F7D800092E9CBF36182E702978511801F8014C53
:10F7E80040211970197811B1174801390170197839
:10F7F800012909D12978092902D81848013101704D
:10F8080000211970134B19701168154BC3F81610A5
:10F818005168C3F81A101289DA83124A127802F072
:10F828008002D2B252B12A789B1820225A7505E07C
:10F838009BF800000A4A3121002315E709B0BDE80A
:10F84800F08F00BFCC1D0020E91D0020C41E002041
:10F85800E61D0020121E002010B402089F1E002082
:10F86800F4010020083B002010B5002386B00446B0
:10F878008DF8143011B118460C4901E008460C49BE
:10F88800F9F78CF9217810220139C9B201EB01117D
:10F8980001F5C241483101A802F003FB10200146DE
:10F8A80001AAFDF7DFFD06B010BD00BF1016030862
:10F8B800521603080B4B1B78442B06D0552B0378A4
:10F8C80001D013B17047013B01E0037801330370A5
:10F8D80003780BB9403302E0412B01D1403B037060
:10F8E800FFF7C2BFCC1D00202DE9F74FDFF8CC9100
:10F8F800DFF8D8A199F80030554643F0010389F89C
:10F9080000309AF80130644C23F07F039B46D3B152
:10F9180000206249F9F742F961482A21F0F7B8FD59
:10F9280018B121788222F9F75FF92278002A40F08D
:10F93800AF802B6862F3CF332B605A4B1A7842F0B2
:10F9480003021A70A4E0574F23703B783E4603F039
:10F958000202D2B20192DFF87881002A44D013F073
:10F9680001092BD058465049F9F718F998F8003092
:10F97800232B0CD14D4B4E4A4E481A600121FFF7FC
:10F9880073FF3B7803F0FE036BF341033B7098F879
:10F9980000302A2B7CD1337803F0FE036FF3410348
:10F9A80033702B6843F400432B600F232370414BC3
:10F9B800187803B0BDE8F04F0FF01CB848463E4930
:10F9C800F9F7ECF898F80030232B61D1374B384A17
:10F9D80038481A600121FFF747FF3B7869F30003B5
:10F9E80069F341033B7053E00EF054FF05460028CD
:10F9F8002FD001212F48FFF75DFF98F80030532BD7
:10FA080012D13B78019A03F0F10362F300033B70D3
:10FA1800DAF8003043F40043CAF800300F232370AB
:10FA2800244B18780EF0E6FF98F80030232B2FD1DE
:10FA38003378002203F0FD036FF3000333701D4B8E
:10FA48001A70F9F76FF91D4A137843F0060313701B
:10FA580014E01B49F9F7A2F898F80030232B17D1C6
:10FA68003B7865F3410365F300033B70F9F75AF9F6
:10FA780099F8003043F0060389F80030114A1378EA
:10FA8800013BDBB21370104A52F82320074B1A606F
:10FA980003B0BDE8F08F00BFFA5C0020941603089D
:10FAA800F4010020AB3F0020B5160308041E002017
:10FAB800B4B502089E1E0020D6160308E31E0020D7
:10FAC800F7160308C31E0020D01E0020083B0020A4
:10FAD800CC1D00202DE9FF41364C374D237843F0EB
:10FAE80001032370297801F00401C9B211B9334820
:10FAF800FFF7E0FE2B7803F00402D2B232B1304AAD
:10FB080012781AB92C4A43F0080313702D4E337833
:10FB1800232B26D12B782A4A6FF3C303002113F035
:10FB280004082B70284F117009D0234A61F382030F
:10FB38001370264B21483B60FFF796FE11E0F9F75A
:10FB4800F1F82378224A43F0060323701378013B27
:10FB5800DBB213701F4A52F823303B60174B83F80F
:10FB680000803378532B23D12B780424144A03F0D4
:10FB7800F403234314702B70104B0B221D78164985
:10FB8800013DEDB202FB05F000F5CA40883002F0F5
:10FB980082F900201149F9F701F8FF2300210093A9
:10FBA8000135162022460B460191029502F0E6F92E
:10FBB800BDE8FF81E31E0020AB3F00209E1E002011
:10FBC800FA5C0020CC1D0020041E0020D0B50208DD
:10FBD800C31E0020D01E0020A03F0020731603087B
:10FBE8002DE9F041984B04469A7812F0010F00F085
:10FBF80017811B88002B40F01381944D95F8203015
:10FC08003F2B40F2D780012C14D1914B1B7803F085
:10FC18000203DBB2002B00F0C48095F820208B4B48
:10FC2800402A03D1013283F82020FBE0482283F8E0
:10FC38002020B6E0022C03D1482385F82030B0E01C
:10FC4800844E337803F02002D2B28AB195F820208E
:10FC5800402A0DD1032C0BD07F4B804A03F11001B1
:10FC680053F8040B8B4242F8040BF9D1412395E079
:10FC780003F01003DBB28BB195F82030412B0DD186
:10FC8800032C0BD0764B754A03F1100153F8040B83
:10FC98008B4242F8040BF9D142237FE0F37813F04A
:10FCA800010F0FD095F82020422A0BD16D4B6B4ADB
:10FCB80003F1100153F8040B8B4242F8040BF9D1FD
:10FCC80043236BE003F00202D2B27AB195F8202008
:10FCD800432A0BD1644B614A03F1100153F8040B1A
:10FCE8008B4242F8040BF9D1442357E003F0040295
:10FCF800D2B27AB195F82020442A0BD15B4B574AEF
:10FD080003F1100153F8040B8B4242F8040BF9D1AC
:10FD1800452343E003F00803DBB28BB195F82030AC
:10FD2800452B0DD1032C0BD0514B4C4A03F110013C
:10FD380053F8040B8B4242F8040BF9D146232DE00B
:10FD48000FF03EFCA0B14B4B1B788BB195F82030DF
:10FD5800462B0DD1032C0BD0474B404A03F1100121
:10FD680053F8040B8B4242F8040BF9D1472315E0F2
:10FD7800F37803F04003DBB29BB195F82030472BB2
:10FD88000FD1032C0DD03D4B344A03F1100153F829
:10FD9800040B8B4242F8040BF9D1482385F8203034
:10FDA80078E095F820300133DBB2472B85F8203016
:10FDB8007FF629AF95F82060472E04D9234B0026FB
:10FDC80083F8206001E00136F6B206F14007FFB281
:10FDD80012E02B48314615F0A2FB08B1032C04D1E0
:10FDE800284B9B5D23B1032C02D185F820600FE0DE
:10FDF8000136F6B2BE4203D03F2EEAD9402E07D1D3
:10FE0800214B1E221A70402385F82030BDE8F0816E
:10FE180095F820001149652246F61563F8F70AFEA1
:10FE2800012C37D1194B0D4A03F1100153F8040B7B
:10FE38008B4242F8040BF9D1044B93F820303F2B46
:10FE48003CD9002012493EE0F41E0020F4010020B5
:10FE5800301A0020083B0020481D0308FB1E002024
:10FE6800691D03088A1D0308AB1D0308CC1D030880
:10FE7800ED1D0308C44200200E1E0308501E03088F
:10FE8800DA1A0020901A0020A01E002048800308DB
:10FE9800061D0308104BD87800F02000C0B220B12E
:10FEA800022C06D000200D490DE0032C01D10C498D
:10FEB80009E00C4B93F820303F2B02D800200A4968
:10FEC80001E00A490020F8F769FE1020084A0146B7
:10FED800BDE8F041F8F71ABE083B002021140308DA
:10FEE800271D0308F4010020C41C03082F1E030863
:10FEF800F41E002010B5F8F715FF084B1B7803F027
:10FF08000403DBB22BB106490020BDE81040F8F726
:10FF180045BE0220BDE81040FFF762BE301A00203F
:10FF2800F61A030870B5224B06461B78214CF3B924
:10FF3800257819E02048294615F0F1FA78B12368A8
:10FF48009D4202D9FF2E02D007E0FF2E02D19D422A
:10FF580008D202E036B91DB913B9256012E00EB90E
:10FF6800013500E0AD19EDB23F2DE3D90AE0013BC0
:10FF78002021124810222360F0F70CFA00201049C3
:10FF8800F8F70CFE0F48F8F7AFFD46F61563207832
:10FF98000D496522F8F74EFD084D216805F110005E
:10FFA80001310222F8F720FE2D23AB7470BD00BF8B
:10FFB800931E0020AC1E00200A1E0020F401002021
:10FFC800C45E0308F41E0020FB1E0020F8B5594B40
:10FFD800F02259481A700378044613F00E051DD113
:10FFE800564A43F00203156000F8013B15F03CFA4D
:08FFF8002C46534BE35C1BB1E6
:020000040801F1
:100000005248214615F079FA0134402CF5D1504B75
:1000100001221A7010F026FB4E4B1A7842F00102B2
:100020001A70F8BD13F00C0543D12E4647482946F7
:1000300015F079FA08B10136F6B20135402DF5D147
:100040001EB9237843F0040331E0002542482946D5
:10005000EFB215F068FA68B13B4BEB5C53B13F4B24
:1000600001371F700020FFF761FF237843F008037A
:10007000237002E00135402DE8D1394D3A21284660
:10008000F0F70AFA38B1401BC0B2013028183146E7
:100090000222F8F7ADFD334B1B78532B4CD12F4B7D
:1000A00000201870FFF742FF237843F00803237005
:1000B000F8BD6FF34103037003F00403DBB2294D75
:1000C00023B100202849F8F76DFD0EE02B78552B61
:1000D00001D1FF2002E0442B02D10120FFF726FFCF
:1000E00013200D21214AF8F715FD2B78232B23D15E
:1000F0002478134E04F00204F4B9154B1C7010F070
:10010000B1FA337803F0FB0364F3C30333700D4B90
:100110001C60F8F70BFE0F4B1A7842F006021A70BB
:10012000134A1378013BDBB21370124A52F82320B2
:10013000114B1A60094B1C70F8BD00BFEF1E002068
:10014000091E0020AC1E0020302D00200A1E0020B9
:1001500078140020E31E0020311A0020931E002096
:10016000F4010020CC1D00200A700308F41E0020BA
:10017000C31E0020D01E0020041E002070B50546BE
:100180000C4616463BB1400000F536403930401869
:10019000114601F06FFE054B292202FB0535F309DC
:1001A0002C1906F07F066370E67070BD793D002063
:1001B00038B510B3A0F14103DBB2432B1FD9C509F9
:1001C00000F07F040BD0052C19D90021601E0A46CF
:1001D0000BF072FAD0F1010038BF002038BD082CB6
:1001E0000FD9601EC0B229462A460AF0C7FE50B990
:1001F000402C8CBF0020012038BD012038BD0020DC
:1002000038BD284638BD284638BD0000F7B5604FD8
:10021000604C387831234000237400F536400133B8
:1002200023763930053B6374637601F02DFEC0B24E
:1002300020F07F0200F07F01D2B28DF804108DF81B
:10024000002004F1120359B9534A04F11500118832
:10025000927861829A7020210222F0F79FF80CE0D8
:10026000D20904EB8202526A10886082927804F10B
:1002700015009A700222F8F7BBFC3878400000F5B0
:1002800036403A3001F000FEC0B220F07F0300F0AB
:100290007F01DBB28DF805108DF801303F4851B970
:1002A0003D4B20311A889B78628383700222033091
:1002B000F0F774F80BE0DB0904EB83035B6A1A8840
:1002C00062839B78022283700330F8F791FC344BF1
:1002D0001B7813F0010F5AD0324D02A92A788B18DF
:1002E00013F8041C13F8086C2F4B1B78232B04D134
:1002F000002A41D1223B2B703EE02A2B04D1002A58
:100300003AD0013A2A7037E0552B46EA010611D15E
:100310000DE02B7802AAD318013E13F8081CF6B2A0
:100320003046C90913F8042CFFF742FF98B9002E94
:10033000EFD121E0442B19D115E02B7802A9CB187D
:10034000013613F8081CF6B23046C90913F8042C1C
:10035000FFF72EFF38B1134B387819783246012356
:10036000FFF70CFF08E0902EE7D905E0532B03D1EF
:10037000533B2B70F9F7CCFC0C4B1B7803F080033C
:10038000DBB223B12B782022023304F83320FEBDE8
:10039000931E0020F4010020077C03080E020020B9
:1003A000E31E00209E1E0020CC1D0020083B0020E4
:1003B000024800210922EFF7F1BF00BFB11E002063
:1003C00070B50A46002405E01B19811A2A2501345C
:1003D0005D54E4B20F4D104B295D09B19442F3D145
:1003E000801A001918182021121BEFF7D7FF0B4BAA
:1003F0001E7876B1432E07D114B1013CE4B201E07E
:10040000074B1C7000232B553046F8F787FC00B1D2
:100410002E5570BDB11E0020F4010020CC1D00201F
:10042000F21E002038B5184C184DA07800F01000CE
:10043000C0B250B91649F8F7B5FBFFF7B9FF23680A
:1004400043F4801323600F232B702A782AB9236882
:10045000FF2062F31453236038BD0E48C5792DB9CF
:100460001C200821FFF7ACFF284638BD23680A4945
:100470006FF3145308222360F0F710FA00280CBF22
:100480000120FF2038BD00BF083B0020F21E0020E5
:10049000591B0308B11E0020609B0308F0B55C4C9B
:1004A00085B0667806F01006F6B2002E3ED1594BA4
:1004B0001A78594B013A53F82230584A934204D1E2
:1004C000574B1A7842F0020207E002F11C018B42FE
:1004D00008D1534B1A7842F00402022161F3C7029B
:1004E0001A7019E03832934216D1FFF79BFF0028AB
:1004F00000F08C8001284A4D06D12B78022243F06F
:10050000010362F3C70306E030464649F8F74AFBA9
:100510002B7866F3C7032B70434B1A7842F0010225
:100520001A70236843F4805323606FE03C4D2B78AE
:1005300013F0F80606D03D49002005B0BDE8F040B4
:10054000F8F730BB13F0070F41D003F00202D7B227
:100550004FB11220314611F0FBF9FF2300930196B1
:10056000029643202AE003F00406F6B2A6B139460B
:10057000384611F0EDF9382102200FF079FD0AF02C
:10058000B3FA0EF0B3F9FF230093019702974420CA
:10059000394604223B4614E013F0010F13D0012129
:1005A00043F6206011F0D4F93046F5F7F5FE204B04
:1005B00045201E80FF2300930196029631460422B7
:1005C000334601F0DFFC00201A49F8F7EBFA2B78EC
:1005D00003F0FA036FF341032B70174B1B78232BA7
:1005E00014D123686FF30C332360F8F79FFB0E4B95
:1005F0001A7842F006021A70064A1378013BDBB201
:100600001370054A52F823200C4B1A6005B0F0BD58
:10061000083B0020C31E0020D01E0020ECB50208BD
:10062000745A00207A1B0308E31E0020A6730308F7
:10063000E21D002085730308CC1D0020041E00204D
:100640001FB50446F5F794FFA8B14B2002F070F8EF
:10065000FF2300930121FF3B0193392004220B4625
:100660000134029401F08EFC064B01205A7842F0CE
:1006700004025A7004E0044B1888003818BF0120A7
:1006800004B010BD783F0020105D0020F0B5204E72
:100690000024337A0546013385B00F4633721020AB
:1006A0002146012223460094F2F72EF855B9FF2384
:1006B00000934F20294604222B460195029701F012
:1006C00061FC0EE0012D0CD1FF2300935020234646
:1006D000214604220194029701F054FC337A013B35
:1006E0003372337A052B11D1FA33012100240093A0
:1006F00027200B4604220194029401F043FC044B92
:100700001C7205B0BDE8F04001F0E4BF05B0F0BDDB
:10071000A21E0020074B292202FB00335B7913F055
:10072000100F05D0044B283ADA711A7109321A7287
:10073000704700BF793D002033130020044B187828
:10074000A0F1010CDCF1000040EB0C00704700BF91
:10075000001E0020034B1878A0F10202504240EB2B
:1007600002007047001E0020034B1878012894BF38
:1007700000200120704700BF001E0020064B1A78A1
:1007800002F0F7026FF304121A70044B00221A7081
:10079000034B03321A707047B01E0020F21E002077
:1007A000001E002010B52148214903680A789C7B6F
:1007B000944203D99C8914F0200F18D09A8912F022
:1007C000800F01D105E01C3B9A8912F0400FFAD04E
:1007D00000E01C33036000230B7003689B8913F057
:1007E000200F16D0134BDA79114B1A7011E0013239
:1007F000D2B20A70986843F60953984209D101E0D1
:100800000132D2B2162A03D80B4853B29840F7D41B
:100810000A700A4A136843F480731360F8F7CAF841
:10082000074B1A7842F006021A7010BD041E002011
:10083000931E0020A21E002000060088083B002016
:10084000E31E002010B52349234A0B78D3B110686A
:10085000848914F0200F15D1013BDBB20B70846842
:1008600043F60952944228D104E013B1013BDBB2B4
:1008700000E0837B162B03D8184C5AB29440F4D472
:100880000B701AE01368988910F0400F01D106E050
:100890001C33988910F0800FFAD0136002E00E48E4
:1008A0001C3B036013689A7B0A709B8913F0200F2E
:1008B00003D00B4BDA79074B1A700A4A136843F4DA
:1008C00080731360F8F776F8074B1A7842F0060247
:1008D0001A7010BD931E0020041E00200006008820
:1008E000A21E0020083B0020E31E0020074B084A00
:1008F0001B68934202D01C32934205D1054B1878F5
:10090000003818BF0120704700207047041E0020E7
:1009100040B602082C1A0020074B084A1B68934275
:1009200002D01C32934205D1054B1878003818BF0D
:100930000120704700207047041E002078B602088E
:100940002C1A002070B50A4C0546E07100F56A507B
:100950007C3001F099FA207005F5D840E93001F0BB
:1009600093FA60702046BDE87040F5F72DBD00BFDA
:10097000A21E00202DE9F0479A4B86B01A78064651
:100980000F461C461AB1012A40F0DA812FE0964B3F
:100990001A68964B9A4200F0D581F5F769FA944BA4
:1009A0005B7803F00203DBB253B9924B5B7803F040
:1009B0008003DBB223B901F0B3FE08B90AF094F862
:1009C0008D4B1A686FF310421A6037B98B4B187849
:1009D000F8F7A4F9002800F0B581FFF7E9FC884B8F
:1009E0003C221A70F7F7E6FF237801332370844B1B
:1009F0001B7813B9FFF7C2FEA4E1012130460AF0CB
:100A0000ADF8F7F7CBFF00207E49F8F7CBF80621C9
:100A10001B20FFF7D5FC7C4B7C491A7898468A1836
:100A200012F8312C002A00F08D81794A7949137827
:100A300091F80090C3F3C00AC3F3001503F0F70365
:100A40006FF3041309F00109137017B10223237027
:100A500000E027700B21062204A801F026FA98F87E
:100A6000002004A86949303AEFF7BEFB044610B1F4
:100A70001227002429E04AF6EB0001F005FA0028CD
:100A8000F6D0654D2C72F5F759FB0446002840F06E
:100A90005981624A544B21461A60FF23009301900A
:100AA000029004220820234601F06CFA012223461A
:100AB0000E2021460094F1F727FE594B1A7842F098
:100AC00004021A700123AB713CE13946062204A8E6
:100AD00001F0EBF998F8002004A84C49303AEFF700
:100AE00083FB002840F020812046FFF7A9FD002865
:100AF00040F02881DFF82081012188F80800204695
:100B0000F5F72AFB49EA0A090746F5F717FB00281B
:100B100040F0BF8038464349EFF744FDC0B901F0CB
:100B200011FD314BB9F1000F02D115B93E4A24E055
:100B300035B13E4A1A603E4B1A786FF3410205E028
:100B40003C4A1A603A4B1A7865F341021A70E5E0A4
:100B500038463949EFF726FD20B138463749EFF7D7
:100B600021FD78B9B9F1000F40F0EC80002D40F084
:100B7000E98001F0E7FC324A1B4B1A603046FFF770
:100B8000C9FDCBE038462F49EFF70CFD50B94AF6C6
:100B9000E900012101F06EF9174A136843F400538C
:100BA0001360DFE738462849EFF7FCFC40B9B9F19C
:100BB000000F40F0C780002D40F0C480234A0DE0B4
:100BC00038462349EFF7EEFC002845D1B9F1000F74
:100BD00040F0B880002D40F0B5801E4A024B1A60EC
:100BE0009CE000BF001E0020041E002040B602084A
:100BF000F2340020873F0020083B0020CC1D00205D
:100C0000F21E002000140308E81D0020B11E002081
:100C1000B01E00205B680020A21E0020B0B60208B3
:100C2000FE260020C1A30308FCB8020884BA02080B
:100C3000E31E00205CB602083DA30308CDA503080F
:100C4000A0BA020878A303087AA30308D8BA020856
:100C50008AA5030878B6020838463C49EFF7A2FC9B
:100C600000285BD101F06EFCB9F1000F07D0384AC3
:100C7000384B1A60384B1A786FF3410261E0002D4F
:100C800060D0364A334B1A60334B1A7869F341020D
:100C900057E038462D49EFF785FC054628B901F0A5
:100CA00051FCB9F1000F4DD01EE038462C49EFF74A
:100CB00079FC002846D038462A49EFF773FC40B942
:100CC000B9F1000F3ED1284A224B88F807401A603C
:100CD00038E038462549EFF765FC054660B9B9F1BB
:100CE000000F16D001F02EFC194A1A4B1A601A4B4D
:100CF0001A7865F3410224E038461D49EFF752FCAB
:100D000020B138461B49EFF74DFC10B9B9F1000F7F
:100D100018D1194A0F4B1A6001F014FC2046FFF756
:100D200011FE402C0ED105E00134E4B20737402C0F
:100D30007FF4CBAE711C0020C9B2FFF7A7FC01E025
:100D400000221A7006B0BDE8F08700BF7CA303083C
:100D50005CB60208041E0020E31E002084BA0208CC
:100D60007AA303088AA5030878B60208C1A303087A
:100D70003DA3030878A303082CBB0208034B1B7890
:100D800053FA00F000F00100704700BFA21E0020DF
:100D9000034B1B189878003818BF0120704700BF1C
:100DA000A21E0020F8B504460D460E78FFF7F0FFAE
:100DB00000B3124A13199F78104600230219927843
:100DC0001A4112F0010F4FF001020BD0BE422978F8
:100DD00003D09A4042EA010102E09A4021EA02016E
:100DE000297004E09A40297821EA02022A7001332E
:100DF000082BE3D12B7803B92E70F8BDA21E00207A
:100E000070B57D4B044631B11B78532B40F0F28016
:100E1000533B037070BD1A78302A32D1774B1A7960
:100E20005AB1774A77491278292000FB0212527989
:100E300012F0100F01D001221A71734A257812782E
:100E4000154011D01D7A002D40F0D480E8B2FFF794
:100E500095FF28B10123AB40227822EA03032370D7
:100E60000135082DF2D13FE0E8B2FFF787FF20B14E
:100E70000123AB402278134323700135082DF3D1B1
:100E800032E0A2F13101C9B2072939D85B4E32797B
:100E90005AB15B4A5B491278292000FB0212527951
:100EA00012F0100F01D0012232711D78313DEDB2E8
:100EB0002846FFF763FF002800F09C80237853FA50
:100EC00005F212F0010F09D0327A002A40F0928028
:100ED000013212FA05F523EA050304E0012212FAB1
:100EE00005F545EA03032370002112224748EFF776
:100EF00055FA464920461022BDE87040FCF784BAF6
:100F0000132A0CD0552A18D13D4B3E4A1B78292173
:100F100001FB03235B7913F0200F03D170BD374B26
:100F200001221A7100202146FFF73CFF0020FFF745
:100F30002FFF00285ED0002054E0142A0CD02A2A6B
:100F400018D12F4B2F4A1B78292101FB03235B79F2
:100F500013F0200F03D170BD284B01221A7101201C
:100F60002146FFF71FFF0120FFF712FF002841D0A5
:100F7000012037E0152A0CD0232A18D1204B214A12
:100F80001B78292101FB03235B7913F0200F03D188
:100F900070BD1A4B01221A7102202146FFF702FF91
:100FA0000220FFF7F5FE002824D002201AE0162ABE
:100FB0000CD0442A1ED1124B124A1B78292101FB66
:100FC00003235B7913F0200F03D170BD0B4B01227B
:100FD0001A7103202146FFF7E5FE0320FFF7D8FE34
:100FE00040B103200949102246F67973BDE87040EC
:100FF000F7F724BD70BD00BFCC1D002033130020C7
:10100000961E0020793D0020A21E0020CE1D00204B
:101010002DE9F043002387B08DF81730804B1B7803
:10102000012B00F07E827F4C227872B17E4B5B7880
:10103000002B40F076827D4D2B78002B40F0B9805C
:10104000F7F774FE09232B70B3E0784B19781D462F
:10105000082900F2AE8076490978232913D11A7045
:10106000F7F764FE7349744A0B7853B17348013B38
:101070000478DBB244F0060404700B70704951F838
:1010800023301360C1E26D4B1A7812F0010F04D1C6
:1010900001210A438DF817101A70F1F767FF28B97C
:1010A0002B781BB90DF11700FCF7A8FDF1F76CFFC9
:1010B00030B92B78012B03D10DF11700FCF79EFD01
:1010C000F1F770FF30B92B78022B03D10DF1170027
:1010D000FCF794FDF1F772FF30B92B78032B03D1A5
:1010E0000DF11700FCF78AFDF1F776FF48B9F1F72B
:1010F0009FFF30B92B78042B03D10DF11700FCF7BB
:101100007DFDF1F7C9FF30B92B78052B03D10DF127
:101110001700FCF773FDF1F7B3FF30B92B78062BFE
:1011200003D10DF11700FCF769FDF1F763FF30B94A
:101130002B78072B03D10DF11700FCF75FFDF1F7BA
:1011400067FF30B92B78082B03D10DF11700FCF79E
:1011500055FD9DF81730002B2BD02B78082B23D86A
:10116000DFE803F005080D101316191C1F000020FE
:10117000344901E034490020F7F714FD16E000205F
:101180003249F9E700203249F6E700203149F3E718
:1011900000203149F0E700203049EDE700203049D8
:1011A000EAE700202F49E7E7F7F7C0FD2A782E4B42
:1011B0001A701E4F3B783D46092B40F0BD801F4BF7
:1011C0001B4F1978984611F001015CD1274E12226D
:1011D0003046EFF7E3F80123737415F09DFA10B968
:1011E0002278234B1A70237803B97374737C13B17C
:1011F000204B00221A70FCF7E3FC1D48717CFFF7BE
:10120000FFFD98F8003003F0FD0343F0010388F878
:101210000030194B1A788AB33A7000221A7032E003
:10122000EF1E00202C1A002033130020E01E0020A7
:10123000CC1D0020C31E0020041E0020E31E002041
:10124000D01E0020BA44030899440308DB44030875
:10125000FC4403081D4503083E4503085F45030899
:1012600080450308A1450308F1670020CE1D00203A
:10127000081E00202C130020981E002015F04CFAA8
:1012800008B930233B703B78884E13B93379112B62
:101290004ED1DFF86892FCF793FC854899F811105D
:1012A000FFF7AEFD824B1A78984622B1002010213C
:1012B0004A46FCF7DBF8237898F800407D4A24EA98
:1012C000030111707C4A23EA040111703A78A2F1FB
:1012D0005200C0B2012803D93079744F11280CD1C3
:1012E000002333711CB911B10133009311E10423C0
:1012F000F3702B7801332B701AE0432A18D1BBB955
:101300007C78ACB96D4BD879F4F7DCFF38B96C490F
:10131000F7F748FC0523FB7008332B7004E02046E8
:101320006849F7F73FFCFC70674A684B1A606CE14C
:101330005F48FCF7C1F868E10A2B31D15D4807F03E
:1013400059F8C6B2594C36B3E378042B02D10020C9
:101350005F4903E0022B04D15E490020F7F722FC2D
:1013600002E00BB90433E370314602225A48F7F722
:101370003FFC5A4B1E78232E00F0D3803046F7F7FF
:10138000CDFC002800F04181312E40F03E812B78C9
:1013900001332B7002E03B7801333B70042332E0D1
:1013A0000B2B32D1434807F00BF8C6B23F4C36B393
:1013B000E378042B02D10020494903E0022B04D139
:1013C00048490020F7F7EEFB02E00BB90433E37065
:1013D000314602224048F7F70BFC404B1E78232E83
:1013E00000F09F803046F7F799FC002800F00D814F
:1013F000312E40F00A812B7801332B7002E03B78CC
:1014000001333B700823E370FFE00C2B40F0FD80BC
:10141000284806F0BBFF0021C4B2264806F08CFF26
:10142000002C6DD0214EB3782BB9BE2014F0A0FE55
:10143000B3780133B370F3781C4A092B02D900202A
:101440001F4915E010D11D4B00241C70D470264B91
:10145000194A1849164801251C7014700C70047044
:101460000095019402949EE0082B04D11F490020AE
:10147000F7F798FB11E0062B02D100201C49F7E793
:10148000042B02D100201B49F2E7022B02D10020DD
:101490001949EDE70BB90833D370F378082B3CD822
:1014A0000D4821460222F7F7A3FB36E03313002054
:1014B000081E0020F11E0020E41E0020A21E0020B5
:1014C0000E3F03088A3E030848BB0208041E0020A2
:1014D000923F0308B33F0308F4010020CC1D002015
:1014E000503F0308713F0308CD1D0020AB3E0308A9
:1014F000CC3E0308ED3E03082F3F0308CE1D00201D
:10150000012543484349444A2B460095F2F728FBFE
:101510000095424B01941B7840E0414F3C78232CCE
:1015200002D1FCF775FB70E02046F7F7F7FB0028C7
:101530006BD0303CE4B2631EDBB2012B3C7039D877
:10154000022C364D1ED1E879F4F7BCFE002838D0C5
:101550002F48FCF717FB002833D1082246F64E012E
:10156000304800F0A2FC2A492E4813F094FF2D4980
:10157000082246F64E0000F092FC2A492A4813F051
:10158000A0FF06E0012322482249234A0093F2F7F4
:10159000E7FA01230024009301942B780293234857
:1015A0001D49234A1B4BFCF779FAF7F7BFFB214B88
:1015B0001C602AE0032C28D1184BD879F4F782FE5E
:1015C00010B90C23F37020E015F0A6F870B90446AA
:1015D0000F48214613F0A7FF28B1E02014F0C8FD02
:1015E000204614F001FE0134402CF1D1124A0023B0
:1015F0001370F3702B78114A01332B700D4B1A6066
:101600000F4B1A7842F006021A7007B0BDE8F0835B
:10161000331C0020CD1D0020F11E0020A21E002042
:10162000CC1D0020141A0020851A0020081E00205E
:10163000E41E0020041E00209E1E002048BB02085D
:10164000E31E0020194A00231360194A1948137039
:10165000194A1178037001F0F60163F30711117054
:10166000164A1748117863F301011170154A117871
:1016700063F3C5011170144A1370144A117801F014
:10168000FC0163F382011170114A1168037021F4A7
:10169000805163F3CF3111600E4A117801F0F401EB
:1016A00063F3820111700C4A93717047041E00208D
:1016B000C31E00209E1E0020E31E0020E51D00200A
:1016C000EE1E0020991E0020A11E0020B01E00204A
:1016D000083B0020AB3F0020331300202DE9F04FE2
:1016E0006A4B6B4D1970A0F11103DBB2012B87B06F
:1016F0000E46287006D8122801D1113800E00020CB
:10170000F4F7A8FE2B78522B0DD1F1F715FD28B96F
:10171000F1F706FD10B9F1F727FD20B15D4B1A78FE
:1017200042F008021A705C4B5C4C1B782BB92268A3
:101730005B4B9A4201D0FFF785FF2368002B40F0F6
:101740004081584F7B7803F02003DBB273B1564BD6
:1017500093F80080B8F1000F08D14AF6E90041463D
:1017600000F088FB3B6868F34D333B604F4B1878C3
:1017700010F01E0002D000204D4907E04D4B93F8B9
:1017800005909846B9F1000F05D04B4907B0BDE868
:10179000F04FF7F707BA494F97F801B0BA46BBF1D7
:1017A000000F2DD0BBF1070F15D94548F7F7A0F969
:1017B0004449B878652246F61573F7F73FF938784B
:1017C000072310F003007B700EBF3F4948463F4996
:1017D000F7F7E8F90CE0BBF1020F09D83848437875
:1017E00023B1F7F785F987F8019093E202237B7024
:1017F0001020334A014607B0BDE8F04FF7F78AB929
:10180000334B9A795AB183F806B000F0A1FC8E20D0
:10181000594601225B46CDF800B0F0F775FF002075
:10182000F1F7ECFD2B4A2C4913782C4843F00603C2
:10183000137000230B702A4923600B7088F8013065
:1018400088F80430037029337343264F9146F95CBE
:101850008346C1F3C00111B93046FFF78BF8292345
:1018600003FB06777B7913F0100F04D02A78133A24
:10187000D2B2032A3AD913F0200F5DD02B78442B33
:1018800034D031D8232B31D02A2B2EE0961E0020C5
:10189000CC1D0020821A0020EF1E0020041E002014
:1018A00048BB0208083B00202C1A0020F95C0020ED
:1018B0006314030833130020C24503089B1E002055
:1018C000F41E0020FB1E00206B1503084A150308B8
:1018D000A21E0020E31E0020C31E0020981E002030
:1018E000931E0020793D0020552B25D1844B1B7879
:1018F00013BB844B1F78FFB943F6DB2000F0C4FA1A
:101900000128014618D188F801003F200591FFF712
:1019100019F899F80030304667F3410389F8003030
:10192000059909F01BF9F7F701FA774B2360774B1C
:101930001F602B788BF800302B78432B0AD1714B2A
:101940001B783BB90121724B88F8011030462360A7
:1019500009F004F928781738C3B2072B27D86D4946
:10196000FF220BF0AFF89AF800106B4B60F3010107
:101970008AF8001001F00301022918D00122032087
:1019800041B1009001929B7868309B18029300212E
:10199000033206E0009001929B786C2001330293A1
:1019A00004220B4600F0EEFAFF238AF8013098F883
:1019B0000730002B00F0AE8152232B70574B0022D2
:1019C000DA712268524B9A4250D12878A0F1430331
:1019D000DAB2122A22D8524A5BB29A401ED5432864
:1019E00040F09881464B1B78002B40F0938100F02B
:1019F000B3FD4C4B48B11A7803201109013191FB1A
:101A0000F0F000EB4000091A04E01A7811090131E6
:101A100001F0070161F307121A707BE1F7F77EF915
:101A2000002823D03F4F3B7813F0F00108D161F339
:101A300007133B703C4B21601A7842F008020EE01D
:101A4000102913D100F088FD80B13B7800216FF39D
:101A500007133B70344B21601A7842F01002304675
:101A60001A7007B0BDE8F04FFEF784BF2F4B1E2160
:101A70001A78254F61F346021A702B78232B1CD15C
:101A80002368BB4219D12A4B292202FB06367379FF
:101A900013F0100F11D0274B1B7873B1264EF7F7B8
:101AA00045F9FCF7B5F8F07900F56A507C3000F0A4
:101AB000EBF93070AA20F1F7A1FC1A4E337813F03D
:101AC000010F41D02368BB420BD01C4A934208D07F
:101AD000FEF70CFF28B9FEF71FFF10B9AA30F1F787
:101AE0008DFC2268164B9A4202D10020F1F786FC49
:101AF0002B78522B40F0D3805322124BC7E000BF0B
:101B00002C1A0020001E00202CBB0208D01E002032
:101B100040B602089D1E00209B1E002033130020AB
:101B2000002000C0E31E0020B01E0020611F002026
:101B3000793D0020C31E0020A21E002048BB0208E1
:101B400064BB0208CC1D00202368BB420BD0734A43
:101B5000934208D0FEF7CAFE28B9FEF7DDFE10B9A1
:101B6000AA30F1F74BFC2B78552B1ED1FEF76AFEFD
:101B700033786B4843F0060333708378694F03F082
:101B80000203DBB24BB1F6F7B3FF23681868FAF72C
:101B90001DF93B786FF341033B706348837803F092
:101BA0000203DBB20BB1F6F7A3FF2B78442B1ED157
:101BB000FEF7F8FD33785A4843F006033370837814
:101BC000584F03F00203DBB24BB1F6F791FF2368E5
:101BD0001868FAF7FBF83B786FF341033B70524803
:101BE000837803F00203DBB20BB1F6F781FF2B78A9
:101BF000522B09D13378002243F0010333704B4B51
